:100000000C9436170C946F170C946F170C946F1791
:100010000C94A7420C94A7420C94A7420C94A742BC
:100020000C946F170C946F170C946F170C946F1738
:100030000C946F170C949E2A0C946F170C946F17E6
:100040000C946F170C94EA260C94ABCE0C946F179B
:100050000C947F8B0C94758B0C946F170C946F170A
:100060000C946F170C946F170C946F170C946F17F8
:100070000C946F170C946F170C946F170C946F17E8
:100080000C9468800C946F170C946F174E414E4976
:100090004E495459494E46CDCCCC3D0AD7233C1746
:1000A000B7D13877CC2B329595E6241FB14F0A0093
:1000B0000020410000C84200401C4620BCBE4CCA83
:1000C0001B0E5AAEC59D7400407A10F35A00A07200
:1000D0004E18090010A5D4E80000E8764817000083
:1000E000E40B54020000CA9A3B000000E1F5050051
:1000F0000080969800000040420F000000A086019A
:10010000000000102700000000E803000000006469
:1001100000000000000A00000000000100000000D4
:10012000002C76D888DC674F0823DFC1DFAE59E1A9
:10013000B1B796E5E3E453C63AE651997696E8E618
:10014000C28426EB898C9B62ED407C6FFCEFBC9CEB
:100150009F40F2BAA56FA5F490055A2AF75C936BFD
:100160006CF9676DC11BFCE0E40D47FEF520E6B5B8
:1001700000D0ED902E0300943577050080841E0892
:100180000000204E0A000000C80C333333330F98B0
:100190006E12831141EF8D2114893BE65516CFFE77
:1001A000E6DB18D1844B381BF77C1D901DA4BBE403
:1001B00024203284725E228100C9F124ECA1E53D45
:1001C000275045544700504C41005072696E7420CE
:1001D00041626F72746564004D3235005061757311
:1001E000696E672E2E2E004D323400454550524F19
:1001F0004D2056657273696F6E204572726F720082
:10020000454550524F4D20496E64657820457272C5
:100210006F7200454550524F4D2043524320457266
:10022000726F72003F0049676E6F726500526573AE
:10023000657400496E697469616C697A6520454529
:1002400050524F4D0000FE0003FF8007C7C007015A
:10025000E00000E00000F00000700400700E00708C
:100260001F00703F80F00E00E00F01E007C7C003E1
:10027000FF8000FE0000FE0003FF8007C7C00F01E3
:10028000E00E00E03F80F01F00700E007004007070
:100290000000700000F00000E00701E007C7C003A5
:1002A000FF8000FE000E000E000E000E000E000E7D
:1002B000000E000E007FC03F801F000E00040004EF
:1002C000000E001F003F807FC00E000E000E000ECB
:1002D000000E000E000E000E00FFFFFF7F80FFC02B
:1002E000FFC0FFC07F807F80FFC0FFC0FFC03F0016
:1002F0001E000C0050726F6265205A204F666673B4
:1003000065740020082046616374002008204D6158
:1003100078002008204D696E004F6666004F6E0021
:100320004175746F74656D700045207374657073EA
:100330002F6D6D005A2053746570732F6D6D0059C9
:100340002053746570732F6D6D0058205374657061
:10035000732F6D6D00416476616E63656420536533
:100360007474696E67730054656D7065726174753D
:1003700072650053746570732F6D6D00436F6E6608
:10038000696775726174696F6E003F004E657874BD
:1003900020436F726E657200446F6E65004E657823
:1003A0007400486F6D696E672058595A0053746F16
:1003B00072652053657474696E6773004C6F616475
:1003C0002053657474696E677300426564205472CB
:1003D000616D6D696E670050726F6265205A204FC3
:1003E0006666736574004661646520486569676880
:1003F00074004F6666004F6E00426564204C65765F
:10040000656C696E67004C6576656C2042656400BA
:100410004732394E00473239004175746F20486FBA
:100420006D65004D6F74696F6E00526573746F7205
:10043000652044656661756C7473004C6F6164205F
:1004400053657474696E67730053746F72652053DB
:10045000657474696E67730050726F6265205A200C
:100460004F666673657400416476616E63656420EF
:1004700053657474696E6773004D61696E003F0067
:100480004261636B0053746F70004D3232004174EF
:1004900074616368204D65646961004D32310050BC
:1004A00072696E742066726F6D204D6564696100BB
:1004B00052656C65617365204D6564696100436FC9
:1004C0006E66696775726174696F6E0054656D70F0
:1004D00065726174757265004D6F74696F6E00525C
:1004E0006573756D65205072696E740054756E6524
:1004F0000053746F70205072696E74005061757390
:1005000065205072696E7400496E666F2053637285
:1005100065656E000A4D3234004D3233202573007C
:100520003F005374617274205072696E74004361AD
:100530006E63656C005072696E740043616E6E6F1D
:100540007420656E746572207375626469723A20F6
:100550000002202E2E000152656672657368004D00
:1005600061696E002100486F74656E6420746F6F5E
:1005700020636F6C64004261636B0050726F63654F
:100580006564004D6F74696F6E0044697361626CDD
:1005900065205374657070657273004D3834004285
:1005A0006564204C6576656C696E67004175746F93
:1005B00020486F6D6500473238004D61696E00500C
:1005C000726568656174202420426564005072651C
:1005D00068656174202420456E640054656D706503
:1005E00072617475726500C601C101436F6F6C64FE
:1005F0006F776E00507265686561742024004661F3
:100600006E20537065656400426564004E6F7A7AAF
:100610006C65004D61696E0050726F6265205A20F2
:100620004F666673657400466C6F770046616E2096
:10063000537065656400426564004E6F7A7A6C653C
:10064000005370656564004D61696E00486F6D69A7
:100650006E67204661696C6564006F70656E00545A
:100660005249474745524544003A20007A5F6D6938
:100670006E00795F6D696E00785F6D696E0052651E
:10068000706F7274696E6720656E6473746F70202A
:100690007374617475730A0020746F6F206C6F6ED1
:1006A0006720657874727573696F6E2070726576F5
:1006B000656E7465640A0020636F6C6420657874ED
:1006C000727573696F6E2070726576656E7465649D
:1006D0000A00486F6D6520257325732573204669D0
:1006E000727374005761726E696E673A20486F6D5D
:1006F000696E672042756D702044697669736F7208
:10070000203C20310A000202040000E0C00000008A
:10071000C000000000000068430000634300007A4E
:10072000430000A0400000A04000000040FFFDFC8E
:10073000FAF8F6F4F2F0EEECEAE9E7E5E3E1E0DE00
:10074000DCDAD9D7D5D4D2D0CFCDCBCAC8C7C5C3B0
:10075000C2C0BFBDBCBAB9B7B6B4B3B2B0AFADAC2E
:10076000AAA9A8A6A5A4A2A1A09E9D9C9A99989783
:1007700095949392908F8E8D8B8A898887868483B7
:100780008281807F7E7D7B7A7978777675747372CB
:1007900071706F6E6D6C6B6A6968676665646362C1
:1007A00061605F5E5D5C5B5A5958585756555453AB
:1007B000525150504F4E4D4C4B4A4A49484746467D
:1007C000454443424241403F3E3E3D3C3B3B3A393B
:1007D000383837363535343332323130302F2E2EEB
:1007E0002D2C2B2B2A29292827272625252423238E
:1007F00022212120201F1E1E1D1C1C1B1B1A191923
:100800001818171616151514131312121111100FAC
:100810000F0E0E0D0D0C0C0B0A0A0909080807072C
:10082000060605050404030302020100000000009F
:1008300001000000010000800055555500000040F7
:100840000033333300AAAA2A004992240000002072
:1008500000C7711C0099991900D14517005555150D
:10086000003BB113002449120011111100000010C7
:10087000000F0F0F00E3380E0043790D00CCCC0CB5
:1008800000C3300C00E8A20B0064210B00AAAA0AE6
:1008900000703D0A009DD80900427B09009224099E
:1008A00000DCD30800888808001042080000000817
:1008B00000F0C107008787070075500700711C070B
:1008C000003EEB0600A1BC060069900600666606C5
:1008D00000703E06006118060017F4050074D1058B
:1008E000005BB00500B29005006272050055550529
:1008F0000078390500B81E0500050505004EEC041A
:100900000087D40400A1BD040090A704004992040C
:1009100000C17D0400EE690400C75604004444048D
:10092000005C3204000821040041100400000004AF
:10093000003FF00300F8E0030026D20300C3C30326
:1009400000CCB503003AA803000A9B0300388E03CD
:1009500000C08103009F750300D0690300505E034F
:10096000001D53030034480300913D03003333035B
:100970000016290300381F030097150300300C03ED
:1009800000030303000BFA020049F10200BAE80277
:10099000005CE002002DD802002DD0020059C802F0
:1009A00000B0C0020031B90200DAB10200AAAA0206
:1009B00000A0A30200BC9C0200FA9502005C8F021A
:1009C00000DF88020082820200457C020027760256
:1009D0000027700200436A02007C640200D05E02BD
:1009E000003F590200C8530200000061430000614B
:1009F0004300007A430000E0C0000000C000000097
:100A00000053657474696E67732053746F72656404
:100A1000000000FA430000FA430000A0400000C8B4
:100A2000410000A0420000A0420000C8430080C076
:100A300043F4010000F4010000640000008813008A
:100A40000024F4D43050C38E20C2A24017828B7091
:100A500011127A910D816CD90AA861E108C7586614
:100A600007615143061E4B5D05C145A7041A41119C
:100A700004093D9803713931034036DB0265339137
:100A800002D4305402802E1D02632CEE01752AC55B
:100A900001B028A001102781018F2564012B244B70
:100AA00001E0223401AC211F018D200D01801FFCCB
:100AB00000841EED00971DDF00B81CD200E61BC6A7
:100AC00000201BBC00641AB200B219A8000A19A0C9
:100AD000006A189900D117910040178B00B5168451
:100AE0000031167E00B31579003A157300C7146FF4
:100AF0000058146A00EE1366008813630025135E25
:100B000000C7125B006C12570015125400C111513E
:100B10000070114F0021114B00D61049008D104775
:100B2000004610440002104200C00F4000800F3EFB
:100B300000420F3C00060F3B00CB0E3800930E37EF
:100B4000005C0E3500270E3400F30D3200C10D316C
:100B500000900D3000600D2E00320D2D00050D2C83
:100B600000D90C2B00AE0C2900850C29005C0C2749
:100B700000350C27000E0C2600E80B2400C40B24C3
:100B800000A00B23007D0B23005A0B2100390B2101
:100B900000180B2000F80A1F00D90A1E00BB0A1E0D
:100BA000009D0A1D00800A1D00630A1C00470A1BE5
:100BB000002C0A1B00110A1A00F7091A00DD091996
:100BC00000C4091900AB091900920917007B091824
:100BD00000630917004C0916003609160020091693
:100BE000000A091500F5081500E0081400CC0814E7
:100BF00000B8081400A4081400900813007D08121F
:100C0000006B08130058081200460812003408113F
:100C100000230811001208110001081100F007104C
:100C200000E0071000D0071000C0071000B0070F49
:100C300000A107100091070E0083070F0074070F33
:100C40000065070E0057070E0049070E003B070D11
:100C5000002E070E0020070D0013070D0006070DDC
:100C600000F9060C00ED060D00E0060C00D4060CA1
:100C700000C8060C00BC060C00B0060C00A4060B55
:100C80000099060C008D060B0082060B0077060B00
:100C9000006C060B0061060A0057060B004C060AA2
:100CA0000042060A0038060A002E060A0024060A38
:100CB000001A060A001006090007060A00FD0509C9
:100CC00000F4050900EB050900E2050900D9050952
:100CD00000D0050900C7050900BE050900B50508D3
:100CE00000AD050800A50509009C0508009405084D
:100CF000008C050800840508007C050800740508C0
:100D0000006C050700650508005D0507005605082D
:100D1000004E050700470507004005080038050795
:100D200000310507002A050700230507001C0506FA
:100D300000160507000F0507000805060002050755
:100D400000FB040600F5040700EE040600E80406B4
:100D500000E2040700DB040600D5040600CF040609
:100D600000C9040600C3040600BD040600B704065B
:100D700000B1040500AC040600A6040600A00405AA
:100D8000009B04060095040500900406008A0405F3
:100D90000085040500800406007A0405007504053A
:100DA00000700405006B040500660405006104057D
:100DB000005C04050057040500520405004D0405BD
:100DC0000048040500430405003E0404003A0405FD
:100DD0000035040500300404002C04050027040439
:100DE00000230405001E0404001A04040016040570
:100DF00000110404000D04040009040500040404A7
:100E00000000040400FC030400F8030400F40304DD
:100E100000F0030400EC030400E8030400E403040E
:100E200000E0030400DC030400D8030400D403043E
:100E300000D0030400CC030400C8030300C503036F
:100E40000024F404D9201BC40C5C0E9804C4095F70
:100E50000265077101F405F900FB04B3004804873B
:100E600000C10369005803550003034500BE023A60
:100E7000008402310053022A0029022500040220C6
:100E800000E4011C00C8011900AF0117009801140B
:100E90000084011300710110006101100051010E66
:100EA0000043010D0036010B002B010B0020010B4C
:100EB00000150109000C01090003010800FB0008EE
:100EC00000F3000800EB000700E4000600DE000667
:100ED00000D8000600D2000600CC000500C70005BF
:100EE00000C2000500BD000400B9000400B5000404
:100EF00000B1000400AD000400A9000400A5000337
:100F000000A20003009F0004009B00030098000360
:100F1000009500020093000300900003008D000282
:100F2000008B00030088000200860002008400039A
:100F300000810002007F0002007D0002007B0002B1
:100F400000790002007700010076000200740002C0
:100F50000072000100710002006F0002006D0001CC
:100F6000006C0002006A00010069000200670001D5
:100F700000660001006500010064000200620001DB
:100F80000061000100600001005F0002005D0001DF
:100F9000005C0001005B0001005A000100590001E3
:100FA00000580001005700010056000100550001E3
:100FB00000540001005300000053000100520001E2
:100FC0000051000100500001004F0001004E0000E0
:100FD000004E0001004D0001004C0001004B0000DC
:100FE000004B0001004A00010049000100480000D8
:100FF00000480001004700010046000000460001D3
:1010000000450000004500010044000100430000CD
:1010100000430001004200000042000100410000C6
:101020000041000100400001003F0000003F0001BE
:10103000003E0000003E0001003D0000003D0001B8
:10104000003C0000003C0000003C0001003B0000B0
:10105000003B0001003A0000003A000100390000A6
:10106000003900010038000000380000003800019D
:101070000037000000370001003600000036000095
:101080000036000100350000003500000035000189
:101090000034000000340000003400010033000080
:1010A0000033000000330001003200000032000075
:1010B0000032000100310000003100000031000169
:1010C000003000000030000000300001002F000060
:1010D000002F0000002F0000002F0001002E000054
:1010E000002E0000002E0001002D0000002D000049
:1010F000002D0000002D0001002C0000002C00003D
:10110000002C0000002C0001002B0000002B000030
:10111000002B0000002B0001002A0000002A000024
:10112000002A0000002A0001002900000029000018
:10113000002900000029000000290001002800000B
:1011400000280000002800000028000000280001FE
:1011500000270000002700000027000000270000F3
:1011600000270001002600000026000000260000E5
:1011700000260000002600010025000000250000D8
:1011800000250000002500000025000000250001CA
:1011900000240000002400000024000000240000BF
:1011A00000240001002300000023000000230000B1
:1011B00000230000002300000023000000230001A2
:1011C0000022000000220000002200000022000097
:1011D0000022000000220001002100000021000088
:1011E000002100000021000000210000002100007B
:1011F000002100010020000000200000002000006D
:10120000002000000020000000200000002000005E
:1012100000200001001F0000001F0000001F000050
:10122000001F0000001F0000001F0000001F000141
:10123000001E0000001E0000001E0000001E000036
:1012400000393000003325000087190000B00F007E
:1012500000DB080000BD040000740200003F010034
:101260000020436F756E7420583A00426564004553
:1012700031004500626564002C2073797374656DDC
:101280002073746F707065642120486561746572A5
:101290005F49443A20004572723A204D4158544506
:1012A0004D50004D415854454D5020747269676748
:1012B000657265640048656174696E67204661699E
:1012C0006C65640048656174696E67206661696C6D
:1012D0006564004572723A204D494E54454D5000A8
:1012E0004D494E54454D502074726967676572656B
:1012F0006400544845524D414C2052554E4157418F
:101300005900546865726D616C2052756E61776129
:101310007900202F002042403A0020403A007C3CD7
:101320003E5E2B3D3F2F5B5D3B2C2A225C00434FF2
:101330004D4D554E49434154494F4E004452595228
:10134000554E004552524F525300494E464F0045AC
:1013500043484F0053544F505045442E2000507284
:10136000696E7465722073746F7070656420647543
:101370006520746F206572726F72732E20466978D3
:1013800020746865206572726F7220616E642075CA
:101390007365204D39393920746F2072657374611B
:1013A00072742E202854656D706572617475726553
:1013B0002069732072657365742E205365742069EB
:1013C00074206166746572207265737461727469E9
:1013D0006E67290A004E6F20436865636B73756DF5
:1013E0002077697468206C696E65206E756D626522
:1013F000722C204C617374204C696E653A20004E4B
:101400006F20436865636B73756D2077697468201E
:101410006C696E65206E756D6265722C204C61730F
:1014200074204C696E653A2000636865636B737560
:101430006D206D69736D617463682C204C617374E9
:10144000204C696E653A20004C696E65204E756DC2
:10145000626572206973206E6F74204C6173742012
:101460004C696E65204E756D6265722B312C204C77
:10147000617374204C696E653A20004D3131300043
:1014800053657269616C20737461747573206D6942
:10149000736D617463680A0053442072656164204F
:1014A0006572726F720A002121204B494C4C2063F7
:1014B000617573656420627920746F6F206D756348
:1014C0006820696E6163746976652074696D652052
:1014D0002D2063757272656E7420636F6D6D616E21
:1014E000643A20004D6564696120496E73657274C9
:1014F000656400627573793A207061757365642064
:10150000666F7220696E7075740A00627573793A3D
:101510002070617573656420666F722075736572E3
:101520000A00627573793A2070726F63657373692C
:101530006E670A00506C656173652052657365744F
:10154000005052494E5445522048414C54454400A5
:1015500025533A202553004B494C4C45442E20003E
:101560005072696E7465722068616C7465642E20B7
:101570006B696C6C28292063616C6C6564210A00BE
:101580006563686F3A004572726F723A004F464663
:10159000004F4E0042696C696E656172204C657641
:1015A000656C696E6720477269643A0A004F464667
:1015B0000A004661646520486569676874200042D6
:1015C0006564204C6576656C696E672000466169CC
:1015D0006C656420746F20656E61626C6520426585
:1015E00064204C6576656C696E670A00496E7661A9
:1015F0006C6964206D6573682E0A0050726F6269B1
:101600006E6720506F696E740025532025692F2561
:1016100069002E0A002F0050726F62696E67206D9C
:1016200065736820706F696E7420002028445259D9
:1016300052554E2900473239204175746F2042655A
:1016400064204C6576656C696E67003F20284C2CE1
:10165000522C462C4229206F7574206F6620626FD1
:10166000756E64732E0A003F2856296572626F7387
:1016700065206C6576656C20696D706C6175736949
:10168000626C652028302D34292E0A0042616420C6
:101690005A2076616C75650A004E6F2062696C692C
:1016A0006E65617220677269640A004732384C3097
:1016B0000020204D3230312058004D6178204163A8
:1016C00063656C65726174696F6E2028756E6974EC
:1016D000732F7332290020204D3230332058004DB3
:1016E0006178206665656472617465732028756E23
:1016F0006974732F73290020520020204D3230343A
:10170000205000416363656C65726174696F6E207F
:1017100028756E6974732F7332292028503C7072BB
:10172000696E742D616363656C3E20523C72657412
:10173000726163742D616363656C3E20543C747206
:101740006176656C2D616363656C3E2900204A00FB
:1017500020540020530020204D32303520420041DB
:101760006476616E6365642028423C6D696E5F73C8
:1017700065676D656E745F74696D655F75733E2036
:10178000533C6D696E5F66656564726174653E2089
:10179000543C6D696E5F74726176656C5F666565F9
:1017A00064726174653E204A3C6A756E635F64656D
:1017B000763E2900205500204C0020204D32383143
:1017C000205000536572766F20416E676C65730020
:1017D00020440020490020204D3330312050004863
:1017E0006F74656E64205049440020440020490015
:1017F00020204D333034205000426564205049444D
:10180000002E0A00206E6F742064697361626C653B
:10181000642E2053686172656420776974680020C3
:101820003B204C6576656C696E67200020204D3446
:1018300032302053004175746F20426564204C653E
:1018400076656C696E6700204600204200204800E3
:1018500020204D3134352053004D6174657269612B
:101860006C2068656174757020706172616D65745B
:1018700065727300204A00202047323920572049E2
:101880000020204D3134392043203B20556E6974AF
:101890007320696E2043656C736975730A00546523
:1018A0006D706572617475726520556E6974730030
:1018B0002020473231203B004C696E656172205513
:1018C0006E6974730020496E76616C696420657876
:1018D0007472756465722000536C6565702E2E2ECF
:1018E000005A2050726F6265205061737420426507
:1018F000640A005A2050726F626520506173742030
:1019000042656400205A3A200020593A200042657E
:101910006420583A20004D65736820706F696E74BA
:10192000206F7574206F662072616E67650A0043D0
:101930006C69636B20746F20526573756D652E2E14
:101940002E00616C736F20656E61626C6564290A9C
:10195000004E6F204D6F76652E004E6F206D6564D2
:1019600069610A00456E642066696C65206C697364
:10197000740A00426567696E2066696C65206C694F
:1019800073740A00286E6F2066696C6529004E6FBB
:1019900074205344207072696E74696E670A005334
:1019A00044207072696E74696E6720627974652074
:1019B0000043757272656E742066696C653A20002A
:1019C0002E0A0044656C6574696F6E206661696CEF
:1019D00065642C2046696C653A200046696C652078
:1019E00064656C657465643A002569730025696DEA
:1019F00020256973002569682025696D2025697394
:101A000000256964202569682025696D2025697392
:101A10000025697920256964202569682025696D7C
:101A200020256973005072696E742074696D653A7F
:101A300020006F6B006F6666004F134A1343133C20
:101A4000132E1344454255473A004D31313220534D
:101A5000687574646F776E004D3131332053004DDB
:101A6000656761205A65726F20322E30204F4646DE
:101A70002E00434F4E4649475F4558504F52540041
:101A80004D4541545041434B00434F4F4C45525FED
:101A900054454D5045524154555245004348414DDF
:101AA0004245525F54454D504552415455524500B0
:101AB000424142595354455050494E4700415243C8
:101AC00053004D4F54494F4E5F4D4F4445530054C2
:101AD0004845524D414C5F50524F54454354494F35
:101AE0004E00455854454E4445445F4D3230004CFD
:101AF0004F4E475F46494C454E414D450041555478
:101B00004F5245504F52545F53445F5354415455C4
:101B1000530053445F575249544500524550454184
:101B200054005344434152440050524F4D50545F6F
:101B3000535550504F525400484F53545F414354F3
:101B4000494F4E5F434F4D4D414E445300454D4527
:101B50005247454E43595F5041525345520043410D
:101B600053455F4C494748545F4252494748544E99
:101B700045535300544F47474C455F4C49474854E1
:101B80005300534F4654574152455F504F574552AB
:101B9000004255494C445F50455243454E54004C19
:101BA0004556454C494E475F44415441005A5F50A9
:101BB000524F42450052554E4F5554004155544FD7
:101BC0004C4556454C005052494E545F4A4F4200D6
:101BD00050524F4752455353004155544F52455070
:101BE0004F52545F54454D50004155544F5245504B
:101BF0004F52545F504F5300564F4C554D45545221
:101C0000494300454550524F4D0042494E415259BB
:101C10005F46494C455F5452414E5346455200532E
:101C2000455249414C5F584F4E5F584F464600461B
:101C300049524D574152455F4E414D453A4D6172B3
:101C40006C696E20322E302E392E332D6B6164314B
:101C5000202844656320323720323032312031333E
:101C60003A34353A32322920534F555243455F4377
:101C70004F44455F55524C3A6769746875622E63EC
:101C80006F6D2F6B61642F4D61726C696E205052C5
:101C90004F544F434F4C5F56455253494F4E3A3184
:101CA0002E30204D414348494E455F545950453AE6
:101CB0004D656761205A65726F20322E302045587D
:101CC0005452554445525F434F554E543A31205576
:101CD0005549443A64626663636435352D656262D2
:101CE000612D343631352D616264372D31393661DD
:101CF00061343338663330340A002F2F004D3134CD
:101D00003520533C696E6465783E206F7574206F92
:101D1000662072616E67652028302D31290A003FE8
:101D20004A206F7574206F662072616E6765202887
:101D3000302E303120746F20302E33290A00205885
:101D40000020204D61783A2000200020204D696E4F
:101D50003A2000203B200020204D3231312053001A
:101D6000536F667420656E6473746F7073004652AF
:101D70003A0020466C6F773A2000206F7574206F10
:101D8000662072616E67650A00536572766F200087
:101D90003A200020536572766F2000206F75742002
:101DA0006F662072616E67650A00536572766F20F8
:101DB00000206F7574206F662072616E67650A007F
:101DC000536572766F200050726F6265204F6666B1
:101DD000736574205A0050726F6265204F66667397
:101DE0006574205A0064697300656E0043290A0017
:101DF00061626C656420286D696E2074656D702069
:101E000000436F6C6420657874727564657320613B
:101E1000726520004D34323120696E636F727265D5
:101E2000637420706172616D657465722075736191
:101E300067650A004D65736820706F696E74206F66
:101E40007574206F662072616E67650A00454550A3
:101E5000524F4D204F4B0A00290A0020746F20007A
:101E60003F5A206F7574206F662072616E6765201F
:101E70002800290A0020746F20003F59206F7574D4
:101E8000206F662072616E676520282D00290A0088
:101E900020746F20003F58206F7574206F66207289
:101EA000616E676520282D004D383400446F6E65E3
:101EB000207072696E74696E672066696C650A00CD
:101EC0004D3737004D333100496E76616C696420BF
:101ED00065787472756465720A004361703A002017
:101EE000286D6D2900203B0020204D3835312058C9
:101EF000005A2D50726F6265204F666673657400DC
:101F0000436F6F6C696E672E2E2E00486561746991
:101F10006E672E2E2E0045312025530020573A00A3
:101F200020573A0042656420436F6F6C696E672EDC
:101F30002E2E004265642048656174696E672E2EFE
:101F40002E0023646566696E652044454641554C04
:101F5000545F00626564004B6420004B6920004BB5
:101F6000702000504944204175746F74756E65206F
:101F700066696E69736865642120507574207468A1
:101F800065206C617374204B702C204B6920616E4E
:101F900064204B6420636F6E7374616E747320668B
:101FA000726F6D2062656C6F7720696E746F20436D
:101FB0006F6E66696775726174696F6E2E680A006C
:101FC000504944204175746F74756E65206661696F
:101FD0006C6564212074696D656F75740A005049E1
:101FE00044204175746F74756E65206661696C6517
:101FF00064212054656D706572617475726520741A
:102000006F6F20686967680A00504944204379630C
:102010006C65730025532025692F256900204B64CA
:102020003A2000204B693A2000204B703A200020D3
:10203000436C617373696320504944200A00204E49
:102040006F206F76657273686F6F740A0020547525
:102050003A2000204B753A2000206D61783A20002C
:10206000206D696E3A200020643A20002062696188
:10207000733A20005761697420666F722068656149
:10208000742075702E2E2E00504944204175746FB7
:1020900074756E652073746172740A00504944202F
:1020A0004175746F74756E65206661696C65642135
:1020B0002054656D706572617475726520746F6F00
:1020C00020686967680A00504944204175746F743C
:1020D000756E6500504944204175746F74756E6566
:1020E000206661696C6564212042616420686561D5
:1020F0007465722069640A004572723A20757466CC
:102100003820666F6E74206E6F7420696E69746912
:10211000616C697A65642E004572723A2075746646
:102120003820666F6E74206E6F7420696E697469F2
:10213000616C697A65642E004572723A2075746626
:102140003820666F6E74206E6F7420696E697469D2
:10215000616C697A65642E0042656400456E636C4B
:102160006F73757265002568753A253032687500A1
:1021700025303268753A253032687500253032686E
:10218000752725303268750020202020202020006F
:102190002020202000657272001FE02010201020F7
:1021A0001010201020201020103030084004800330
:1021B000001FE03FF03FF03FF01FE01FE03FF03F27
:1021C000F03FF00FC0078003003FFFF03800703091
:1021D000FC3020FC102078102030102C00D02E3144
:1021E000D02F7BD02F7BD02E31D02C00D0203010A0
:1021F00020781020FC1030FC303800703FFFF03F9A
:10220000FFF03800703186302387102787902F87A2
:10221000D02F03D0203010207810207810203010DC
:102220002F03D02F87D0278790238710318630380F
:1022300000703FFFF01FFFF81FFFF8041040020876
:1022400020020820041040082080104100104100A6
:102250000820800410400000001FFFF81FFFF80056
:102260001DC43F0000000C86198000000D0E19806F
:1022700000000F0B198000000D9F198000000DD386
:10228000998000001CFBFF0000000000000000001F
:102290000000000000F380001F800077000019801C
:1022A000005B1CF6131DAE5B35AB0635FB5B3DA733
:1022B0000CBD9B4B30EB19B19BE39D8E9F9D8E0017
:1022C00001E00000000001200000000001E000002B
:1022D00000000C0F00FE07022503BB017FFE08FE75
:1022E00008FE05080806000040F0C88888987810A5
:1022F000050808060000C0F88888888888F8050561
:10230000050600012030F8302005080806000020EE
:1023100070F820202020E00509090600FF2070A8A1
:10232000A8B888887020070505070001D86C366CAE
:10233000D80509090600FFF8A88888888888A8F8C1
:10234000050A0A0600FE205050505088A8A8887040
:1023500003030306000340A040FFFFFFFFFFFFFF52
:10236000FFFFFFFFFFFFFFFFFFFFFFFFFFFFFF007C
:1023700000000605FF0107070602008080808080BC
:102380000080030303060105A0A0A00506060600C1
:102390000050F85050F8500509090600FF2070A8B9
:1023A000A07028A87020050707060000C8C81020E4
:1023B00040989805070706000040A0A040A8906834
:1023C0000103030602058080800309090601FF203E
:1023D00040408080804040200309090601FF804082
:1023E0004020202040408005070706000020A870FC
:1023F0002070A8200505050600012020F8202002F5
:1024000003030601FFC04080050101060003F80236
:102410000202060100C0C0050707060000081010F0
:1024200020404080050707060000708898A8C888EB
:102430007003070706010040C040404040E0050728
:1024400007060000708808102040F80507070600FE
:1024500000F80810300888700507070600001030E3
:102460005090F81010050707060000F880F00808E3
:102470008870050707060000304080F088887005E6
:102480000707060000F8081010202020050707069F
:102490000000708888708888700507070600007043
:1024A000888878081060020505060100C0C000C0D9
:1024B000C00206060601FFC0C000C040800305053B
:1024C0000601012040804020050303060002F800B9
:1024D000F803050506010180402040800507070636
:1024E00000007088102020002005070706000070FB
:1024F00088B8A8B88070050707060000708888F8BB
:10250000888888050707060000F04848704848F0AA
:10251000050707060000708880808088700507071F
:10252000060000F04848484848F005070706000044
:10253000F88080F08080F8050707060000F88080AA
:10254000F0808080050707060000708880809888EA
:1025500070050707060000888888F88888880307C0
:1025600007060100E04040404040E0050707060044
:1025700000381010101090600507070600008890C2
:10258000A0C0A0908805070706000080808080809A
:1025900080F805070706000088D8A888888888057D
:1025A00007070600008888C8A898888805070706D6
:1025B000000070888888888870050707060000F08A
:1025C0008888F0808080050707060000708888886A
:1025D000A89068050707060000F08888F0A090889A
:1025E00005070706000070888070088870050707D7
:1025F000060000F820202020202005070706000004
:102600008888888888887005070706000088888879
:102610008850502005070706000088888888A8A8E9
:102620005005070706000088885020508888050755
:102630000706000088885020202020050707060094
:1026400000F80810204080F80309090601FFE08027
:10265000808080808080E005070706000080404081
:10266000201010080309090601FFE0202020202087
:102670002020E0050303060005205088050101061F
:1026800000FEF8030303060105804020050505064A
:10269000000070087888780507070600008080F041
:1026A000888888F005050506000070808088700520
:1026B0000707060000080878888888780505050659
:1026C00000007088F0807005070706000030484061
:1026D000E04040400507070600FE708888887808BB
:1026E000700507070600008080F088888888030747
:1026F000070601004000C0404040E004090906010F
:10270000FE10003010101010906005070706000042
:1027100080808890E09088030707060100C0404051
:10272000404040E0050505060000D0A8A8A8A8057F
:102730000505060000B0C888888805050506000064
:1027400070888888700507070600FEF0888888F082
:1027500080800507070600FE7888888878080805C5
:102760000505060000B0C88080800505050600004C
:1027700078807008F00507070600002020F8202068
:102780002018050505060000888888986805050555
:102790000600008888885020050505060000888806
:1027A000A8A8500505050600008850205088050798
:1027B000070600FE88888850204080050505060031
:1027C00000F8102040F80309090601FF20404040AE
:1027D00080404040200109090602FF8080808080FF
:1027E000808080800309090601FF8040404020402E
:1027F00040408005030306000248A890FF43616E35
:102800006E6F74206F70656E2073756264697220DC
:102810000053442063617264206F6B0A006F70651F
:102820006E526F6F74206661696C65640A00766F22
:102830006C756D652E696E6974206661696C65647E
:102840000A004E6F20534420636172640A002E0A0E
:10285000006F70656E206661696C65642C20466946
:102860006C653A200046696C652073656C6563741D
:1028700065640A002053697A653A200046696C65F0
:10288000206F70656E65643A2000454E44205355B4
:1028900042524F5554494E450A002220706F730032
:1028A0002220706172656E743A2200535542524F75
:1028B0005554494E452043414C4C20746172676524
:1028C000743A220053756263616C6C204F766572B6
:1028D000666C6F77004578636565646564206D613B
:1028E0007820535542524F5554494E4520646570E7
:1028F00074683A00667265736800646F696E670099
:102900002066696C653A20004E6F77200057726927
:1029100074696E6720746F2066696C653A20006D7B
:1029200061726C696E66772E6F726700322E302E80
:10293000392E332D6B616431001FFFFFFFFFFFFF56
:10294000600000000001FF400000000000FF800068
:10295000000000007F83CF00000C303F87FF800025
:102960000C301F867980000C000F8C30C7838C30B0
:10297000E78C30CFC7CC31F38C30DCECEC33B98C46
:1029800030D86C6C33198C30D06C0C33198C30D837
:102990006C0C33198C30DC6C0E3B198C30CF7C07FF
:1029A0009F198C30C77C038F194000000000000283
:1029B000600000000000061FFFFFFFFFFFF870012E
:1029C0002C0190012701B0012201C0011D01F0017D
:1029D00018011002130130020E0160020901900279
:1029E0000401C002FF000003FA004003F500800369
:1029F000F000D003EB002004E6007004E100E004E6
:102A0000DC004005D700C005D2004006CD00D0064E
:102A1000C8008007C3003008BE00F008B900C00934
:102A2000B400B00AAF00B00BAA00D00CA500000E95
:102A3000A000500F9B00C01096005012910000148F
:102A40008C00C0158700B0178200B0197D00D01B24
:102A50007800001E730040206E0090226900F02470
:102A6000640040275F0090295A00E02B5500102E8B
:102A7000500020304B0010324600E03341009035CA
:102A80003C001037370070383200A0392D00B03AC2
:102A90002800A03B2300603C1E00103D1900903D23
:102AA0001400103E0F00703E0A00C03E0500003FBB
:102AB0000000403FFBFF803FF6FFC03FF1FF2020BA
:102AC000506C616E6E6572427566666572427974AD
:102AD00065733A20002046726565204D656D6F7202
:102AE000793A200020436F6D70696C65643A204428
:102AF000656320323720323032310A00204C617356
:102B00007420557064617465643A20323032312D1E
:102B100030392D3033207C20417574686F723A2033
:102B2000286B61642C20416E796375626963204D66
:102B3000656761205A65726F20322E302041424C09
:102B400020323456290A004D61726C696E20322E93
:102B5000302E392E332D6B6164310A0020536F669D
:102B600074776172652052657365740A002057613D
:102B7000746368646F672052657365740A0020424D
:102B8000726F776E206F75742052657365740A00DA
:102B90002045787465726E616C2052657365740AA5
:102BA00000506F77657255700A0073746172740A11
:102BB000004732385859004D31303031006572725B
:102BC0006F722077726974696E6720746F2066690E
:102BD0006C650A00446F6E6520736176696E6720CC
:102BE00066696C652E0A004D323900456E64737457
:102BF0006F707300255320256320256320256320F3
:102C0000256300205A3A0020593A0020583A0065BE
:102C10006E6473746F7073206869743A20000000EA
:102C200000010200090A0000000004030807000078
:102C30000000000000000000000000000000004D47
:102C40006F76652025736D6D004D6F766520302E93
:102C5000316D6D004D6F766520316D6D004D6F7675
:102C6000652031306D6D004D6F7665204178697358
:102C7000004D6F7665204578747275646572004DFD
:102C80006F7665205A004D6F76652059004D6F763E
:102C9000652058005072696E742066726F6D204D09
:102CA0006564696100FFFFFF205A3A200020593A0D
:102CB000200042656420583A20004D656761205A23
:102CC00065726F20322E302052656164792E00507B
:102CD00072696E74696E672E2E2E005072696E7462
:102CE0002050617573656400204500205A0020590A
:102CF0000020204D393220580053746570732070C5
:102D0000657220756E6974003B2000220A00556EC2
:102D10006B6E6F776E20636F6D6D616E643A20220B
:102D2000006F6B00DB0FC93F45BCDA3F8FB3024039
:102D3000FCF0274056946140FE4B9B4084A5D84050
:102D4000E0231841346A5641E859974164DBD54184
:102D50006E271742B4B75542CE1A9742C8AED54235
:102D6000B5885A43D40684BFA65FA7BF7443E0BFAB
:102D700010B11AC01C2C58C0E8F697C0B849D6C08C
:102D80004E4E17C124D355C1802497C1A0B5D5C1DB
:102D9000121A17C244AE55C2781797C26CACD5C28E
:102DA00067885AC320746F6F206C6F6E67206578D8
:102DB00074727573696F6E2070726576656E746576
:102DC000640A0020636F6C6420657874727573699F
:102DD0006F6E2070726576656E7465640A006F6B45
:102DE0000A00526573656E643A200020453A00205F
:102DF0005A3A0020593A00583A00000022002500B3
:102E000028002B0000002100240027002A000202D5
:102E10000202020202020404040404040404030380
:102E20000303030303030101010101010101010285
:102E30000408102040800102040810204080010294
:102E400004081020408080402010080402014572D0
:102E5000726F722077726974696E6720746F204593
:102E60004550524F4D210A009FDB8CE211241FBEBA
:102E7000CFEFD0E4DEBFCDBF84B78093991514BEE9
:102E80000FB6F894A89580916000886180936000E7
:102E9000109260000FBE12E0A0E0B1E0E6E4F1EEB7
:102EA00001E00BBF02C007900D92A239B107D9F71C
:102EB00025E1A2E9B2E001C01D92A939B207E1F70C
:102EC00017E1C5E3D7E104C02197FE010E94F1EDAF
:102ED000C433D107C9F70E946EDC0C9497F00C94B0
:102EE0000000A0E1B0E0E7E7F7E10C941AEE8C01F6
:102EF000DC01ED91FC910280F381E02DBE016F5F5A
:102F00007F4F0995882309F45DC08981807C91F504
:102F10006F81637070E0762F6627770F770F888553
:102F2000B4E08B9FC0011124682B792B8985829591
:102F3000869586958370682B6F5F7F4F90E080E069
:102F40002A852370220F3B8537FB332730F9232B4B
:102F50003E813F70230F3327331F2750310904C0B0
:102F6000660F771F881F991F2A95D2F76096E4E0B5
:102F70000C9436EE803419F568856695669570E098
:102F800090E080E0CB01772766272A85622B0985B0
:102F900010E0102F0027012E000C220B330B602BAA
:102FA000712B822B932B6F5F7F4F8F4F9F4F4AE088
:102FB000660F771F881F991F4A95D1F7D7CF8BE0EF
:102FC000F801848360E070E0CB01D0CF0895FC016C
:102FD000828108954F925F926F927F928F929F921B
:102FE000AF92BF92CF92DF92EF92FF92CF93DF9397
:102FF000CDB7DEB728970FB6F894DEBF0FBECDBFB2
:1030000060913E0770913F076115710511F1809144
:103010003A0790913B07A0913C07B0913D07898307
:103020009A83AB83BC83072E000C880B990B0E94FC
:103030002CE729813A814B815C810E9443EE4B0150
:103040005C0120E030E040E251EC0E9426E787FF7F
:1030500007C081E080933201C12CD12C760113C0CE
:1030600020E030E040E251E4C501B4010E94A7EF46
:10307000181604F581E080933201C12CD12C9FE712
:10308000E92E93E4F92EC701B60128960FB6F894FD
:10309000DEBF0FBECDBFDF91CF91FF90EF90DF90ED
:1030A000CF90BF90AF909F908F907F906F905F90E8
:1030B0004F9008958091450790914607A09147074A
:1030C000B09148078D839E83AF83B887809132018A
:1030D000882391F01092960410929704109298040D
:1030E00010929904109292041092930410929404F6
:1030F0001092950410923201209196043091970419
:103100004091980450919904C501B4010E9444EE85
:103110002B013C0120E030E0A9010E94A7EFC12C67
:10312000D12C760187FD14C02D813E814F815885B9
:1031300060E070E08FE793E40E94BBEE6B017C01DE
:10314000A30192010E9426E7181614F4730162018C
:10315000C0929604D0929704E0929804F092990459
:103160002091410730914207409143075091440715
:10317000C501B4010E948BE74B015C0180928A0477
:1031800090928B04A0928C04B0928D04A7019601BA
:103190006D817E818F8198850E948BE76B017C0118
:1031A000C0928E04D0928F04E0929004F092910429
:1031B0004090920450909304609094047090950411
:1031C00029813A814B815C816091860470918704EA
:1031D00080918804909189040E9443EE20914907D0
:1031E00030914A0740914B0750914C070E948BE762
:1031F000A30192010E9443EE20ED3CEC4CE45DE320
:103200000E948BE7A30192010E9444EE9B01AC0156
:103210002093920430939304409394045093950424
:1032200089819A81AB81BC818093860490938704C5
:10323000A0938804B0938904C501B4010E9444EEB0
:10324000A70196010E9444EE6B017C0120E030E072
:103250004FE753E40E9426E7181634F4C12CD12C12
:103260008FE7E82E83E4F82E20E030E0A901C701C3
:10327000B6010E94A7EF87FF06CFEECE60913A0716
:1032800070913B0780913C0790913D070895FC01A8
:1032900090E1A5E7B4E001900D929A95E1F70895C9
:1032A000EF92FF920F931F93E0928E03F0928F03A1
:1032B0000093900310939103B62F172F022FF32E34
:1032C000242F582FB0939203109393035093940399
:1032D0006FEFFF27B01B1F09520B30F4509510956C
:1032E000B195160B560B66276093AB04A6E0BA9F08
:1032F00000929F04712DEE271A9F700DE11D5A9FB9
:10330000E00D7093A004E093A104AFE0BA9F009297
:10331000A304712DEE271A9F700DE11D5A9FE00D39
:103320007093A404E093A504AAE0BA9F0092A704B6
:10333000712DEE271A9F700DE11D5A9FE00D7093BD
:10334000A804E093A9041F910F91FF90EF900895B6
:10335000A5E0B0E0EEEAF9E10C9413EE6F367105EA
:103360008105910578F4FB01EE0FFF1FEE0FFF1FA3
:10337000E35DF74F65917591859194912596EBE00A
:103380000C942FEEF62EE72E282FEDE2F7E0002723
:10339000BB275F2D8E2D922F992341F4982F852FD7
:1033A000B85F992319F4982F8827B85F903138F4C3
:1033B00082959295582F5F70807F952BBC5F9034DB
:1033C00028F4880F991F880F991FBE5F903818F452
:1033D000880F991FB395880F991FE90FF01F54911B
:1033E00081E09927B85079F1C0F0B0FF02C0550FC5
:1033F000881FB1FF04C0550F881F550F881FB2FFEB
:1034000006C082955295152F1F70507F812BB3FFF8
:103410001AC0982F852F552716C0B195B0FF02C04E
:1034200085955795B1FF04C0859557958595579516
:10343000B2FF05C08295507F5295582B8F70B3FF15
:1034400002C0582F8827BB247727AA27B2E0F59E11
:10345000B0187109A00BB00BE59E7019A109B00B53
:10346000259FA019B109F89E7019A109B00BE89E1B
:10347000A019B109289FB019F99EA019B109E99EB8
:10348000B0195B9DA12C99244427662733278B9D77
:10349000A00C911C401F601F301F9B9D900C411D74
:1034A000601F301F579FA00C911C401F601F301FD2
:1034B000879F900C411D601F301F979F400D611D1D
:1034C000301F5A9F900C411D601F301F8A9F400D76
:1034D000611D301F9A9F600D311D5B9F400D611D66
:1034E000301F8B9F600D311D9B9F300DB1E0AA27CF
:1034F0007727BB24F49EB0187109A00BB00BE49E93
:103500007019A109B00B249FA019B109F69E70197A
:10351000A109B00BE69EA019B109269FB019F39E30
:10352000A019B109E39EB019BF187E09A20B20F0C3
:10353000B1E04B0F601F301F1124762F642F90E0F5
:10354000832F1CCFFC017081472F50E0062E02C054
:10355000559547950A94E2F740FF14C040910D0439
:1035600050E0062E02C0559547950A94E2F740FFB9
:1035700009C021E030E001C0220F6A95EAF72095EA
:103580002723208308958F929F92AF92BF92CF926C
:10359000DF92EF92FF92FC01C080D180E280F38045
:1035A00020E030E048EC52E4C701B6010E948BE70E
:1035B0004B015C0120E030E0A901C701B6010E9487
:1035C00026E720E030E040EA50E487FF04C020E036
:1035D00030E040EA50ECC501B4010E9444EE2DEC0D
:1035E0003CEC4CEC5DE30E948BE70E9423EF9B01D7
:1035F0008BE237FF05C022273327261B370B8DE2CE
:1036000080939C02C90168EE73E00E94DEEDCB015D
:10361000EAE0F0E0BF010E94DEED805D80939D0254
:10362000C90164E670E00E94DEEDCB01BF010E949B
:10363000DEED805D80939E02C901BF010E94DEED38
:103640009C01CB01BF010E94DEED805D80939F0253
:103650008EE28093A002205D2093A1028CE992E08B
:10366000FF90EF90DF90CF90BF90AF909F908F90A2
:1036700008954F925F926F927F928F929F92AF9236
:10368000BF92CF92DF92EF92FF92FC01C080D18077
:10369000E280F38020E030E04AE754E4C701B6015D
:1036A0000E948BE74B015C0120E030E040E251ECEE
:1036B000C701B6010E9426E7181654F420E030E056
:1036C00048EC52E4C701B6010E94A7EF87FD8AC00B
:1036D00020E030E0A901C701B6010E9426E787FF7C
:1036E00072C060E070E080EA90ECA50194010E9455
:1036F00044EE2DEC3CEC4CEC5DE30E948BE70E9429
:1037000023EF6B017C01F7FC63C020E137E240E06E
:1037100050E00E9476EDCA01B9012AE030E040E0B5
:1037200050E00E9476ED605D60939C02C701B60197
:1037300028EE33E040E050E00E9476ED9AE0892EDA
:10374000912CA12CB12CCA01B901A50194010E94B0
:1037500076ED605D60939D02C701B60124E630E01E
:1037600040E050E00E9476EDCA01B901A501940144
:103770000E9476ED605D60939E028EE280939F02D0
:10378000C701B601A50194010E9476ED6B01CA0143
:10379000B901A50194010E9476ED605D6093A002DD
:1037A000F0E3CF0EC092A1028CE992E0FF90EF907F
:1037B000DF90CF90BF90AF909F908F907F906F9051
:1037C0005F904F90089560E070E080EA90E48DCFC4
:1037D000F094E094D094C094C11CD11CE11CF11C65
:1037E0006DE2A2CF20E030E0A901C701B6010E943E
:1037F00026E787FF6BC060E070E080EA90ECA501EF
:1038000094010E9444EE2DEC3CEC4CEC5DE30E94F4
:103810008BE70E9423EF4B015C0120E030E0A9011F
:10382000C701B6010E9426E787FD0BC020E030E00B
:1038300040E251E4C701B6010E94A7EF60E287FDB4
:1038400013C0B7FC48C0C501B40128EE33E040E026
:1038500050E00E9476EDCA01B9012AE030E040E074
:1038600050E00E9476ED605D60939D02C501B40159
:1038700024E630E040E050E00E9476ED8AE0482EF9
:10388000512C612C712CCA01B901A30192010E9433
:1038900076ED605D60939E028EE280939F02C5018B
:1038A000B401A30192010E9476ED6B01CA01B90136
:1038B000A30192010E9476ED605D6093A00280E317
:1038C000C80EC092A1028DE992E070CF60E070E076
:1038D00080EA90E494CFB094A09490948094811C5A
:1038E000911CA11CB11C6DE2BFCF282F81E32436AF
:1038F00009F080E280939E0290E22A3040F03AE0A4
:10390000822F632F0E94B1ED0E94B1ED905D9093E4
:103910009F02822F6AE00E94B1ED905D9093A00219
:1039200085E28093A1028EE992E0089560912C01D6
:1039300070912D01072E000C880B990B0E942CE72B
:103940002AE037ED43E25CE30E948BE760936F016E
:103950007093700180937101909372010895CF93D9
:10396000DF93EC01CB01BA010E942CE723E333E3A0
:1039700043E250E40E948BE720E030E040E05FE368
:103980000E9444EE0E9428EF6883DF91CF91089552
:103990000E942CE723E333E343E250E40E948BE7E9
:1039A00020E030E040E05FE30E9444EE0E9428EF18
:1039B00024E6629FC001112481589F4F6FEF70E091
:1039C0000E94DEED862F91CF80917E07811104C089
:1039D000809132078093B20708958091DE14882386
:1039E000C1F081508093DE14E4E0F3E1882351F0CC
:1039F0008150990B2BE1289FF001299FF00D112494
:103A0000E053FC4E8BE1A9EEB2E101900D928A9554
:103A1000E1F72091DE14211105C08091E814806443
:103A20008093E81481E090E0A0E0B0E0211103C0B1
:103A300080E090E0DC018093740790937507A09379
:103A40007607B093770710926F0781E08093710734
:103A500083E080936A010895CF93DF93EC01CB015B
:103A6000BA010E942CE7688379838A839B83DF9164
:103A7000CF910895CF93DF93EC01CB01BA010E945F
:103A80002CE72DEC3CEC4CEC5DE30E948BE768836B
:103A900079838A839B83DF91CF910895CF93DF93BE
:103AA000EC01CB01BA010E942CE72AE037ED43E29A
:103AB0005CE30E948BE7688379838A839B83DF9131
:103AC000CF910895CF92DF92EF92FF92CF93DF9341
:103AD00000D000D0CDB7DEB70E942CE72AE037ED4A
:103AE00043E25CE30E948BE76B017C0120E030E065
:103AF000A9010E9426E72DEB37E346E055E387FF57
:103B000004C02DEB37E346E055EBC701B6010E9438
:103B100044EE69837A838B839C83CE010196A9DD71
:103B20000F900F900F900F90DF91CF91FF90EF903B
:103B3000DF90CF900895CF93DF93EC01CB01BA01D2
:103B40000E942CE70E9423EF79836883DF91CF9155
:103B500008958F929F92AF92BF92CF92DF92EF9291
:103B6000FF92FC01C080D180E280F38020E030E051
:103B7000A901C701B6010E9426E787FD99C06DEB38
:103B800077E386E095E3A70196010E9444EE9F77D4
:103B900020E030E048EC52E40E948BE720E030E087
:103BA00040EA50E40E9444EE2DEC3CEC4CEC5DE32A
:103BB0000E948BE70E9423EF6B017C0180E28093DF
:103BC0009B0260E2F0E1CF16F7E2DF06E104F104C8
:103BD0008CF0C701B60120E137E240E050E00E94DE
:103BE00076EDCA01B9012AE030E040E050E00E94E1
:103BF00076ED605D60939C0260E288EEC81683E01B
:103C0000D806E104F1048CF0C701B60128EE33E0D8
:103C100040E050E00E9476EDCA01B9012AE030E0B0
:103C200040E050E00E9476ED605D60939D0260E2AE
:103C3000E4E6CE16D104E104F1048CF0C701B6012C
:103C400024E630E040E050E00E9476EDCA01B90180
:103C50002AE030E040E050E00E9476ED605D609345
:103C60009E028AE0882E912CA12CB12CC701B601AE
:103C7000A50194010E9476ED6B01CA01B901A5016D
:103C800094010E9476ED605D60939F028EE28093C6
:103C9000A002F0E3CF0EC092A1028BE992E0FF9068
:103CA000EF90DF90CF90BF90AF909F908F9008954E
:103CB0006DEB77E386E095EB66CFA4E0B0E0E3E65A
:103CC000FEE10C941CEE0E942CE72DEC3CEC4CEC3D
:103CD0005DE30E948BE769837A838B839C83CE01AB
:103CE000019637DF2496E2E00C9438EECF93DF9311
:103CF000EC018D810E94B58B60E08B810E940FCD1D
:103D0000DF91CF910895CF92DF92EF92FF920F93C0
:103D10001F93CF938C01C62F69017A01E7DF0E94C0
:103D20008BCE8C2F80640E94A98B8F2D0E94A98B33
:103D30008E2D0E94A98B8D2D0E94A98B8C2D0E9407
:103D4000A98B87E8C11101C085E90E94A98BCC30FD
:103D500011F40E94AE8BC0E00E94AE8BF801868306
:103D600087FF04C0CF3F11F0CF5FF6CFCF911F91F7
:103D70000F91FF90EF90DF90CF90089561E0FC01EC
:103D800083810E940FCD8FEF0C94A98B0F931F930B
:103D9000CF938C01ABDF0E948BCEC82F882369F0B4
:103DA0008DEF0E94A98B0E948BCEC82FC801E6DF41
:103DB0008C2FCF911F910F91089582E1F801848398
:103DC000F5CFB0E0A0E0E7EEFEE10C9412EEEC01DE
:103DD0006A017B014801590120E030E0A90167E355
:103DE00092DFA501980167E1CE018DDF81111DC031
:103DF0008F81833039F089E0CC0CDD1CEE1CFF1C78
:103E00008A95D1F7A701960169E1CE017CDF11E027
:103E1000882319F010E087E08C83CE01AFDF812F7B
:103E2000CDB7DEB7ECE00C942EEE89E08C8310E089
:103E3000F4CFCF93DF93EC016EBDFA01CA019E5F10
:103E40000DB407FEFDCF20812EBD0DB407FEFDCFC2
:103E500021812EBD3296E817F90791F70DB407FEC0
:103E6000FDCF8FEF0E94A98B8FEF0E94A98B0E943C
:103E7000AE8B8E838F71853041F083E18C83CE01D0
:103E80007DDF80E0DF91CF91089581E0FBCF0F933C
:103E90001F93CF93DF93EC018B0128DF0E948BCE21
:103EA00081110BC085E18C8310E0CE0167DF812F8B
:103EB000DF91CF911F910F910895A8016CEFCE0172
:103EC000B8DF182F882371F3F0CF0F931F93CF9390
:103ED000DF93EC0189018F81833039F089E0440F51
:103EE000551F661F771F8A95D1F79A01AB0168E1CC
:103EF000CE0109DF811127C0A8016EEFCE0199DF45
:103F0000182F8823A9F00E948BCE182F8823C1F088
:103F100020E030E0A9016DE0CE01F5DE882321F03C
:103F200086E18C8310E004C00E94AE8B8111F8CF33
:103F3000CE0124DF812FDF91CF911F910F91089542
:103F400087E18C83F5CF86E0ECCF1F93CF93DF938F
:103F5000EC01CCDE20E030E0A9016CE0CE01D3DE44
:103F600011E0882319F010E083E08C83CE0106DF96
:103F7000812FDF91CF911F9108951F93CF93DF93EE
:103F8000EC018F81833039F089E0440F551F661FA3
:103F9000771F8A95D1F79A01AB0162E1CE01B3DEBA
:103FA00011E0882319F010E085E08C83CE01E6DE75
:103FB000812FDF91CF911F9108958F929F92AF92A1
:103FC000BF92EF92FF920F931F93CF93DF938C01D9
:103FD000EB017A010E94F7CD4B015C012CE2820ECD
:103FE00021E0921EA11CB11C0E94AE8BF8018683B9
:103FF0008F3F69F40E94F7CD681979098A099B09F6
:1040000097FDF2CF81E1F8018483C0E021C08E3FAB
:1040100069F5F1E0EF1AF1088FEF8EBDFE012FEF89
:104020000DB407FEFDCF8EB581932EBDCF018C1B45
:104030009D0B8E159F05A0F30DB407FEFDCF8EB529
:10404000CE0DDF1D88830E94AE8B0E94AE8BC1E037
:10405000C80194DE8C2FDF91CF911F910F91FF90BB
:10406000EF90BF90AF909F908F9008958FE0CBCF4F
:104070000F931F93CF93DF93EC018B0137DE40E06A
:1040800052E0B801CE0199DFDF91CF911F910F91DE
:1040900008950F931F93CF93DF93EC0189018F81D4
:1040A000833039F089E0440F551F661F771F8A95CA
:1040B000D1F79A01AB0161E1CE0125DE882351F0F1
:1040C00084E08C83CE015ADE80E0DF91CF911F9196
:1040D0000F91089540E052E0B801CE016EDFF5CFB8
:1040E000B0E0A0E0E6E7F0E20C9412EEEC01162F4F
:1040F0001F821C824B830E94F7CD6B017C0120ED57
:10410000C20E27E0D21EE11CF11CA89561E08B8154
:104110000E940FCD8B810E94CEB2249A2C9A279AAE
:104120002698259A81E00E94B58B85E08D830E94B8
:10413000B58B0AE08FEF0E94A98B0150D9F7A895A3
:1041400020E030E0A90160E0CE01DDDD8E8381302A
:1041500079F00E94F7CD6C197D098E099F0997FDB2
:10416000EFCF81E08C83CE0109DE1A8280E065C04A
:10417000A8952AEA31E040E050E068E0CE01C3DDD6
:10418000853031F581E08F83A8958F81812C912C2A
:104190005401823029F4812C912CA12C80E4B82E7A
:1041A00020E030E0A90167E3CE01ADDDA501940177
:1041B00069E2CE01A8DD8E838823F1F00E94F7CD5D
:1041C0006C197D098E099F0997FDEACF8AE0CACF55
:1041D00004E00E94AE8B8E830150D9F78A3A11F425
:1041E00082E0D1CF0E94F7CD6C197D098E099F091D
:1041F00097FDBFCF82E0B6CF8F818230B9F420E047
:1042000030E0A9016AE3CE017EDD882311F088E069
:10421000A9CF0E94AE8B807C803C11F483E08F8319
:104220000E94AE8B0E94AE8B0E94AE8BCE01A6DDAB
:1042300081E08A83173030F41D83CDB7DEB7ECE020
:104240000C942EEE88E18C8391CF0F931F93CF9324
:10425000DF93EC018B0120E030E0A90169E053DD40
:10426000882351F080E18C83CE0188DD80E0DF91EE
:10427000CF911F910F91089540E150E0B801CE0118
:104280009CDEF5CFCF93C82FCB010E94488189E6F1
:1042900096E00E9448818AE596E0CC2311F08FE5F4
:1042A00096E00E9448818AE00E942781CF9108957C
:1042B000EF92FF920F931F93CF937B018A01C2E489
:1042C0008F3F09F0C4E580E20E9427818C2F0E9475
:1042D00027818AE30E942781F701608171818281B1
:1042E000938142E00E94EDB282E193E10E94488115
:1042F000F801608171818281938142E00E94EDB278
:1043000062E070E080E090E00E946BCDCF911F9161
:104310000F91FF90EF9008950C9403CE40918C0381
:1043200021E042276CE070E00C94A2B240918C0333
:1043300021E0422764E070E00C94A2B240918C032B
:1043400021E0422761E070E00C94A2B240918C031E
:1043500021E0422761E070E00C94A2B240918C030E
:1043600021E0422768E070E00C94A2B240918C03F7
:1043700021E042276CE070E00C94A2B241E061E0E1
:1043800070E00C94A2B240918C0321E042270C947F
:10439000A2B26CE070E00C949ECD61E070E00C94F1
:1043A0009ECD6CE070E00C949ECD64E070E00C94C7
:1043B0009ECD9091B30281E089270C94377761E01C
:1043C00082E397E00C94C37720E030E0A901BC01C0
:1043D00085E791E00C94BCC380E090E0A0E8B0E4F5
:1043E00080937D0190937E01A0937F01B093800123
:1043F0008AE192E0E9DF80E090E0A0EFB1E4809311
:10440000750190937601A0937701B0937801809322
:10441000790190937A01A0937B01B0937C01E091A4
:10442000EA03EE0FFF0BE650FE4F8081918183304F
:10443000910539F184309105C9F1029761F480E06A
:1044400090E0A3E4B3E48093750190937601A09388
:104450007701B093780182E092E0B6DF10927D019F
:1044600010927E0110927F01109280018AE192E009
:10447000ABDF8091EA038F5F8430ECF48093EA0332
:10448000089580E090E0A3E4B3E4809375019093F5
:104490007601A0937701B09378018093790190938E
:1044A0007A01A0937B01B0937C01D5CF80E090E0AE
:1044B000A3E4B3E4F2CF1092EA030895B0E0A0E0E1
:1044C000E4E6F2E20C941CEE20E24F8158856E8106
:1044D0008D810E94C2C8E2E00C9438EE80913207D0
:1044E000909133070C9438CE609132078FEF0C9483
:1044F00042CE80913207682F0C9442CE6FEF8091AC
:1045000032070C9442CE65E072E582E00C94D0CA8A
:1045100069E072E581E00C94D0CA6DE072E580E05C
:104520000C94D0CA61E172E583E00C94D0CA109279
:104530006F070C94FCDA4FE350E06AE874E081EF17
:1045400096E00C947DF080916A1390916B13891B17
:104550008F7011F40C94177981E0089580916A01AD
:10456000882341F06091E2037091E30341E081E030
:104570000C9462C80895CF93DF93EC010E9481D51B
:104580001B82DF91CF910895CF93DF93EC01462FEB
:1045900041706C857D858E859F850E9492D288238F
:1045A00051F0888920E2829FC001112480569F4EDD
:1045B000DF91CF91089590E080E0FACFCF93DF9321
:1045C000EB01FC012381211104C080E0DF91CF9138
:1045D00008952250223028F48FE28883198281E0E6
:1045E000F5CF60E0D1DF009781F3DC0160E080E08F
:1045F0009EE22D91203299F0883031F49E01260FF1
:10460000311DF90190836F5F9E01260F311DAD01B1
:1046100041505109FA014081F90140836F5F8F5F7A
:104620008B3039F7FE01E60FF11D1082D8CFACE0D8
:10463000B0E0EDE1F3E20C940DEE5C01DC01599683
:104640008D909C90F40181859285A385B4859C0111
:10465000AD012F5F3F4F4F4F5F4F29873A874B8701
:104660005C87D50114964D905D906D907C90179766
:10467000411451046104710409F459C0BFEF4B1A8D
:104680005B0A6B0A7B0A312C730162011D821E8258
:104690001F821886F40181859285A385B4852D81BA
:1046A0003E814F815885281739074A075B0708F074
:1046B00056C089859A85AB85BC858C159D05AE0550
:1046C000BF0550F482E0C82ED12CE12CF12C92E0F1
:1046D000492E512C612C712C9E012F5F3F4FB70149
:1046E000A601C4010E949CD48823C9F189819A81C2
:1046F000AB81BC81892B8A2B8B2B01F126013701E1
:104700009FEF491A590A690A790A2D813E814F8122
:1047100058852F5F3F4F4F4F5F4F2D833E834F8311
:1047200058873FEFC31AD30AE30AF30AB3CF408096
:1047300051806280738033243394A6CFC414D5048F
:10474000E604F70411F70FEF1FEF2FEF3FE0B7017B
:10475000A601C4010E9422D4782E811106C0712CBA
:10476000872D2C96E1E10C9429EEF50144815581C9
:1047700066817781411551056105710539F0970111
:104780008601C4010E9422D4882349F3D5011496DE
:10479000CD92DD92ED92FC921797332051F0D70124
:1047A000C6010196A11DB11DF40180839183A283EE
:1047B000B383F50185899689A789B08D892B8A2BCA
:1047C0008B2B71F6C58AD68AE78AF08E8181806844
:1047D0008183C6CF40E050E0BA010C94CAD54F9215
:1047E0005F926F927F92AF92BF92CF92DF92EF92E1
:1047F000FF920F931F93CF93DF931F92CDB7DEB736
:104800008C017B015A01C22EDB0159968D919C913E
:10481000F801928F818FCB01DDDF712CF70180854C
:104820009185A285B38541895289638974898417EA
:104830009507A607B70708F052C055E0B695A795AB
:10484000979587955A95D1F7F82FFF70DF2ED701EE
:1048500013968C91823010F480E0DAC041E050E091
:10486000BE016F5F7F4FC7010E94C5D60197A1F7B8
:10487000F70180859185A285B3854F96A11DB11D55
:1048800080879187A287B387F0E2DF9EB001112471
:1048900060567F4E61157105F9F2DB018C9188231A
:1048A00041F0853E09F04BC0772029F077247394BE
:1048B000B5CF71100EC08091A0129091A112A0915D
:1048C000A212B091A312F80184879587A687B787B3
:1048D000D08ADB018C918111E9CF772473948C2DE0
:1048E0008274823409F0B8CF772009F4A1C0F801AE
:1048F000D08861E0C80148DE009709F4ADCF20E21E
:10490000DC011D922A95E9F72BE0F501DC0101900D
:104910000D922A95E1F721E238E2FC01318B208BE0
:1049200040E058E057874687338B228B318F208FAA
:10493000578B468B0E9449D2811109C08DCF4BE025
:1049400050E0C5010E942DF0892B09F067CFF0E2FD
:10495000DF9ED00111249D0120563F4EF901838531
:10496000817121F08C2D827109F000C1F801818DD7
:10497000928D4091A0125091A1126091A21270915B
:10498000A3124487558766877787D08AFD01E05652
:10499000FF4E44885588712C612C320155244424E3
:1049A000D80155964D925D926D927C925897428DAA
:1049B000538D70E060E04429552966297729559682
:1049C0004D935D936D937C935897D9011B962C91D1
:1049D000287109F0BDC0848D958DA68DB78DF80125
:1049E000818B928BA38BB48B81E083838C2D8F7012
:1049F000F80181831482158216821782108611862F
:104A00001286138681E0C4FE03C0C8010E944FD6FF
:104A10000F90DF91CF911F910F91FF90EF90DF905A
:104A2000CF90BF90AF907F906F905F904F90089520
:104A3000D70113968C911397823009F40DCF5196BC
:104A40008D919D910D90BC91A02D803E9F4FAF41C7
:104A5000B10508F001CFC701EADD882309F4FCCED7
:104A60000E9449D2882309F4F7CED7015996ED91D7
:104A7000FC915A9714964D905D906D907C9017978D
:104A8000B2E04B1A510861087108858504C0440CD6
:104A9000551C661C771C8A95D2F786859785A08958
:104AA000B189480E591E6A1E7B1E81E08093A412B4
:104AB0004092A0125092A1126092A2127092A31280
:104AC000E0EAF0E180E092E0DF019C011D922150DC
:104AD0003040E1F7DD24D394D7015996ED91FC9154
:104AE0008481D816C0F48091A5129091A612DC01A1
:104AF000ED91FC910288F389E02D20EA30E1B301C9
:104B0000A2014D0D511D611D711D0995882309F4E8
:104B1000A3CED394E1CF258580E092E0A0E0B0E081
:104B200004C0880F991FAA1FBB1F2A95D2F7F7014F
:104B30004189528963897489840F951FA61FB71F05
:104B4000818B928BA38BB48B80EA90E1D12CD7CE52
:104B5000203161F498012F5E3F4F0E9418D58823C1
:104B600029F084E0D80113968C9340CFD801139696
:104B70001C9272CEFC0123812111FDCC0895A1E489
:104B8000B0E0E5ECF5E20C940CEE4C015B017A012F
:104B9000222E19821C821C8E1F8E6115710569F4EC
:104BA00010E0CE014C96E6DFCE010196E3DF812FC7
:104BB000CF5BDF4FE2E10C9428EEFC018381811191
:104BC000EFCFFA0180818F3251F18B01CE01019636
:104BD0006C012C0180E2382E360122963FAE2297DE
:104BE00021963FAE21973FAE3EAE3DAE3CAE3BAED2
:104BF0003AAE39AE38AE3FAA970190E047E0D9010E
:104C00008D91882309F447C08F3209F444C08E3255
:104C100009F54A3029F298E04AE09D01F0CFFB0106
:104C2000838182508230A0F0618D728DCE014C96CE
:104C30000E94ADDA882309F4B3CF8E01045E1F4FC2
:104C4000C7017C010196F70120812F32D1F3BECF3D
:104C50008B01F6CFEEE1F3E12491222321F031968E
:104C60008213FACF9DCF491708F49ACF813208F406
:104C700097CF8F3709F494CF3FE9380F3A3108F4D2
:104C800020EEE7E3F0E0EC0FFD1FE90FF11D820FCE
:104C900080839F5FC2CF8FA9803209F481CF7901D1
:104CA000F90180812F5F3F4F8F32C9F38823C1F014
:104CB00021E0AE01495C5F4FB801C60190DD882359
:104CC00009F46ECF0A151B0511F0C80154DCCE01A2
:104CD0004C964C145D0409F0C30186016C017DCF34
:104CE000222DAE01495C5F4FB801C40178DD182F59
:104CF00058CFEF92FF921F93CF93DF93CDB7DEB7DC
:104D000028970FB6F894DEBF0FBECDBF182F85EBE6
:104D1000E82E82E1F82EF70160857185072E000CE0
:104D2000880B990B0E942CE76D837E838F83988775
:104D3000F70184819581A681B78189839A83AB83AA
:104D4000BC83AE014B5F5F4FBE016F5F7F4F80E062
:104D5000AFDA96E3E92E97E0F92EF70160857185C9
:104D6000072E000C880B990B0E942CE76D837E8325
:104D70008F839887F70184819581A681B781898384
:104D80009A83AB83BC83AE014B5F5F4FBE016F5F05
:104D90007F4F8FEF8DDA87E11802F0011124EB5479
:104DA000FD4E628570E08AE193E10E94C98AF701B5
:104DB000628570E085E193E10E94C98A28960FB66A
:104DC000F894DEBF0FBECDBFDF91CF911F91FF9052
:104DD000EF9008950F930FB70F9300916E000B7F24
:104DE00000936E0078940F930BB70F930CB70F924C
:104DF0001F922F933F934F935F936F937F938F9364
:104E00009F93AF93BF93EF93FF9311240E94596335
:104E1000FF91EF91BF91AF919F918F917F916F9192
:104E20005F914F913F912F911F900F900CBF0F9169
:104E30000BBF0F910460F89400936E000F910FBFA9
:104E40000F911895CF93DF9310929C03C5EBD2E19D
:104E5000198618860E9403CE1A865D98C6E3D7E0AD
:104E6000198618860E949F671A865C98DF91CF91F9
:104E70000895B0E0A0E0EFE3F7E20C9412EEB0E4A6
:104E8000A0E06A2F70E0AB014B0F511D559547957F
:104E9000411111C0E0ECF9E265917491072E000C0C
:104EA000880B990B0E942CE7CDB7DEB7ECE00C9491
:104EB0002EEEB42FE8CFA41711F0B41303C0ECEB1F
:104EC000FAE2EACF9A0121503109220F331F220F53
:104ED000331FF901E254F64DE590F490F901EE53D9
:104EE000F64DC591D4918E159F051CF3A42FC817BC
:104EF000D9070CF4C6CFF901E054F64D0591149191
:104F0000F901EC53F64DC590D490BC016E197F09A0
:104F1000072E000C880B990B0E942CE74B015C01BB
:104F2000B601601B710B072E000C880B990B0E94B9
:104F30002CE79B01AC01C501B4010E948BE74B013A
:104F40005C01BE016E197F09072E000C880B990BBE
:104F50000E942CE79B01AC01C501B4010E94BBEE8D
:104F60006B017C01B801012E000C880B990B0E948B
:104F70002CE79B01AC01C701B6010E9444EE94CF1F
:104F8000EF92FF920F931F93CF93DF93C82F7B0174
:104F90008A0180913107833090F00E94B587C70164
:104FA0000E94488188E792E10E944881CF3F79F5CD
:104FB00084E792E10E9448818AE00E94278142DFD3
:104FC000A8958091850481113EC081E0809385047D
:104FD00082E08093310736DFD5E1D150149A49F150
:104FE00069E170E080E090E00E946BCDA895149894
:104FF00068E270E080E090E00E946BCDA89568E2E6
:1050000070E080E090E00E946BCDA895E6CFC7FDF0
:10501000D3CF82E792E10E9448816C2F0C2E000CC6
:10502000770B880B990B0E94A3B08AE00E9427811E
:10503000C3CF6BE672E1CF3F11F06FE672E140E063
:10504000C8010E94D78ACDB7DEB7E6E00C9434EEF3
:10505000B0E0A0E0EEE2F8E20C940EEEEC016B01A1
:105060004A01B22EFA014080518062807380A30110
:1050700092016D817E818F8198850E9426E7882329
:10508000A1F04D825E826F827886AA24A39420E0EC
:1050900030E0A901F40160817181828193810E94D5
:1050A000A7EF18160CF0A12CAC828C818230A1F0F5
:1050B000833009F44FC08130D1F52D813E814F817D
:1050C0005885F60160817181828193810E9426E773
:1050D00087FD2DC082E08C83B7010F2C000C880B5C
:1050E000990B0E942CE79B01AC016D817E818F8121
:1050F00098850E9443EE9B01AC01F60160817181AD
:10510000828193810E94A7EF87FD16C00E94F7CD90
:105110006B017C019801A8EEB3E00E94A2EDC60EDF
:10512000D71EE81EF91EC882D982EA82FB82CDB75B
:10513000DEB7E0E10C942AEE0E94F7CD08811981D8
:105140002A813B81601B710B820B930B97FDEFCF84
:1051500083E08C8342EF52E162E073E18B2D10DF3C
:10516000E6CF46E952E163EA72E10ACFCF93DF93DB
:10517000A8958091B7129091B8120E941BB26093CB
:10518000B9127093BA128093BB129093BC128091A3
:105190003807909139076DDE60933A0770933B07AB
:1051A00080933C0790933D07C091B712D091B812FD
:1051B0008091630190916401C817D90714F480E0CD
:1051C000D0DF8091BD129091BE12181619066CF4B2
:1051D00080916101909162018C179D0734F443ED39
:1051E00052E160EE72E180E0CBDE20913807309131
:1051F00039078091E5069091E6062817390714F4DF
:105200008FEFAFDF80913E0790913F071816190688
:105210008CF4209138073091390780915F0190918B
:1052200060018217930734F443ED52E160EE72E1BE
:105230008FEFA6DEDF91CF910895A4E0B0E0E3E226
:10524000F9E20C9412EE80913107811106C0A89505
:105250002496ECE00C942EEE28C180919A048111E2
:10526000F7CF81E080939A0480919D03811107C05C
:1052700010929A042496ECE00C942EEE16C176DF80
:1052800010929D030E94F7CD4B015C010E94BEB0BD
:105290006B017C016091670170916801072E000C21
:1052A000880B990B0E942CE79B01AC01C701B6014A
:1052B0000E94A7EF18160CF4E7C06091BD12709120
:1052C000BE12072E000C880B990B0E942CE76983F5
:1052D0007A838B839C8334E0E32EF12C08E210E088
:1052E00020E0AE014F5F5F4F69EB72E18FE193E128
:1052F000AFDEC090B912D090BA12E090BB12F0901D
:10530000BC126091650170916601072E000C880B3C
:10531000990B0E942CE79B01AC01C701B6010E94CA
:10532000A7EF1816CCF46091670170916801072E01
:10533000000C880B990B0E942CE79B01AC01C70164
:10534000B6010E9426E787FF07C00E94C7B00E94EF
:1053500023EF7595679501C060E06093BF1280915F
:10536000B1129091B212A091B312B091B412009701
:10537000A105B105C1F0A5019401281B390B4A0B09
:105380005B0BDA01C901B7FD0EC00E94BEB00E94DE
:1053900023EF2091AF123091B012621773070CF413
:1053A0007DC00E9403CE0E943E1920E030E04AEF0B
:1053B00052E40E94A7EF18160CF463C08091980382
:1053C00090919903A0919A03B0919B030097A10536
:1053D000B105A1F0881A990AAA0ABB0AB7FC0EC047
:1053E0000E943E190E9423EF20919603309197036B
:1053F000621773070CF44BC00E949F6760913E07D1
:1054000070913F07072E000C880B990B0E942CE728
:1054100069837A838B839C8392E0E92EF12C04E1EB
:1054200010E02FEFAE014F5F5F4F6AE377E088E255
:1054300093E10EDE80903A0790903B07A0903C07E6
:10544000B0903D0720E030E040EA50E4C501B401EF
:105450000E94A7EF87FD11C020E030E04AEF52E440
:10546000C501B4010E9426E718163CF00E94EA1715
:105470000E9423EF7595679501C060E06093400737
:10548000F7CE8FEF6EDE9ACF80E06BDE16CF45EB66
:1054900052E164EC72E18FEF73DDB0CF45EB52E186
:1054A00064EC72E180E06CDD7ECFCF92DF92EF9210
:1054B000FF92CF93DF93EC01C880D980EA80FB8014
:1054C00081E692E10E944881C701B6010E9484737F
:1054D000CC80DD80EE80FF8083EF9DE20E944881DA
:1054E000C701B6010E948473C884D984EA84FB840E
:1054F0008FEE9DE20E944881C701B6010E9484732D
:105500008AE00E942781DF91CF91FF90EF90DF909A
:10551000CF900895BC0120916604309167044091BA
:105520006604509167042417350731F481E026178B
:10553000370709F080E008959A01F1CF0F930FB774
:105540000F9300916E000F930B7F00936E000091FC
:105550006F000D7F00936F000F930BB70F930CB785
:105560000F921F922F933F934F935F936F937F936D
:105570008F939F93AF93BF93EF93FF931124E1D445
:10558000FF91EF91BF91AF919F918F917F916F911B
:105590005F914F913F912F911F900F900CBF0F91F2
:1055A0000BBF0F910260F89400936F000F9100936E
:1055B0006E000F910FBF0F91189500C000C0809131
:1055C000E90680FF1FC0459A8FEF80931F048091EA
:1055D000E90681FF1AC0479A8FEF809320048091DB
:1055E000E90682FF15C02A988FEF809321048091ED
:1055F000E90683FF10C028988FEF8093220400C033
:1056000000C00895459881E0E0CF479881E0E5CF5C
:105610002A9A81E0EACF289A81E0EFCF80918D032A
:10562000982F977F90938D03982F937081E011F0BE
:1056300080E008955E9A08955E9880918D03886059
:1056400080938D030895E82FF0E021E030E0082EEC
:1056500002C0220F331F0A94E2F7209530959091F3
:105660008D03922390938D03EA50FE4F2081922365
:1056700021E019F020E0822F0895813079F038F090
:105680008230C9F7159A909182079B7F04C05E9A79
:10569000909182079E7F90938207EDCF5E9A9091C2
:1056A00082079D7FF8CF80E0CEDF81E0CCDF82E013
:1056B000CADFB4CF813079F070F0823071F021E030
:1056C00030E001C0220F8A95EAF780918D03822B8A
:1056D00080938D0308955E98F2CF1598F0CFB0E0D7
:1056E000A0E0E5E7FBE20C9414EEC4E7DDE00AE994
:1056F00017E084E8A82E8DE0B82EC12CD12C7601BD
:10570000C39469917991899199910E942AE7288996
:1057100039894A895B890E948BE70E9428EFF8014A
:1057200061937193819391938F01C616D706E80612
:10573000F90610F46B017C01AC16BD0611F76FEF92
:105740007FEFCB01A70196010E9454ED2093AA0799
:105750003093AB074093AC075093AD07CDB7DEB79E
:10576000EAE00C9430EE0F931F93CF93DF9308E899
:105770001DE0C3EBD7E0F8012191319141915191A6
:105780008F0160E070E080E89FE30E94BBEE6993C8
:10579000799389939993F7E0C33CDF0761F70E94FF
:1057A000DFC39DDFDF91CF911F910F910895DBCF74
:1057B000DACFD9CFD8CF90916A1380916B13981319
:1057C00006C08091BC0D9091BD0D892B21F080E029
:1057D0000E94C68BF0CF089590916A1380916B134D
:1057E000981307C08091BC0D9091BD0D892B09F4D1
:1057F0005ACF80E00E94C68BEFCFCF92DF92EF921C
:10580000FF92CF93DF932091B302222319F1EC0191
:1058100008960E94E8746B017C0120E030E0A90149
:105820000E9426E720E030E0A901882349F0CE015C
:105830000E946075A70196010E948BE79B01AC0155
:10584000688579858A859B850E9443EE688779877C
:105850008A879B87DF91CF91FF90EF90DF90CF9069
:105860000895CF92DF92EF92FF92CF93DF93209132
:10587000B302222319F1EC0108960E94E8746B012F
:105880007C0120E030E0A9010E9426E720E030E022
:10589000A901882349F0CE010E946075A7019601F5
:1058A0000E948BE79B01AC01688579858A859B8581
:1058B0000E9444EE688779878A879B87DF91CF9122
:1058C000FF90EF90DF90CF900895AEE1B0E0EBE66F
:1058D000FCE20C940EEE9E8F8D8F5B018A01FC0121
:1058E000EA5BFF4F2081318142815381298B3A8BC2
:1058F0004B8B5C8BCA01B9010E942AE76B017C01CA
:10590000D5012D913D914D915C910E948BE70E94B4
:10591000A8EE2B013C01F8012081318142815381A5
:10592000C701B6010E948BE70E94A8EE4B015C0103
:10593000C301B2010E9428EF6D8B7E8B8F8B988FF5
:10594000683771058105910540F428E730E040E0B3
:1059500050E02D8B3E8B4F8B588FC501B4010E94B8
:1059600028EF698F7A8F8B8F9C8F6837710581053F
:10597000910540F488E790E0A0E0B0E0898F9A8F2D
:10598000AB8FBC8FED8DFE8DEE5AFF4F20813181A4
:105990004281538129873A874B875C87CA01B901C5
:1059A0000E942CE72B013C016D897E898F89988D9F
:1059B0000E942AE76D837E838F83988720E030E002
:1059C000A901C301B2010E9426E7882309F4BBC1E3
:1059D000A7019601C701B6010E948BE74B015C014C
:1059E0002D813E814F815885CA01B9010E948BE704
:1059F0009B01AC01C501B4010E9443EE4B015C0167
:105A0000A3019201C301B2010E9444EE9B01AC01CB
:105A1000C501B4010E94BBEE0E94A8EE0E9428EFCF
:105A200069837A838B839C8369857A858B859C8542
:105A300090958095709561957F4F8F4F9F4F0E94F5
:105A40002CE74B015C01698D7A8D8B8D9C8D0E94BA
:105A50002AE769877A878B879C8720E030E0A90155
:105A6000C501B4010E9426E7882309F470C1298585
:105A70003A854B855C85CA01B9010E948BE76D8729
:105A80007E878F87988BA7019601C701B6010E9478
:105A90008BE79B01AC016D857E858F8598890E947F
:105AA00043EE6B017C01A5019401C501B4010E9484
:105AB00044EE9B01AC01C701B6010E94BBEE0E94FF
:105AC00054EFAD8DBE8D95962D913D914D915C918C
:105AD00098972D873E874F87588B69017A012981D6
:105AE0003A814B815C81C21AD30AE40AF50A0E940A
:105AF00028EFC61AD70AE80AF90AF7FE8CC02D81EA
:105B00003E814F815885CA01B9010E948BE76B0124
:105B10007C0120E030E0A901C301B2010E9426E728
:105B2000882309F418C16D857E858F8598890E9428
:105B30002AE79B01AC010E9444EEA30192010E945E
:105B40008BE74B015C0129853A854B855C85CA0151
:105B5000B9010E948BE79B01AC01C501B4010E9411
:105B600044EEA70196010E9443EE4B015C0120E048
:105B700030E040E850E4C301B2010E948BE79B0192
:105B8000AC01C501B4010E94BBEE0E94A8EE4B011E
:105B90005C0120E030E0A9010E94A7EF87FF03C06D
:105BA000812C912C5401C501B4010E9428EF698316
:105BB0007A838B839C832D853E854F855889261754
:105BC00037074807590720F429833A834B835C83BE
:105BD00069817A818B819C810E942AE74B015C015B
:105BE000A3019201C301B2010E9444EE9B01AC01EA
:105BF000C501B4010E948BE7A70196010E9444EE03
:105C00000E94E0EF0E9428EF698B7A8B8B8B9C8B34
:105C1000C12CD12C760169897A898B899C892D893F
:105C20003E894F89588D621B730B840B950B0E9424
:105C30002AE7A30192010E94BBEE20E034E244EF88
:105C400059E40E948BE70E9428EF4B015C016989AF
:105C50007A898B899C89298D3A8D4B8D5C8D621B4D
:105C6000730B840B950B0E942AE7A30192010E94FB
:105C7000BBEE20E034E244EF59E40E948BE70E943F
:105C800028EF6D837E838F839887C501B4010E94BE
:105C9000A8192B013C016D817E818F8198850E941E
:105CA000A81929813A814B815C81AD8DBE8D999671
:105CB0002D933D934D935C939C9789019A010C0D14
:105CC0001D1D2E1D3F1DFD0105A716A727A730ABE3
:105CD000E65BFF4F2D893E894F89588D20833183A4
:105CE00042835383D5968D929D92AD92BC92D89764
:105CF0002D813E814F815885D9962D933D934D93AB
:105D00005C93DC973D974082518262827382349625
:105D1000608371838283938329893A894B895C8963
:105D2000D1962D933D934D935C93D4973D96298DB9
:105D30003A8D4B8D5C8D20833183428353836E96E5
:105D4000E0E10C942AEE60E070E0CB0165CE60E00B
:105D500070E0CB01B4CE60E070E0CB0116CF909143
:105D60006F0081E091FD02C080E0089590916F0086
:105D70009D7F90936F000895EFE6F0E08081826050
:105D800080830895CF93C82FEADF94E0C99F9001E4
:105D90001124F901E759FB4F2B583B4FD9014D9185
:105DA0005D916D917C91408351836283738391E017
:105DB000909368048111E0DFCF910895CF93DF9332
:105DC0008091E806811105C08091EE06882309F4D0
:105DD0004EC08091FA03329B4DC081608093FA03DC
:105DE0008091FA03339B48C082608093FA038091CC
:105DF000FA03349B43C084608093FA03C091590432
:105E0000C0FF0FC08091E90680FF0BC08091FA03AC
:105E100080FF07C08091810781608093810780E0C7
:105E2000B1DFC1FF0FC08091E90681FF0BC08091F7
:105E3000FA0381FF07C08091810782608093810708
:105E400081E0A0DFC2FF13C08091E90682FF0FC08E
:105E50008091EE06882359F08091FA0382FF07C0F3
:105E60008091810784608093810782E08BDFDF91DE
:105E7000CF9108958E7FB2CF8D7FB7CF8B7FBCCF70
:105E80006EDF1092AE071092AF071092B00710921B
:105E9000B107811171CF08950F931F9380916A13F9
:105EA00090916B13891B8F7009F449C0909167130F
:105EB000992361F0833040F48FEF890F29F08093AC
:105EC000671390E080E038C01092671380916B13E5
:105ED0002BE5829FC00111248D53984FFC01208136
:105EE00020FDEFCF4091AE075091AF076091B00712
:105EF0007091B107E95AFF4F0081118122813381EE
:105F0000401B510B620B730B4093AE075093AF07CE
:105F10006093B0077093B10720916B132F5F2F70C0
:105F20002093681330916B1320916913321304C0CE
:105F300020916813209369131F910F910895A0DF9A
:105F4000C0CFA3E1B0E0E7EAFFE20C940CEE8FEFE4
:105F50009FEF90938900809388002AE02983312C59
:105F6000212C78948091620490916304A091640440
:105F7000B0916504892B8A2B8B2B09F0C2C18091CB
:105F800068048823D1F08091660490916704109290
:105F90006804892B91F010926704109266041092A5
:105FA000590490916A1380916B13981731F0809186
:105FB0006B138F5F8F7080936B1380916604909149
:105FC0006704892B09F49DC140915E0450915F04E0
:105FD000609160047091610480915A0490915B0417
:105FE000A0915C04B0915D040091500410E030E099
:105FF00020E0841B950BA60BB70B081719072A077F
:106000003B0710F4D901C8018A8B840F951FA61F86
:10601000B71F80935E0490935F04A0936004B093D5
:106020006104E1E0C0902704D0902804E0902904A6
:10603000F0902A048091370490913804A09139049B
:10604000B0913A04C80ED91EEA1EFB1EC092370456
:10605000D0923804E0923904F0923A04F7FC33C04D
:1060600040911F04042E000C550B660B770B80919A
:10607000750490917604A0917704B0917804840F10
:10608000951FA61FB71F8093750490937604A09365
:106090007704B09378048091230490912404A09114
:1060A0002504B0912604B701A601481B590B6A0BC1
:1060B0007B0BDB01CA018093370490933804A093D3
:1060C0003904B0933A0400912B0410912C042091D0
:1060D0002D0430912E0480913B0490913C04A091BA
:1060E0003D04B0913E04080F191F2A1F3B1F009367
:1060F0003B0410933C0420933D0430933E0437FD51
:1061000033C040912004042E000C550B660B770B16
:106110008091790490917A04A0917B04B0917C04E1
:10612000840F951FA61FB71F8093790490937A045C
:10613000A0937B04B0937C04809123049091240469
:10614000A0912504B091260428013901481A590A62
:106150006A0A7B0AD301C20180933B0490933C04FA
:10616000A0933D04B0933E0440912F04509130041D
:10617000609131047091320480913F049091400409
:10618000A0914104B0914204480F591F6A1F7B1F20
:1061900040933F0450934004609341047093420441
:1061A00077FD33C080902104082C000C9908AA08C0
:1061B000BB0880917D0490917E04A0917F04B091F2
:1061C0008004880D991DAA1DBB1D80937D049093AA
:1061D0007E04A0937F04B093800480912304909167
:1061E0002404A0912504B09126043A014B01681AB9
:1061F000790A8A0A9B0AD401C30180933F049093D1
:106200004004A0934104B0934204809033049090E2
:106210003404A0903504B0903604809143049091EA
:106220004404A0914504B0914604880D991DAA1D0F
:10623000BB1D8093430490934404A0934504B09302
:106240004604B7FD33C040902204042C000C5508CE
:10625000660877088090810490908204A09083045F
:10626000B0908404840C951CA61CB71C80928104F9
:1062700090928204A0928304B092840480902304BC
:1062800090902404A0902504B09026042C013D0198
:10629000481859086A087B08530142018092430458
:1062A00090924404A0924504B0924604E11104C0C7
:1062B000E0918400F0918500F7FE5F9A37FF469ADF
:1062C00077FF2B9AB7FF299AE0918400F09185001F
:1062D000E0918400F0918500F7FE5F9837FF4698C3
:1062E00077FF2B98B7FF29985A88552021F0809185
:1062F0008400909185002A8921502A8BE0E02111A9
:1063000091CE8091620490916304A0916404B09155
:106310006504892B8A2B8B2B09F0B0C6409066044C
:10632000509067045B8A4A8A4114510409F402C7F9
:1063300080915E0490915F04A0916004B09161042B
:1063400040915A0450915B0460915C0470915D042B
:1063500084179507A607B70708F449C01092670489
:10636000109266041092590490916A1380916B13F5
:10637000981709F4DFC680916B138F5F8F7080933D
:106380006B13A0EDCA2EA7E0DA2EE12CF12C809140
:10639000660490916704892B09F068C67DDD9093AF
:1063A000670480936604892B09F460C640906604F4
:1063B000509067045B8A4A8AD2018C9183FF08C59A
:1063C000C20145960E944719109267041092660414
:1063D0001092590490916A1380916B139817F1F2FF
:1063E00080916B138F5F8F7080936B13D7CF409129
:1063F0005504509156046091570470915804481701
:1064000059076A077B0708F40FC240915104509165
:1064100052046091530470915404EA89FB8985A960
:1064200096A9A7A9B0AD481759076A077B0708F0D6
:10643000D0C1411551056105710509F066C0809014
:10644000920390909303A0909403B090950381E4FD
:1064500092E1A1E0FC010591159125913491081577
:1064600019052A053B0558F4B694A7949794879488
:10647000AA0F0496EDE5F2E1E817F90759F7A093A2
:106480005004F0E28F169104A104B10428F4E0E274
:106490008E2E912CA12CB12C20E2821A9108A108F9
:1064A000B108811438E09306A104B10408F49AC13C
:1064B000A4E09A9EC00111248F5B914FFC0132969B
:1064C00025913491B82DEE27B39F8001B29F010D25
:1064D0001E1F06940E1F1E1F112430E020E0FC0139
:1064E000C590D490F12CE12CC01AD10AE20AF30A2B
:1064F0004C0D5D1D6E1D7F1D409351045093520441
:10650000609353047093540442CF10E00A81942F97
:10651000852E862FBC81AD81FE81EF81388529854E
:106520004B80E0918E03E99FA12DFF2730918F03CF
:10653000399FA00DF11D10909003199EF00DE89D5C
:10654000A00DF11D389DF00DE89FF00D4A2EBF2FD4
:106550004A9EE12D332722274F9EE00D311D211F3A
:10656000BA9FE00D311D211FBF9F300D211D432E0D
:10657000B22F4A9E012D332722274F9E000D311D39
:10658000211FBA9F000D311D211FBF9F300D211DFE
:10659000432EB22FEE279091920380909303809127
:1065A00094030090AB04012A09F483C03091A7043E
:1065B000349DE119910B810A810B2091A804249D3F
:1065C000E0199109810A810B0091A904049D901999
:1065D0008108810B3B9FE0199109810A810B2B9F58
:1065E00090198108810B0B9F801881094A9E012D0B
:1065F000332722274F9E000D311D211FBA9F000D0A
:10660000311D211FBF9F300D211D432EB22F309110
:10661000A304349DE10D911F811E811F2091A404CC
:10662000249DE00D911D811E811F0091A504049DF4
:10663000900D811C811F3B9FE00D911D811E811FCC
:106640002B9F900D811C811F0B9F800C811D4A9EEA
:10665000012D332722274F9E000D311D211FBA9F88
:10666000000D311D211FBF9F300D211D432EB22F64
:1066700030919F04349DE119910B810A810B209187
:10668000A004249DE0199109810A810B0091A104C5
:10669000049D90198108810B3B9FE0199109810AA3
:1066A000810B2B9F90198108810B0B9F801881090A
:1066B00082C03091A704349DE10D911F811E811F7E
:1066C0002091A804249DE00D911D811E811F009141
:1066D000A904049D900D811C811F3B9FE00D911D1D
:1066E000811E811F2B9F900D811C811F0B9F800C91
:1066F000811D4A9E012D332722274F9E000D311DFB
:10670000211FBA9F000D311D211FBF9F300D211D7C
:10671000432EB22F3091A304349DE119910B810ACD
:10672000810B2091A404249DE0199109810A810B19
:106730000091A504049D90198108810B3B9FE019ED
:106740009109810A810B2B9F90198108810B0B9F66
:10675000801881094A9E012D332722274F9E000D64
:10676000311D211FBA9F000D311D211FBF9F300D0C
:10677000211D432EB22F30919F04349DE10D911FB6
:10678000811E811F2091A004249DE00D911D811E7A
:10679000811F0091A104049D900D811C811F3B9FCE
:1067A000E00D911D811E811F2B9F900D811C811F6B
:1067B0000B9F800C811D11244B820A83BC83AD8307
:1067C000FE83EF8338872987982C892EB12CA82E39
:1067D0003ECEAA89BB89D1968D909D90AD90BC90FC
:1067E000D49735CED501C401B695A79597958795D1
:1067F0008C7F8F5B954FFC01C590D490FC01329645
:1068000025913491E82DE7708E2EE29FC001E39F21
:10681000900D112433E0969587953A95E1F7C81AC3
:10682000D90AF12CE12C64CE40914C0450914D04D6
:1068300060914E0470914F04481759076A077B070F
:1068400008F030C28090470490904804A09049041A
:10685000B0904A0480914B04EA89FB8981117CC085
:10686000EF5BFF4FE080F18002811381EA89FB89B1
:10687000E25BFF4F2081318142815381AA89BB892C
:10688000D1966D917D918D919C91D4970E945019D4
:10689000B1E0B0934B04EA89FB8941A952A963A9ED
:1068A00074A981E492E1A1E0FC0105911591259183
:1068B0003491041715072607370758F4769567951E
:1068C00057954795AA0F0496EDE5F2E1E817F90709
:1068D00059F7A0935004403251056105710520F429
:1068E00040E250E060E070E04052510961097109F6
:1068F0004115F8E05F076105710508F4B3C124E0B4
:10690000529FC00111248F5B914FFC01329625915B
:106910003491AA27439FF001429FE10DFA1F06948C
:10692000EA1FFA1F1124AF0170E060E0FC01C5907E
:10693000D490F12CE12CC41AD50AE60AF70A8C0C83
:106940009D1CAE1CBF1C8092470490924804A092EC
:106950004904B0924A041BCD81AD92ADA3ADB4AD54
:1069600088169906AA06BB0608F072C18114910424
:10697000A104B10449F440919203509193036091B2
:106980009403709195038DCFA0E0BA85982D492D81
:106990008A2DFB85EC857D856E855F853889298903
:1069A00050918E03599F712D662730918F03399F27
:1069B000700D611D10909003199E600D549F700D15
:1069C000611D349F600D589F600DF72FE62FF79FD4
:1069D000512D33272227F69F500D311D2A1FE79F87
:1069E000500D311D2A1FE69F300D211DF32FE22F80
:1069F000F79FB12D33272227F69FB00D311D2A1F97
:106A0000E79FB00D311D2A1FE69F300D211DF32F8A
:106A1000E22F552790919203409193038091940324
:106A20000090AB040A2A09F483C03091A7043F9F69
:106A300051199A0B4A0B8A0B2091A8042F9F5019C9
:106A400091094A0B8A0BB091A904BF9F9019410983
:106A50008A0B3E9F501991094A0B8A0B2E9F901961
:106A600041098A0BBE9F40198109F79FB12D332739
:106A70002227F69FB00D311D2A1FE79FB00D311D53
:106A80002A1FE69F300D211DF32FE22F3091A30422
:106A90003F9F510D9A1F4A1F8A1F2091A4042F9FC8
:106AA000500D911D4A1F8A1FB091A504BF9F900DE4
:106AB000411D8A1F3E9F500D911D4A1F8A1F2E9F08
:106AC000900D411D8A1FBE9F400D811DF79FB12D66
:106AD00033272227F69FB00D311D2A1FE79FB00DE7
:106AE000311D2A1FE69F300D211DF32FE22F30911B
:106AF0009F043F9F51199A0B4A0B8A0B2091A004C7
:106B00002F9F501991094A0B8A0BB091A104BF9F86
:106B1000901941098A0B3E9F501991094A0B8A0B23
:106B20002E9F901941098A0BBE9F4019810982C08E
:106B30003091A7043F9F510D9A1F4A1F8A1F209131
:106B4000A8042F9F500D911D4A1F8A1FB091A904C0
:106B5000BF9F900D411D8A1F3E9F500D911D4A1FE2
:106B60008A1F2E9F900D411D8A1FBE9F400D811DC3
:106B7000F79FB12D33272227F69FB00D311D2A1F15
:106B8000E79FB00D311D2A1FE69F300D211DF32F09
:106B9000E22F3091A3043F9F51199A0B4A0B8A0BA5
:106BA0002091A4042F9F501991094A0B8A0BB09190
:106BB000A504BF9F901941098A0B3E9F5019910966
:106BC0004A0B8A0B2E9F901941098A0BBE9F4019D0
:106BD0008109F79FB12D33272227F69FB00D311D74
:106BE0002A1FE79FB00D311D2A1FE69F300D211D82
:106BF000F32FE22F30919F043F9F510D9A1F4A1FA0
:106C00008A1F2091A0042F9F500D911D4A1F8A1F9B
:106C1000B091A104BF9F900D411D8A1F3E9F500D52
:106C2000911D4A1F8A1F2E9F900D411D8A1FBE9FD6
:106C3000400D811D1124BA87FB87EC877D876E8705
:106C40005F87388B298B542F492F70E0682F29CE0E
:106C50002A893B89225B3F4FD9014D915D916D910E
:106C60007C911FCEDB01CA01B695A79597958795B4
:106C70008C7F8F5B954FFC01C590D490FC013296C0
:106C8000259134914770429FC001439F900D11247C
:106C9000A3E096958795AA95E1F7C81AD90AF12C31
:106CA000E12C4DCE80912E0190912F01A0913001C9
:106CB000B0913101B7FF61C0EA89FB89EA5BFF4F00
:106CC000C080D180E280F38081E492E121E0FC0188
:106CD00045915591659174914C155D056E057F0543
:106CE00058F4F694E794D794C794220F04964DE590
:106CF00052E14817590759F72093500450E2C5163E
:106D0000D104E104F10428F470E2C72ED12CE12C67
:106D1000F12C60E2C61AD108E108F108C11478E04C
:106D2000D706E104F10408F431C0A4E0DA9EC00102
:106D300011248F5B914FFC01329625913491BC2D2B
:106D40006627B39FA001B29F410D561F0694461FB0
:106D5000561F112470E060E0FC0185919491B0E031
:106D6000A0E0841B950BA60BB70B80932E0190938C
:106D70002F01A0933001B0933101C0902E01D0902B
:106D80002F01E0903001F090310101CBD701C60115
:106D9000B695A795979587958C7F8F5B954FFC014E
:106DA00025913491FC01329645915491EC2DE77078
:106DB000E49FC001E59F900D112463E096958795AF
:106DC0006A95E1F7281B390BC901B0E0A0E0CDCFEF
:106DD000EA89FB8985889688A788B08C81E0811430
:106DE0009104A104B10409F480E0AA89BB895996F1
:106DF000CD90DD90ED90FC905C97C114D104E1043E
:106E0000F10409F08260EA89FB89458D568D678D12
:106E100070A1411551056105710509F084608093E9
:106E20005904109247041092480410924904109299
:106E30004A0410925104109252041092530410927A
:106E40005404EA89FB8985A196A1A7A1B0A58093E6
:106E50005A0490935B04A0935C04B0935D044424B3
:106E600055243201481A590A6A0A7B0A40923704AB
:106E7000509238046092390470923A0440923B0474
:106E800050923C0460923D0470923E0440923F0454
:106E900050924004609241047092420441A052A07A
:106EA00063A074A0440C551C661C771C880C991CAC
:106EB000AA1CBB1C8092270490922804A09229044B
:106EC000B0922A04CC0CDD1CEE1CFF1CC0922B04DB
:106ED000D0922C04E0922D04F0922E04440F551F02
:106EE000661F771F40932F04509330046093310442
:106EF000709332044092330450923404609235040B
:106F000070923604880F991FAA1FBB1F8093230419
:106F100090932404A0932504B093260410925E0459
:106F200010925F04109260041092610481A592A5F2
:106F3000A3A5B4A58093550490935604A093570439
:106F4000B093580485A596A5A7A5B0A980934C0435
:106F500090934D04A0934E04B0934F04EB5BFF4F0E
:106F600080819091E906891721F08093E9060E94BB
:106F7000DD2A0E94DE2E44244A94542C3201409291
:106F80002E0150922F016092300170923101EA89F6
:106F9000FB89FD96E080F18002811381AA89BB897B
:106FA000D1962D913D914D915C91D4976D01BAE4AC
:106FB000CB0ED11CF60160817181828193810E9488
:106FC000501910924B04D6014D915D916D917C91B9
:106FD00081E492E1A1E0FC010591159125913491A4
:106FE000041715072607370758F4769567955795C0
:106FF0004795AA0F0496EDE5F2E1E817F90759F76E
:10700000A0935004403251056105710520F440E21F
:1070100050E060E070E0405251096109710941158A
:10702000F8E05F076105710508F462C024E0529F33
:10703000C00111248F5B914FFC0132962591349150
:10704000AA27439FF001429FE10DFA1F0694EA1F11
:10705000FA1F1124AF0170E060E0FC01C590D490EC
:10706000F12CE12CC41AD50AE60AF70AC092620490
:10707000D0926304E0926404F0926504809162040B
:1070800090916304A0916404B0916504AC01BD01CA
:10709000009731E0A307B10520F04FEF5FEF60E00C
:1070A00070E0841B950BA60BB70B80936204909342
:1070B0006304A0936404B0936504F8948091840001
:1070C000909185004096A981A150A983AA2381F1BE
:1070D000240E351E2816390610F40C94B12F309268
:1070E00089002092880078946396E2E10C9428EE5F
:1070F000DB01CA01B695A795979587958C7F8F5B25
:10710000954FFC01C590D490FC01329625913491A5
:107110004770429FC001439F900D112433E0969524
:1071200087953A95E1F7C81AD90AF12CE12C9ECF40
:107130001C01D5CF80EDC82E87E0D82EE12CF12C94
:107140002DC9CF93DF9380916A1390916B13891BA4
:1071500080958F7019F40E94C68BF5CF80916A13C9
:107160008F5F8F70A0916A139BE5A99FD0011124B6
:10717000FD01ED53F84FEF0119929A95E9F798E068
:107180009083A852B84F90E1ECE6F3E101900D92A4
:107190009A95E1F720916A1390916B13291303C01C
:1071A00094E69093671380936A130E94BC2EDF913C
:1071B000CF910895FC0120813181428153816091FA
:1071C000940D7091950D8091960D9091970D0E9460
:1071D0008BE70E94ACEF60937813709379138093E0
:1071E0007A1390937B1390916A1380916B13981785
:1071F00009F0A7CF0E94DB2B0E94AF2E409178139D
:107200005091791360917A1370917B1340938104AC
:1072100050938204609383047093840481110C94CE
:10722000BC2E08954F925F926F927F928F929F92A1
:10723000AF92BF92CF92DF92EF92FF92CF93DF9304
:10724000EC012091940D3091950D4091960D509147
:10725000970D6C857D858E859F850E948BE70E94AA
:10726000ACEF6B017C012091900D3091910D40911C
:10727000920D5091930D688579858A859B850E9432
:107280008BE70E94ACEF4B015C0120918C0D30919B
:107290008D0D40918E0D50918F0D6C817D818E8171
:1072A0009F810E948BE70E94ACEF2B013C01209153
:1072B000880D3091890D40918A0D50918B0D688118
:1072C00079818A819B810E948BE70E94ACEF609359
:1072D0006C1370936D1380936E1390936F134092A1
:1072E00070135092711360927213709273138092A4
:1072F000741390927513A0927613B0927713C09284
:107300007813D0927913E0927A13F0927B139091D4
:107310006A1380916B13981781F013DFDF91CF917F
:10732000FF90EF90DF90CF90BF90AF909F908F90A5
:107330007F906F905F904F9008950E94DB2B0E948A
:10734000AF2EC82F8CE693E10E944719CC2331F36E
:107350000E94BC2EE3CFCF92DF92EF92FF92CF93A9
:10736000DF93C82F0E94AF2E94E0C99FE001112443
:10737000FE01EB58FB4FC080D180E280F380811189
:107380000E94BC2ECD54D84FC701B6010E942CE7F5
:10739000288139814A815B810E948BE7DF91CF91FF
:1073A000FF90EF90DF90CF900895CF92DF92EF9211
:1073B000FF92CF93DF93C82F0E94AF2E94E0C99F16
:1073C000E0011124FE01E759FB4FC080D180E2802B
:1073D000F38081110E94BC2ECD54D84FC701B60155
:1073E0000E942CE7288139814A815B810E948BE7CA
:1073F000DF91CF91FF90EF90DF90CF900895A1E0C3
:10740000B0E0E5E0FAE30C941CEE898360E0CE0185
:1074100001960E94A21A61E0CE0101960E94A21A72
:1074200062E0CE0101960E94A21A89812196E2E0D3
:107430000C9438EEA2E1B0E0E0E2FAE30C9418EE2E
:10744000DEDF8823C1F1EDB6FEB641E952E082FFEE
:1074500002C048E852E021E932E081FF02C02AE898
:1074600032E080FD25C081E992E05F934F933F9326
:107470002F939F938F9382ED96E09F938F938E012E
:107480000F5F1F4F1F930F930E94BFE60E94B887A4
:10749000C8010E943981C8010E9448C20FB6F89401
:1074A000DEBF0FBECDBF81E06296E6E00C9434EE05
:1074B0008CE892E0DACF80E0F7CFA0E2B0E0E3E63C
:1074C000FAE30C940CEE80911201882309F4BEC0FB
:1074D00080910D04082F10E080FF3CC0C090140183
:1074E000D0901501E0901601F09017012091A302B1
:1074F0003091A4024091A5025091A602C701B601A5
:107500000E94A7EF181644F4C092A302D092A402DE
:10751000E092A502F092A602C0902001D090210135
:10752000E0902201F09023012091A3023091A40267
:107530004091A5025091A602C701B6010E9426E71C
:1075400087FF08C0C092A302D092A402E092A502D5
:10755000F092A60201FF3CC0C0901801D090190122
:10756000E0901A01F0901B012091A7023091A8022F
:107570004091A9025091AA02C701B6010E94A7EF4B
:10758000181644F4C092A702D092A802E092A90271
:10759000F092AA02C0902401D0902501E09026012B
:1075A000F09027012091A7023091A8024091A902F2
:1075B0005091AA02C701B6010E9426E787FF08C0C2
:1075C000C092A702D092A802E092A902F092AA0269
:1075D00002FF3CC0C0901C01D0901D01E0901E0134
:1075E000F0901F012091AB023091AC024091AD02AE
:1075F0005091AE02C701B6010E94A7EF181644F4DD
:10760000C092AB02D092AC02E092AD02F092AE0218
:10761000C0902801D0902901E0902A01F0902B0120
:107620002091AB023091AC024091AD025091AE027C
:10763000C701B6010E9426E787FF08C0C092AB02CF
:10764000D092AC02E092AD02F092AE028091730D46
:1076500083FD61C0209181013091820140918301BD
:10766000509184016091AF027091B0028091B1029B
:107670009091B2020E9426E7882309F44CC00E9430
:107680009BB3182F882331F00E94B88787EB96E0D0
:107690000E944881209181013091820140918301B3
:1076A000509184016091AF027091B0028091B1025B
:1076B0009091B2020E9443EE9F7720916F0130912A
:1076C000700140917101509172010E948BE720E09E
:1076D00030E046E154E40E94A7EF1816D4F40E946B
:1076E000B88788E996E00E9448818091AF02909126
:1076F000B002A091B102B091B20280938101909347
:107700008201A0938301B09384018FEA92E052DD5D
:1077100002C01111EACF2AE037ED43E25CE3609149
:107720000C0170910D0180910E0190910F010E944A
:107730008BE76B017C016091100170911101072EA4
:10774000000C880B990B0E942CE79B01AC01C70130
:10775000B6010E948BE7698B7A8B8B8B9C8B809117
:10776000B302882309F18090B4029090B502A090F2
:10777000B602B090B702C090AB02D090AC02E090DD
:10778000AD02F090AE0220E030E0A901C501B401E5
:107790000E9426E78823F9F0A7019601C501B401EC
:1077A0000E94A7EF1816BCF020E030E0A901BE014E
:1077B0006F5E7F4F83EA92E00E94BCC380E1E3EA00
:1077C000F2E0A5E7B1E001900D928A95E1F7A0966D
:1077D000E2E10C9428EE2091750130917601409100
:1077E0007701509178016091A3027091A402809179
:1077F000A5029091A6020E9443EE4B015C012091EC
:10780000790130917A0140917B0150917C01609126
:10781000A7027091A8028091A9029091AA020E94E9
:1078200043EE6D8B7E8B8F8B988F20917D013091F5
:107830007E0140917F0150918001C701B6010E94F5
:1078400043EE6D8F7E8F8F8F98A3209181013091B1
:10785000820140918301509184016091AF02709147
:10786000B0028091B1029091B2020E9443EE698F02
:107870007A8F8B8F9C8F20E030E0A901C501B40185
:107880000E9426E781110CC020E030E0A9016D893B
:107890007E898F89988D0E9426E7882309F484CFFA
:1078A000A5019401C501B4010E948BE76B017C0125
:1078B0002D893E894F89588DCA01B9010E948BE7F5
:1078C0009B01AC01C701B6010E9444EE6B017C0133
:1078D0002D8D3E8D4F8D58A1CA01B9010E948BE7B5
:1078E0009B01AC01C701B6010E9444EE6B017C0113
:1078F000298D3A8D4B8D5C8DCA01B9010E948BE7B1
:107900009B01AC01C701B6010E9444EE6B017C01F2
:107910000E94E0EF2B013C012CEC3CEB4CE85BE2DD
:10792000C701B6010E9426E787FF06C0498C5A8C22
:107930006B8C7C8CE89477F82DEB37E346E855E3C5
:10794000C301B2010E9426E787FD38CF2DEC3CEC45
:107950004CE45EE3C301B2010E948BE70E9428EF72
:107960001B01672B19F422242394312CB10190E0E0
:1079700080E00E942AE79B01AC0160E070E080E8B3
:107980009FE30E94BBEE6B017C01AC019B01C30134
:10799000B2010E948BE72B013C01A7019601C501B2
:1079A000B4010E948BE74B015C01A70196016D8930
:1079B0007E898F89988D0E948BE76D8B7E8B8F8B54
:1079C000988FA70196016D8D7E8D8F8D98A10E9455
:1079D0008BE76D8F7E8F8F8F98A3A7019601698D9E
:1079E0007A8D8B8D9C8D0E948BE7698F7A8F8B8F20
:1079F0009C8F80E1E5E7F1E08E010F5F1F4FD8011A
:107A000001900D928A95E1F70E94F7CD6B017C0100
:107A100028ECC20ED11CE11CF11C81E0281A3108AF
:107A200009F454C00E94F7CD9B01AC012C193D090B
:107A30004E095F0957FD4DC06B017C0128ECC20E59
:107A4000D11CE11CF11C80E00E94C68BA5019401B1
:107A500069817A818B819C810E9444EE69837A835B
:107A60008B839C832D893E894F89588D6D817E81C2
:107A70008F8198850E9444EE6D837E838F839887E3
:107A80002D8D3E8D4F8D58A169857A858B859C857E
:107A90000E9444EE69877A878B879C87298D3A8D6F
:107AA0004B8D5C8D6D857E858F8598890E9444EE17
:107AB0006D877E878F87988BA3019201BE016F5ED1
:107AC0007F4FC8010E94BCC38111A7CFA3019201BF
:107AD0006ECE0E941D29BACF8091090490910A04AC
:107AE000A0910B04B0910C0480930C0190930D01B4
:107AF000A0930E01B0930F018091070490910804A8
:107B00009093110180931001089580910C01909140
:107B10000D01A0910E01B0910F0180930904909383
:107B20000A04A0930B04B0930C048091100190916F
:107B30001101909308048093070484E690E09093E9
:107B40001101809310010895ACE0B0E0EAEAFDE392
:107B50000C940EEE2B013C0129873A874B875C87FA
:107B600047015801D601CD90DD90ED90FC9020E0CA
:107B700030E0A901C701B6010E9426E7811171C05A
:107B800080916B0190916C01A0916D01B0916E019B
:107B900089839A83AB83BC8320E030E0A901C701CD
:107BA000B6010E9426E7811106C0C12CD12C80E8C5
:107BB000E82E80E4F82ECD82DE82EF82F886A501E1
:107BC000940160917D0170917E0180917F0190917F
:107BD00080010E9426E787FF0CC080927D01909271
:107BE0007E01A0927F01B0928001CE0105960E9495
:107BF000E421409275015092760160927701709273
:107C0000780189859A85AB85BC85809379019093AD
:107C10007A01A0937B01B0937C01CE0101960E9472
:107C2000E421A501940160917D0170917E01809114
:107C30007F01909180010E94A7EF181664F4809252
:107C40007D0190927E01A0927F01B0928001CE01D1
:107C500005960E94E4210E94DB2B2C96E0E10C9417
:107C60002AEED701C60194CFCF92DF92EF92FF9216
:107C70000F931F936B01FC01E080F180028113815F
:107C8000E5E7F1E02481358146815781608171818A
:107C90008281938159DF1F910F91FF90EF90DF90C8
:107CA000CF9008958F929F92AF92BF92CF92DF9222
:107CB000EF92FF921F93CF93DF93CDB7DEB760971C
:107CC0000FB6F894DEBF0FBECDBF182F80E043DBA8
:107CD0004B015C018092FB039092FC03A092FD0398
:107CE000B092FE0381E037DB6B017C01C092FF03A1
:107CF000D0920004E0920104F092020482E02BDBB7
:107D00006093030470930404809305049093060425
:107D10001D861E861F86188A89829A82AB82BC8243
:107D2000CD82DE82EF82F88669877A878B879C878F
:107D300083E011DB6D877E878F87988BCE0101965C
:107D40000E94FD2B1E3FD9F480E1FE013196A5E78C
:107D5000B1E001900D928A95E1F760960FB6F89424
:107D6000DEBF0FBECDBFDF91CF911F91FF90EF908F
:107D7000DF90CF90BF90AF909F908F90089584E058
:107D8000189FF0011124DF01AB58BE4F81E090E055
:107D90008C0F9D1FE80FF91F408151816281738113
:107DA0004D935D936D937C931397D7CF0C94DFC362
:107DB000CF930E94AF2EC82F80916B1380936A13CC
:107DC000809369138093681384E6809367130E94FD
:107DD000402F80ED93E09093BD0D8093BC0DC111B9
:107DE0000E94BC2E81E0809368040E94DB2B8EEF02
:107DF00059DFDCDFCF910895ACE0B0E0E2E0FFE3D3
:107E00000C941CEE0E945AB30E94AF2E9CE0E5E752
:107E1000F4E0DE01119601900D929A95E1F781113F
:107E20000E94BC2ECE0101960E94552A2C96E2E0BB
:107E30000C9438EEB0E0A0E0E0E2FFE30C940EEE2C
:107E400040907501509076016090770170907801B4
:107E50008090790190907A01A0907B01B0907C0194
:107E6000C0907D01D0907E01E0907F01F090800174
:107E70000E946F2B60912C0170912D01072E000C38
:107E8000880B990B0E942CE72AE037ED43E25CE374
:107E90000E948BE760936F01709370018093710172
:107EA0009093720104E111E0D0E0C0E0CE018B506C
:107EB000964F0E94E274F8016193719381939193BC
:107EC0008F01CE018751964F0E94E274F8016087BE
:107ED0007187828793872496CC30D10539F760E08B
:107EE0008BE194E00E94C3770E9490780E94B32BAC
:107EF000A3019201609175017091760180917701E3
:107F0000909178010E9426E781111BC0A501940180
:107F10006091790170917A0180917B0190917C014F
:107F20000E9426E781110DC020917D0130917E01D4
:107F300040917F0150918001C701B6010E9426E760
:107F400081115ADFCDB7DEB7E0E10C942AEE8EE75F
:107F500096E00E94488186B168E776E082FB882738
:107F600080F90E94422186B162E776E083FB882790
:107F700080F90E94422186B16CE676E0829581709C
:107F80000C9442218091E806811103C08091EE0695
:107F900081110C94DE2E0895ACE0B0E0E2EDFFE339
:107FA0000C941CEEA4E7BDE090E080E0FC01EF5CE7
:107FB000F54F45915591659174914D935D936D93F6
:107FC0007D93FC01EF5DF54F45915591659174915D
:107FD00050964D935D936D937C935397FC01EF5EA8
:107FE000F54F459155916591749190964D935D93A0
:107FF0006D937C939397049680319105B9F680E256
:108000009EE4A0E0B0E08093840D9093850DA09352
:10801000860DB093870D80E090E0AAEFB3E48093E3
:10802000A80D9093A90DA093AA0DB093AB0D8093CA
:10803000AC0D9093AD0DA093AE0DB093AF0D8093AA
:10804000B00D9093B10DA093B20DB093B30D1092FB
:10805000B40D1092B50D1092B60D1092B70D10928E
:10806000B80D1092B90D1092BA0D1092BB0D8AE0A6
:1080700097EDA3EABDE38093960790939707A093AB
:108080009807B093990780E090E0A0E2B1E4809374
:108090001B0490931C04A0931D04B0931E040E9423
:1080A00079778CE0E5E8F1E0DE01119601900D9220
:1080B0008A95E1F789819A81AB81BC8180935913BC
:1080C00090935A13A0935B13B0935C138D819E81A0
:1080D000AF81B88580935D1390935E13A0935F1377
:1080E000B093601389859A85AB85BC8580936113B5
:1080F00090936213A0936313B0936413809126024C
:1081000090912702A0912802B09129028093EA065B
:108110009093EB06A093EC06B093ED068EEB90E007
:1081200090934E0780934D078CE390E09093500717
:1081300080934F07109252071092510786EE90E0FD
:10814000909354078093530786E490E090935607EA
:108150008093550710925807109257078FE892ECBA
:10816000ADE8B1E48093C0129093C112A093C21203
:10817000B093C3128CE998EFA5E4BEE38093C412D8
:108180009093C512A093C612B093C71281E49CEBE2
:10819000ABECB3E48093C8129093C912A093CA12B7
:1081A000B093CB1280E090E0AFEAB3E48093410754
:1081B00090934207A0934307B093440785E996E262
:1081C000A5E2B1E48093450790934607A093470743
:1081D000B093480780EA9CE6ACE2B5E48093490797
:1081E00090934A07A0934B07B0934C071092E80670
:1081F0001092E706C7DE1EDE2C96E2E00C9438EE05
:10820000A4E0B0E0E6E0F1E40C940DEE9091EE060F
:10821000981709F45EC0382E80E090E0A0E2B1E447
:1082200089839A83AB83BC8340906113509062131F
:10823000609063137090641320E030E0A901C301E3
:10824000B2010E9426E787FF0CC0A301920160E003
:1082500070E080E291E40E9443EE69837A838B832D
:108260009C83CE0101960E946FC44090750150908E
:1082700076016090770170907801809079019090FC
:108280007A01A0907B01B0907C01E1E0E325F0E071
:10829000EE0FFF1FE651F94F6081718186E593E192
:1082A0000E94A17F19821A821B821C82E0907D01AC
:1082B000F0907E0100917F0110918001CE01019626
:1082C0006C01A5019401C301B2013EDC3092EE06BF
:1082D00059DE80E02496E1E10C9429EE4F925F9202
:1082E0006F927F928F929F92AF92BF92DF92EF92A6
:1082F000FF920F931F93CF93DF93D82EC82FD0E018
:10830000FE01EB55F34DF49082E0D81609F4E3C07A
:108310006F2DFF0C770B880B990B0E942CE72B011C
:108320003C01CE01880F991F880F991F8F5D984FD0
:108330000E94E2744B015C01A3019201C501B401EA
:108340000E948BE74B015C017E01EE0CFF1CEE0CE2
:10835000FF1CC7018B5E984F0E94E2749B01AC0129
:10836000C301B2010E948BE720E030E040EC5FE304
:108370000E948BE7AB01BC0100E010E098018D2D5D
:108380000E94B5C720E030E0A901C501B4010E94F8
:1083900026E7882309F440C082E000E010E020E8EE
:1083A00030E4D81619F000E010E09801B501A401FE
:1083B00070588D2D0E94B5C7A5019401C501B40167
:1083C0000E9444EE4B015C0182E000E010E020E0FE
:1083D00030E4D816E1F0FE01EA5FF84F64916111D4
:1083E00007C00E94B88784EE96E00E9448816AE048
:1083F00070E090E080E00E942AE79B01AC0161E020
:1084000070E088E492E40E94BBEE8B019C01B50110
:10841000A4018D2D0E94B5C781E090E00D2C01C014
:10842000880F0A94EAF790918207982B909382071D
:1084300090910D04892B80930D04C701875F984F9D
:108440000E94E274F701EB58FE4F608371838283D0
:10845000938382E0D8121AC0209161133091621385
:10846000409163135091641360917D0170917E017E
:1084700080917F01909180010E9443EE60937D0185
:1084800070937E0180937F01909380018FDCF701D0
:10849000ED55FD4FD701AB58BE4F8D919D910D907D
:1084A000BC91A02D80839183A283B38382E0D812F4
:1084B00002C080E0A5DEDF91CF911F910F91FF9068
:1084C000EF90DF90BF90AF909F908F907F906F90D4
:1084D0005F904F90089581E093DE8111ECCF89E2A7
:1084E00097E00E94E27420E030E0A9010E9426E7B4
:1084F000882309F40DCF6F2DFF0C770B880B990B98
:108500000E942CE72B013C0189E297E00E94E27473
:108510004B015C0120E030E040EA50E40E94A7EF0C
:1085200087FF0ACF812C912C90EAA92E90E4B92ED6
:1085300003CF80918107882319F010928107089555
:1085400040E070E060E08CE496E00E94D78A1F92E1
:108550000F920FB60F9211240BB60F922F933F93E9
:108560004F935F936F937F938F939F93AF93BF933B
:10857000EF93FF930E94DE2EFF91EF91BF91AF9199
:108580009F918F917F916F915F914F913F912F912B
:108590000F900BBE0F900FBE0F901F9018950F936A
:1085A0001F9380919207813019F50E94F7CD0091B9
:1085B000F2031091F3032091F4033091F503601B53
:1085C000710B820B930B28EE33E040E050E00E94E9
:1085D00054ED6091EE037091EF038091F003909160
:1085E000F103620F731F841F951F1F910F91089550
:1085F0006091F6037091F7038091F8039091F9036D
:10860000D6CF109292071092F2031092F3031092B9
:10861000F4031092F5031092F6031092F7031092F0
:10862000F8031092F9031092EE031092EF031092E8
:10863000F0031092F1030895809192078130E1F0E8
:108640008230C1F4ACDF6093EE037093EF0380934C
:10865000F0039093F10381E0809392070E94F7CD9D
:108660006093F2037093F3038093F4039093F50304
:1086700081E00895C6DFEFCF80E008950E94BDC479
:108680000E942A79882351F08091E81482FD06C067
:1086900087EE91E09093F0068093EF06CDCF809126
:1086A0009207813079F482E0809392070E94F7CD9F
:1086B0006093F6037093F7038093F8039093F903A4
:1086C00081E0089580E00895809192078150823082
:1086D00070F4109292070E94F7CD6093F6037093A6
:1086E000F7038093F8039093F90381E0089580E005
:1086F00008952091BD123091BE12263531053CF40B
:1087000020913E0730913F07263031051CF0882329
:1087100031F092CF662319F0D7DF0C94BDC40895D1
:108720009C0197FF26C0EE27FF27E81BF90B2D3988
:108730008FEF38070CF05DC08DE280939E02CF0171
:1087400064E670E00E94DEEDCB012AE030E0B90182
:108750000E94DEED805D80939F02CF01B9010E94EF
:10876000DEEDCB01B9010E94DEED805D8093A002B9
:108770002AC0283E83E03807B4F1C90168EE73E0EF
:108780000E94DEEDCB01EAE0F0E0BF010E94DEEDE9
:10879000805D80939E02C90164E670E00E94DEED78
:1087A000CB01BF010E94DEED805D80939F02C90175
:1087B000BF010E94DEEDCB01BF010E94DEED805DB6
:1087C0008093A002F901CF016AE070E00E94DEED23
:1087D000805D8093A1028EE992E008958DE237FDDD
:1087E000C5CF80E2C3CFF90180E2243631050CF019
:1087F000A4CF80E280939E0280939F02EA30F1052D
:108800006CF38DE237FF80E280939F02CF016AE034
:1088100070E00E94DEED605D6093A002D4CF9C0109
:1088200097FD2DC080E2243631055CF0C90164E675
:1088300070E00E94DEEDCB016AE070E00E94DEEDA8
:10884000805D80939F0280E22A3031055CF0EAE08F
:10885000F0E0C901BF010E94DEEDCB01BF010E9423
:10886000DEED805D8093A002C9016AE070E00E94A5
:10887000DEED805D8093A1028FE992E0089531954D
:10888000219531098DE2DDCFCF92DF92EF92FF92F9
:10889000FC01C080D180E280F38020E030E0A901BB
:1088A000C701B6010E9426E787FD26C06DEB77E37E
:1088B00086E095E3A70196010E9444EE6B017C01DE
:1088C00020E030E0A9010E9426E720E030E040E00F
:1088D0005FE387FF04C020E030E040E05FEBC701CA
:1088E000B6010E9444EE0E9423EFCB0198DFFF9077
:1088F000EF90DF90CF9008956DEB77E386E095EBF6
:10890000D9CFA4E0B0E0E7E8F4E40C941CEE0E94B8
:108910002CE769837A838B839C83CE010196B4DF35
:108920002496E2E00C9438EEFC0160817181828132
:1089300093810E9423EFCB0172CFA4E0B0E0E3EA81
:10894000F4E40C941CEE0E942CE769837A838B83F9
:108950009C83CE010196E8DF2496E2E00C9438EE89
:108960000F931F930E94F7CD0091E1061091E2064C
:108970002091E3063091E40601151105210531052A
:10898000D9F520917E132223A1F1E0917C1321508F
:1089900020937E1321E02E0F20937C1330917F13C0
:1089A000231302C010927C1324E0E29FF0011124F3
:1089B000E058FC4E00811181228133810093DD0655
:1089C0001093DE062093DF063093E006600F711FE0
:1089D000811D911D6093E1067093E2068093E3068A
:1089E0009093E4068091DF069091E006892B09F0D0
:1089F000149A1F910F910895601B710B820B930BBA
:108A000097FDF7CF14981092E1061092E2061092AB
:108A1000E3061092E406EDCF0F931F93CF93DF93FD
:108A20008C01EB0190917E1320917F13921304C06F
:108A300097DF0E941D29F6CF80917D1334E0839F3C
:108A4000F0011124E058FC4E11830083D383C283CC
:108A50009F5F90937E138F5F281739F080937D136B
:108A6000DF91CF911F910F91089510927D13F8CF50
:108A7000882351F063E972E084E690E0CDDF6AEB91
:108A800072E084E690E0C8CF68EB71E084E190E0AA
:108A9000FACF82DA81E0ECCF8F929F92AF92BF92B1
:108AA000EF92FF920F931F93CF93DF93EC018B0113
:108AB000E42EF22E80919013909191138C179D07C4
:108AC000C9F120E6C93AD20709F03FC08853994757
:108AD00071F40E94F7CD6E517B4F8F4F9F4F609383
:108AE000DE037093DF038093E0039093E103D09360
:108AF0009113C093901330E020E00093740710931B
:108B000075072093760730937707E0926F07F0920E
:108B10007007C853D94721F410929A021092DD03CE
:108B200082E080936A0181E080937107109299023C
:108B30001092E903DF91CF911F910F91FF90EF9079
:108B4000BF90AF909F908F90089529E7C833D207C8
:108B500071F6895A9046D9F40E94F7CD8090DE03D1
:108B60009090DF03A090E003B090E10368197909C9
:108B70008A099B0997FF0BC0809182078770873015
:108B800031F40E94A322CEECD5E58111B0CFC8E329
:108B9000D9E7ADCF20E040E070E060E082E992E20A
:108BA0007BCF0E949BB3882339F020E040E070E047
:108BB00060E080EF94E570CFEDCF21E020939A0242
:108BC000FC0180819181A281B381809308019093FF
:108BD0000901A0930A01B0930B0120E040E070E08E
:108BE00060E080915E0790915F0756CFA4E0B0E00F
:108BF000ECEFF5E40C941CEE8DEC9CECACECBCE3DF
:108C000089839A83AB83BC83CE010196D6DF2496F9
:108C1000E2E00C9438EEA4E0B0E0E1E1F6E40C947C
:108C20001CEE8DEC9CECACECBDE389839A83AB83AA
:108C3000BC83CE010196C1DF2496E2E00C9438EEAD
:108C4000A4E0B0E0E6E2F6E40C941CEE80E090E0F4
:108C5000A0E8BFE389839A83AB83BC83CE010196EE
:108C6000ACDF2496E2E00C9438EEA4E0B0E0EBE355
:108C7000F6E40C941CEE80E090E0A0E2B1E489837D
:108C80009A83AB83BC83CE01019697DF2496E2E002
:108C90000C9438EE81E080939A028091820787706D
:108CA000873051F01092820710920D0486EB95E008
:108CB0009093F0068093EF068091B3028093EB03CC
:108CC00080E00E94377720E040E070E060E08AE6D4
:108CD00096E4E2CE80916A01882331F041E062EAB5
:108CE00073E082E00E9462C880910D048770873033
:108CF00071F41092EA0320E040E070E060E080E769
:108D000095E5CADE81E08093E9030C94EC21089597
:108D100020E040E070E060E088E399E7BDCE10928B
:108D2000B2070E942227F4CFB0E0A0E0EAE9F6E41F
:108D30000C9416EECDB6DEB6E5E8F7E0DF010D9057
:108D40000020E9F7CD018D5797402DB73EB7281B7E
:108D5000390B0FB6F8943EBF0FBE2DBF0DB71EB72F
:108D60000F5F1F4FFF93EF9389E195E09F938F93E0
:108D70001F930F930E94BFE6780134E0E30EF11CCD
:108D80000F900F900F900F900F900F90D7018D9133
:108D90007D01882349F0082E000C990B0E9425F0D4
:108DA000F70131978083F2CF64E175E0C8010E943A
:108DB00058E64FE350E0B80181EF96E00E947DF065
:108DC0000FB6F894DEBE0FBECDBEA2DF0E94BDC4BA
:108DD000E8E00C9432EE8093320720E040E070E04F
:108DE00060E08EE895E558CEA2E8B0E0EAEFF6E460
:108DF0000C940CEEADB6BEB684E690E09093A9124A
:108E00008093A8121092CD121092CC1241E064E02F
:108E100070E0CE0187589F4F0E94A2B243E050E01D
:108E2000BE0167587F4F82E292E00E946FF0892B6B
:108E3000F9F0ED968FADED97882339F08FE3EA9640
:108E40008FAFEA97EB961FAEEB9782E0C4DF81E02D
:108E500080931A0490911A0481E089270FB6F89440
:108E6000BEBE0FBEADBECE57DF4FE2E10C9428EE82
:108E700041E062E070E0CE0183589F4F0E94A2B2B1
:108E8000E9961CAE1DAE1EAE1FAEE9971092CD1234
:108E90001092CC12CE018F579F4F0E94BE21EDB68B
:108EA000FEB6CF57DF4FC880C158D040D12C23E049
:108EB000C20ED11CCC0CDD1CCC0CDD1C8DB79EB7BA
:108EC0008C199D090FB6F8949EBF0FBE8DBFEDB7EC
:108ED000FEB731963F018C199D090FB6F8949EBFDD
:108EE0000FBE8DBFEDB7FEB731964F018C199D09AE
:108EF0000FB6F8949EBF0FBE8DBF0DB71EB70F5FA4
:108F00001F4FB601C3010E94C32140918C0381E031
:108F1000482764E070E084E89DE00E94A2B2B601B8
:108F2000C4010E94C321B601C8010E94C3219091CF
:108F30008C03CE57DF4F9883C258D04091114BC05D
:108F4000CF57DF4F8881C158D04090E00296A4E708
:108F5000BDE050E040E030E020E06DE37AE0EDE29B
:108F6000CE2EEAE0DE2E821793070CF495C0F301B3
:108F7000E40FF51F20803180428053802D923D9276
:108F80004D925D92821793070CF48CC0F401E40FAC
:108F9000F51F208031804280538050962D923D9263
:108FA0004D925C925397821793070CF481C0F8019D
:108FB000E40FF51F208031804280538090962D92DF
:108FC0003D924D925C9293972F5F3F4F4C5F5F4F66
:108FD0002430310541F688EA9DE00E9496218CEA12
:108FE0009DE00E94962180EB9DE00E94962184EBFB
:108FF0009DE00E94962188EB9DE00E949621CE0183
:109000008B589F4F0E949621CE018B589F4F0E94F4
:109010009621CE018B589F4F0E949621CE018B58EE
:109020009F4F0E94962186E997E00E9496210FB6F5
:10903000F894FEBE0FBEEDBE8E010F5F1F4FC8013C
:109040000E94B621CE0183599F4F0E949E21C801E4
:109050000E9496218BE194E00E949621CE018B58CC
:109060009F4F0E949621CE0183599F4F0E94BE219F
:10907000C8010E94BE21AE96CFACAE978981C89E32
:1090800060011124E1E0CE1AD108C8F0CE018B585E
:109090009F4F0E949621F6CFFB0125903590459079
:1090A00054906CCFF601259035904590549075CF33
:1090B000EDE1FAE025903590459054907FCF89E519
:1090C00093E10E94B6218AE0D82EDA94CE01DD2009
:1090D00029F08B589F4F0E949621F7CF80589F4FC1
:1090E0000E94BE21CE0181589F4F0E94BE21C058D0
:1090F000DF4F8881C058D040873009F05EC1C15829
:10910000DF4F8881CF57D040873009F056C1CE5706
:10911000DF4F2881C258D040211103C080E00E9457
:10912000377784E893E00E94AE218CE793E00E94B9
:10913000AE2140918C0381E0482764EC70E088EB1D
:1091400092E00E94A2B2C8010E94A621CE018359DA
:109150009F4F0E949E2140918C03FF24F3944F2542
:1091600064E070E08AEE96E00E94A2B2C8010E941C
:10917000A62140918C034F256CE070E08DE497E0D0
:109180000E94A2B240918C034F2564E170E0C801B7
:109190000E94A2B2F0908C03F11030C089819A81B4
:1091A000AB81BC818093C0129093C112A093C21274
:1091B000B093C3122CEA35EC47E25EE36D817E8109
:1091C0008F8198850E948BE76093C4127093C512BB
:1091D0008093C6129093C71220E030E543EC50E430
:1091E00069857A858B859C850E948BE76093C81280
:1091F0007093C9128093CA129093CB1241E04F250D
:1092000062E070E0C8010E94A2B2C8010E948E21F3
:10921000D0908C03D11030C089819A81AB81BC8100
:109220008093410790934207A0934307B09344076C
:109230002CEA35EC47E25EE36D817E818F81988573
:109240000E948BE76093450770934607809347071A
:109250009093480720E030E543EC50E469857A8537
:109260008B859C850E948BE76093490770934A0722
:1092700080934B0790934C07C8010E948E21C80130
:109280000E949E21C8010E949E21C8010E949E2129
:1092900085E0F80111928A95E9F7FF24F3944D2DAA
:1092A0004F2565E070E0C8010E94A2B2C8010E948B
:1092B000A62140918C034F2560E270E0C8010E9416
:1092C000A2B2CE0183599F4F0E94A62140918C03E8
:1092D0004F2569E070E0C8010E94A2B240918C0362
:1092E0004F2562E170E0C8010E94A2B240918C0358
:1092F0004F2564E270E0C8010E94A2B240918C0345
:109300004F2560E170E0C8010E94A2B240918C0339
:109310004F2569E070E0C8010E94A2B2C8010E9416
:10932000962140918C034F256CE070E0C8010E94AB
:10933000A2B240918C034F256CE670E0C8010E94F8
:10934000A2B219821A821B821C821D821E821F8277
:10935000188619861A861B861C86C8010E948E21D3
:1093600040918C034F2568E070E0C8010E94A2B2D2
:10937000C8010E94B621CE0181589F4F0E949E21B4
:10938000CE0183599F4F0E9496218091A8129091FF
:10939000A9128037934089F510921A042091CC12BB
:1093A0003091CD12EF968EAD9FADEF97281739070C
:1093B00041F1F0921A0480E023C0CE0183599F4FFF
:1093C0000E94AE21C8010E94AE21C058DF4FC88064
:1093D000C058D040C158DF4F8881CF57D040C89E79
:1093E0006001112481E0C81AD10808F4ACCECE0186
:1093F0008B589F4F0E949621F5CFF0921A0481E07E
:10940000EADC80918C03811125CD80911A048111B1
:1094100021CD0E941A3F1ECD81E080938C03E4DCB5
:1094200010928C03882309F0DFCC0E94CC3F80E0AF
:109430000895F2DF1DCBCF93DF93C091DD03CC23E2
:10944000B1F0C150C093DD0389E0C89FE001112451
:10945000C955DC4F6A817B812F814E81888199813A
:109460001BDB888580939A02DF91CF91089550DCB1
:10947000FBCFA4E0B0E0EFE3FAE40C940FEE0E941F
:1094800076C9F0906F076F2C85E0782E7F0C86E010
:10949000E82EEF1885E0D82EDF18AA24AA94B12C64
:1094A00084E0C82ECF1882E0982E9F1881E0882E85
:1094B0008F185F2C5194F1105AC080917207882345
:1094C00009F444C080916A01882359F081E09091A9
:1094D0007207911180E024E047E456E0652D0E9478
:1094E000C2C88091B2078093320724E0F212F7C01D
:1094F00010927E0780917207843009F4DDC080915C
:109500006A018823E1F011E080917207843009F04C
:1095100010E08091320724E6829FC0011124815817
:109520009F4FB5010E94DEED862F0E94751C00E062
:109530009C014CE256E06C2D812F0E94E072F39466
:10954000F710B9CF87E0809370070DC0809159075D
:1095500010925907882309F4B5CF6DDF8091710708
:10956000882309F4AFCF2496EFE00C942BEE21E092
:10957000F21243C080917207813041F180916A01FB
:109580008823F9F011E080917207813009F010E032
:109590006091100170911101072E000C880B990B3E
:1095A0000E942CE769837A838B839C83CE0101968A
:1095B000BBD900E09C0141E456E0682D812F0E9458
:1095C000E0728091B20780933207B9CF809159073A
:1095D00010925907882391F210E000E027EE33E063
:1095E0004AE050E060E171E081E496E00E943BCA0D
:1095F00080917107882311F2B6CF82E0F812D7C0AC
:1096000080917207823021F180916A018823C9F22A
:1096100011E080917207823009F010E06091BD1274
:109620007091BE12072E000C880B990B0E942CE73C
:1096300069837A838B839C83CE01019675D900E080
:109640009C014AE356E0692D812F0E94E07249CFC8
:1096500080915907109259078823B1F20E946AC974
:109660000CE811E225EF30E050E040E06DEB72E1F4
:109670008AE396E00E943BCA80917107882321F219
:1096800072CF8091590710925907882309F497C027
:109690000E946AC90FE917E623E730E050E040E096
:1096A0006EE377E086E396E00E943BCA8091710703
:1096B000882309F484C057CF809159071092590725
:1096C000882309F41CCF0E946AC98CE296E00E94AC
:1096D000B0CC80917107882309F411CF44CF85E085
:1096E000F8123DC080917207853011F180916A01B6
:1096F000882309F424CF11E080917207853009F0A6
:1097000010E060912C0170912D01072E000C880B48
:10971000990B0E942CE769837A838B839C83CE010B
:10972000019602D900E09C0147E256E06D2D04CF7E
:1097300080915907109259078823C1F206E91CE16C
:1097400027EE33E04AE050E06CE271E087E296E019
:109750000E943BCA80917107882341F204CF26E022
:10976000F212EDCE80917207863091F080916A01FD
:10977000882309F4E4CE81E090917207963009F0D5
:1097800080E023E048E156E06E2D0E94C2C8D7CEAB
:109790008091590710925907882341F38EEC95E583
:1097A0000E94CCC980917107882301F3DCCE83E04D
:1097B000F81297CE80917207833009F462CF8091BE
:1097C0006A01882309F4FDCE11E08091720783308D
:1097D00009F010E060913E0770913F07072E000CE2
:1097E000880B990B0E942CE769837A838B839C8377
:1097F000CE01019699D863E0661900E09C0146E32A
:1098000056E022CFA4E0B0E0E8E0FCE40C940DEEDA
:10981000EE24E3948091BD129091BE12892B09F43D
:10982000E12C0E9476C9F0906F074F2C95E0592EDD
:109830005F0C88248A94912C83E0B82EBF1882E0B4
:10984000A82EAF1881E0782E7F183F2C319486E047
:10985000682E6F18F11015C080917207882309F4E3
:10986000D7C080916A01882309F475C181E0909185
:109870007207911180E024E043E156E0632D0E94DD
:10988000C2C88091BD129091BE129093330780930D
:10989000320721E0F212E8C080917207813009F4AA
:1098A000C8C080916A01882309F44DC011E08091FD
:1098B0007207813009F010E0609132077091330730
:1098C000072E000C880B990B0E942CE769837A8382
:1098D0008B839C83CE01019627D800E09C014CE04D
:1098E00056E0672D812F0E94E0728091B20780932D
:1098F000320793E0F91227C010927E078091720719
:10990000833009F4F4C080916A018823E1F011E00A
:1099100080917207833009F010E08091320724E6CD
:10992000829FC001112481589F4FB4010E94DEED37
:10993000862F0E94751C00E09C014EEF55E06B2DB8
:10994000812F0E94E072D12CC12C14E00F2D04193C
:10995000C0923207F1121FC0F601EE0FFF1FE9514E
:10996000FA4F859194919093800780937F0780911F
:1099700072078F1509F4CEC080916A01882359F0CF
:1099800081E090917207911380E023E044EF55E06D
:10999000602F0E94C2C8812F9FEFC91AD90A15E013
:1099A0008530B1F680913E0790913F07892B19F4DD
:1099B000EE2009F4CEC026E0F21221C08091720799
:1099C000863009F4B8C080916A018823C1F08FE81D
:1099D00096E49F938F938BEE95E09F938F936F9276
:1099E00081E090917207963009F080E08F930E9499
:1099F0005E220F900F900F900F900F900F9087E0C6
:109A0000EE24E394F394F51025CF809370070DC0F6
:109A10008091590710925907882309F422CF0BDD52
:109A200080917107882309F41CCF2496E1E10C94FE
:109A300029EE8091590710925907882309F431CFF4
:109A40000E946AC90EE612E225EF30E050E040E0E5
:109A500062E377E08CE096E00E943BCA8091710758
:109A6000882309F41ECFE1CF82E0F8123ECF809127
:109A70007207823019F180916A01882309F463CF5B
:109A800011E080917207823009F010E060913E078A
:109A900070913F07072E000C880B990B0E942CE752
:109AA00069837A838B839C83CE0101960E949444C0
:109AB00000E09C0148E056E06A2D14CF80915907E0
:109AC000109259078823B9F20E946AC90FE917E674
:109AD00023E730E050E040E06EE377E088E096E096
:109AE0000E943BCA80917107882329F29ECF809102
:109AF000590710925907882309F405CF0E946AC9B3
:109B00008EEF95E00E94B0CC80917107882309F414
:109B1000FACE8BCF8091590710925907882309F408
:109B20002BCF84EB9DE40E94CCC9809171078823E0
:109B300009F422CF7ACF80915907109259078823D0
:109B400009F441CFECD880917107882309F43BCF09
:109B50006CCF86E057CF8091BD129091BE1290934A
:109B6000330780933207C1CEB0E0A0E0EAEBFDE41A
:109B70000C940EEE009132070E9476C9C0916F07D7
:109B800010E0000F111F09511A4F95E0592E5C0E7D
:109B90002FEBE22E25E0F22ED3E0DC1B3EE7C32EB6
:109BA00032E2D32E4DECA42E45E0B42E82E0782E86
:109BB0007C1A54EF852E55E0952E81E0682E6C1AA4
:109BC0004C2E4194C1112AC0809172078823B1F0B4
:109BD00080916A01882359F081E090917207911178
:109BE00080E024E04BED55E0642D0E94C2C8CF5FB9
:109BF000C511E8CF84E0809370070BC080915907AE
:109C000010925907882321F316DC8091710788236D
:109C1000F9F2CDB7DEB7E0E10C942AEEC13059F588
:109C2000F801859194919093800780937F078091AC
:109C30007207813081F080916A018823C1F21F92FE
:109C40009F928F926F9281E090917207913009F408
:109C500074C080E072C08091590710925907882320
:109C600051F380913207682F0E9442CE8091710794
:109C7000882309F3CECFC23009F042C0F8018591A4
:109C800094919093800780937F0780917207823030
:109C9000D1F080916A01882309F4A9CFDF92CF9295
:109CA000BF92AF927F9281E090917207923009F05B
:109CB00080E08F930E945E220F900F900F900F9084
:109CC0000F900F9094CF80915907109259078823D5
:109CD00001F30E947E22809171078823D1F299CFEF
:109CE00080915907109259078823C1F0609132077B
:109CF0008FEF0E9442CE80917107882379F089CF3F
:109D0000C33009F074CFF801859194919093800746
:109D100080937F0780917207833011F380916A01ED
:109D2000882309F464CF1F92FF92EF92DF9381E0C2
:109D300090917207933009F08CCF8F930E945E222E
:109D40000F900F900F900F900F9051CFB0E0A0E0C8
:109D5000ECEAFEE40C9413EE0E9476C9C0916F0702
:109D600085E0E82EEC0E9BE9C92E95E0D92ED4E0D3
:109D7000DC1B13E01C1B26EBA22E25E0B22E02E01A
:109D80000C1B81E0F82EFC1A9C2E9194C1112AC064
:109D9000809172078823B1F080916A01882359F07D
:109DA00081E090917207911180E024E04AEB55E048
:109DB000692D0E94C2C8CF5FEC12E8CF85E0809386
:109DC00070070BC08091590710925907882321F31F
:109DD00032DB809171078823F9F2CDB7DEB7EBE073
:109DE0000C942FEEC13011F580917207813079F01B
:109DF00080916A018823F9F281E090917207913095
:109E000009F080E023E047E65CE26F2DD2CF80913D
:109E1000590710925907882359F383E89FE40E9459
:109E2000CCC980917107882319F3D7CFC23009F0CC
:109E300053C090917207923071F080916A0188232B
:109E400009F4B9CF81E0923009F080E020E24CEAD9
:109E500055E0602FAECF80915907109259078823A3
:109E600061F3B092F006A092EF068091710788230B
:109E700021F3B3CF80917207833081F080916A0122
:109E8000882309F498CF81E090917207933009F00C
:109E900080E023E04FE955E0612F8BCF8091590797
:109EA00010925907882351F38EEC9CE50E94CCC98F
:109EB00080917107882311F390CF809159071092F8
:109EC0005907882391F0D092F006C092EF06809156
:109ED0007107882351F081CFC33061F2C43009F09B
:109EE0006ACF90917207943041F380916A01882380
:109EF00009F461CF81E0943009F080E020E24AE883
:109F000055E06D2F56CFB0E0A0E0E9E8FFE40C94F7
:109F100017EE0E9476C9C0916F0785E0E82EEC0E1F
:109F2000D4E0DC1B13E01C1B02E00C1B81E0F82ECC
:109F3000FC1ADC2ED194C1112AC0809172078823AB
:109F4000B1F080916A01882359F081E09091720705
:109F5000911180E024E043E855E06D2D0E94C2C8D5
:109F6000CF5FEC12E8CF85E0809370070BC0809143
:109F7000590710925907882321F35DDA8091710700
:109F80008823F9F2CDB7DEB7E7E00C9433EEC130A9
:109F900011F580917207813079F080916A018823F0
:109FA000F9F281E090917207913009F080E023E0AE
:109FB0004DE85CE26F2DD2CF80915907109259077E
:109FC000882359F38DE892E20E94CCC980917107F1
:109FD000882319F3D7CFC23009F055C0809172079A
:109FE000823081F080916A01882309F4B9CF81E041
:109FF00090917207923009F080E023E046E85CE23D
:10A00000602FACCF8091590710925907882351F3E4
:10A0100088E892E20E94CCC980917107882311F3ED
:10A02000B1CF80917207833081F080916A018823DB
:10A0300009F496CF81E090917207933009F080E0A7
:10A0400023E04FE75CE2612F89CF8091590710929E
:10A050005907882351F383E892E20E94CCC980918A
:10A060007107882311F38ECF8091590710925907F9
:10A07000882391F081ED95E40E94CCC9809171070D
:10A08000882351F07FCFC33061F2C43009F068CF2C
:10A0900080917207843041F380916A01882309F42A
:10A0A0005FCF81E090917207943009F080E023E067
:10A0B00041E75CE26D2F52CFACE0B0E0E2E6F0E5C4
:10A0C0000C940DEE9C878B87362E80915907109249
:10A0D0005907882339F010929A02ADD92C96E1E104
:10A0E0000C9429EE60917407709175078091760742
:10A0F00090917707611571058105910509F45CC0A0
:10A1000020911201222309F4AEC0209113012111E4
:10A11000AAC021E0321609F484C0E2E03E1609F438
:10A1200091C0C0901401D0901501E0901601F090FC
:10A130001701409020015090210160902201709001
:10A1400023010E942CE720910801309109014091E0
:10A150000A0150910B010E948BE76F8378878987F2
:10A160009A87F4E03F9E80011124C8018B589E4FCE
:10A170009E838D83FC0120813181428153816F81D7
:10A18000788589859A850E9444EE4B015C01A30184
:10A190009201C701B6010E9426E7811173C0F80140
:10A1A000EB58FE4F80829182A282B382832D0E945F
:10A1B0008A6B81E080936A01109274071092750790
:10A1C000109276071092770780916A01882309F42C
:10A1D00085CF24E0329EF0011124EB58FE4FC08061
:10A1E000D180E280F380C982DA82EB82FC822DEC9E
:10A1F0003CEC4CEC5DE360910801709109018091A9
:10A200000A0190910B010E94A7EF87FD65C0CE0166
:10A2100001960E94C31ABC018B859C850E947972AD
:10A220005DCFC0901801D0901901E0901A01F09014
:10A230001B014090240150902501609026017090F0
:10A2400027017FCFC0901C01D0901D01E0901E011E
:10A25000F0901F01409028015090290160902A0140
:10A2600070902B016ECF412C20E5522E23EC622EF4
:10A2700027E4722EC12C30E5D32E33ECE32E37ECDD
:10A28000F32E5FCF20E030E0A9016F8178858985CA
:10A290009A850E9426E787FF0FC0A7019601C50196
:10A2A000B4010E9426E787FF7ACFED81FE81C0824C
:10A2B000D182E282F3827ACFA3019201C501B40177
:10A2C0000E94A7EF18160CF06ACFED81FE81408244
:10A2D0005182628273826ACF20E030E44CE156E41E
:10A2E000C701B6010E948BE74B015C0120E030E022
:10A2F000A901C701B6010E9426E720E030E040EA4C
:10A3000050E487FF04C020E030E040EA50ECC50193
:10A31000B4010E9444EE2DEC3CEC4CEC5DE30E9459
:10A320008BE70E9423EF6B017C01F7FC64C020EAFD
:10A3300036E841E050E00E9476EDCA01B9012AE01A
:10A3400030E040E050E00E9476ED605D60939B025B
:10A35000C701B60120E137E240E050E00E9476ED0F
:10A360008AE0882E912CA12CB12CCA01B901A5013B
:10A3700094010E9476ED605D60939C02C701B60176
:10A3800028EE33E040E050E00E9476EDCA01B901CA
:10A39000A50194010E9476ED605D60939D028EE2BE
:10A3A00080939E02C701B60124E630E040E050E011
:10A3B0000E9476EDCA01B901A50194010E9476EDD3
:10A3C000605D60939F02C701B601A50194010E94E0
:10A3D00076ED6B017C01CA01B901A50194010E94CF
:10A3E00076ED605D6093A00280E3C80EC092A1028A
:10A3F0008BE992E010CFF094E094D094C094C11C0B
:10A40000D11CE11CF11C6DE2A1CF62E08FE79CE260
:10A4100053CE61E086E89CE24FCE60E08DE89CE29E
:10A420004BCEA4E0B0E0E7E1F2E50C941CEE8091A5
:10A43000590710925907882341F010929A020E94FE
:10A440001B4A2496E2E00C9438EE609174077091F8
:10A4500075078091760790917707611571058105E1
:10A46000910561F10E942CE72091080130910901CA
:10A4700040910A0150910B010E948BE720918101CC
:10A480003091820140918301509184010E9444EEF9
:10A490006093810170938201809383019093840182
:10A4A00083E00E948A6B81E080936A0110927407B6
:10A4B00010927507109276071092770780916A01C3
:10A4C000882309F4BECF20915A0730915B07409151
:10A4D0005C0750915D0760918101709182018091CC
:10A4E0008301909184010E9443EE69837A838B8378
:10A4F0009C83CE0101960E94C31ABC0181E79CE2B5
:10A500000E9479729ECFB0E0A0E0E9E8F2E50C94F9
:10A5100017EE0E94A322082F0E9476C9C0916F07F0
:10A52000FC2E85E0E82EEC0E11E01C1BDC2ED194F5
:10A53000C11114C0809172078823F9F080916A01DB
:10A54000882309F474C081E090917207911180E032
:10A5500024E04CE753E06D2D0E94C2C801113AC0BF
:10A56000D2E0C130C1F5809172078130B9F080919D
:10A570006A01811122C0D2E044C080915907109233
:10A5800059078823D9F20E941B4A809171078823BA
:10A59000A9F2CDB7DEB7E7E00C9433EE809159070E
:10A5A00010925907882319F384E393E50E94CCC9DC
:10A5B000809171078823D9F2ECCF81E090917207E6
:10A5C000913009F080E023E043E753E0612F0E94DF
:10A5D000C2C8D1CFD1E0DC1314C0809172078D17AF
:10A5E000B9F080916A01882361F06C2F6F1981E0C6
:10A5F000909172079C1380E023E047E653E00E94AD
:10A60000C2C8CF5FCE1194CFDF5FD0937007C1CFA8
:10A610008091590710925907882319F387E598E527
:10A620000E94CCC9809171078823D9F2B2CFD1E0C2
:10A63000002309F4A0CFE5CF80E090E0A0E8B0E4EB
:10A6400080937D0190937E01A0937F01B093800160
:10A650008AE192E00E94E4218091EB030E94377727
:10A6600010929A020C941B4AB0E0A0E0EAE3F3E5F2
:10A670000C9415EE0E9476C9C0916F0785E0C82E34
:10A68000CC0ED4E0DC1B13E01C1B82E0F82EFC1A7D
:10A6900081E0E82EEC1ABC2EB194C1112BC0809140
:10A6A00072078823B1F080916A01882359F081E014
:10A6B00090917207911180E024E045E553E06B2D05
:10A6C0000E94C2C8CF5FCC12E8CF85E080937007AC
:10A6D0000CC08091590710925907882321F30E94DA
:10A6E0001B4A809171078823F1F2CDB7DEB7E9E00C
:10A6F0000C9431EEC13089F5809172078130C1F040
:10A7000080916A018823F1F2DD24D394809172074D
:10A71000813009F0D12C88E89DE00E94A91D00E05D
:10A720009C014AE453E06E2D8D2D0E94E072CACF49
:10A730008091590710925907882311F30E946AC922
:10A740004AED5BE268E87DE08AE493E00E94DBC9C1
:10A75000809171078823A1F2C8CFC23009F073C07D
:10A76000809172078230B1F080916A01882309F4E8
:10A77000A9CFDD24D39480917207823009F0D12CC7
:10A780008CE89DE00E94A91D00E09C014FE353E08E
:10A790006F2DCACF8091590710925907882321F352
:10A7A0000E946AC949ED5BE26CE87DE08FE393E0CB
:10A7B0000E94DBC9809171078823B1F296CF809106
:10A7C00072078330B1F080916A01882309F47ACF4F
:10A7D000DD24D39480917207833009F0D12C80E975
:10A7E0009DE00E94A91D00E09C0144E353E0612F1D
:10A7F0009BCF8091590710925907882321F30E941B
:10A800006AC948ED5BE260E97DE084E393E00E9481
:10A81000DBC9809171078823B1F267CF8091590716
:10A82000109259078823C9F00E946AC947ED5BE27C
:10A8300064E97DE089E293E00E94DBC980917107C1
:10A84000882359F052CFC33009F4B9CFC43009F08E
:10A8500039CF80917207843009F380916A0188238F
:10A8600009F430CFDD24D39480917207843009F04D
:10A87000D12C84E99DE00E94A91D00E09C0149E2E1
:10A8800053E06D2F51CFA3E0B0E0E9E4F4E50C9480
:10A890000CEE4C013B015A011901280181E0809323
:10A8A0009A024091740750917507609176077091F4
:10A8B0007707411551056105710571F014161506EC
:10A8C0000CF080E08093E9031092740710927507F2
:10A8D00010927607109277071091E903809159073B
:10A8E0008B8310925907811105C080916A018823DA
:10A8F00009F46FC0C2010E94326C082F80E0C114BD
:10A90000D10419F0C6010E94326C1A821982E11436
:10A91000F104B1F4402F50E0282F30E0CA01820F3B
:10A92000931F46976CF485E190E0841B950B821B86
:10A93000930B97FD0196959587958A8381E089838E
:10A9400001E022E336E6A201BE016F5F7F4FCE0138
:10A9500002960E948A6DE114F10491F08A818823A5
:10A9600021F01A8289818F5F898300E025E336E632
:10A97000A701BE016F5F7F4FCE0102960E948A6DD4
:10A98000C114D10459F000E022E336E6A601BE016D
:10A990006F5F7F4FCE0102960E948A6D41E0412792
:10A9A000B30181E00E947CD0C4010E94326C412F2F
:10A9B000B40194E1981B892F0E947CD0EB81EE2397
:10A9C00041F0111101C05101A114B10431F0F501A0
:10A9D00009952396E2E10C9428EE0E941B4AF9CFD8
:10A9E000CF92DF92EF92FF920F931F9384E6C82ECF
:10A9F00085E0D82EF12CE12C06E615E030E020E0D1
:10AA00004AEC55E466E775E08BE795E03CDF1F9183
:10AA10000F91FF90EF90DF90CF900895B0E0A0E00D
:10AA2000E4E1F5E50C9414EEADB6BEB680912E10BF
:10AA300065E877E0882311F06EE270E1FB01019098
:10AA40000020E9F7CF01861B970B01962DB73EB783
:10AA5000281B390B0FB6F8943EBF0FBE2DBF8DB724
:10AA60009EB701967C0180E2EDB7FEB78183C701F6
:10AA700001960E9468F080E2C82E85E0D82E02E29E
:10AA800015E030E020E044E956E46EE275E085E34D
:10AA900095E0F9DE0FB6F894BEBE0FBEADBEEAE09B
:10AAA0000C9430EECF92DF92EF92FF920F931F93B0
:10AAB0008EE7C82E84E0D82EF12CE12C01EF14E0B3
:10AAC00030E020E045EF52E660E874E085E894E08D
:10AAD000DADE1F910F91FF90EF90DF90CF900895F5
:10AAE000CF92DF92EF92FF920F931F938AE8C82EC6
:10AAF00083E0D82EF12CE12C0CE813E02CE133E5B7
:10AB00004CEE51E268E973E08DE993E0BCDE1F9101
:10AB10000F91FF90EF90DF90CF900895B0E0A0E00C
:10AB2000E4E9F5E50C9414EEADB6BEB683E392E02D
:10AB30000E94326C90E001962DB73EB7281B390B6E
:10AB40000FB6F8943EBF0FBE2DBF8DB79EB70196CE
:10AB50007C0163E372E00E946EE68091320700E0C0
:10AB600012E0813031F00BEE11E0823011F003E1A0
:10AB700012E084E2C82E82E0D82E28E836E445E7C9
:10AB800050E666E272E08DE292E07DDE0FB6F89468
:10AB9000BEBE0FBEADBEEAE00C9430EE8F929F9227
:10ABA000AF92BF92CF92DF92EF92FF920F9380917C
:10ABB000590710925907882371F010929A020E9447
:10ABC0001B4A0F91FF90EF90DF90CF90BF90AF9016
:10ABD0009F908F90089581E080939A0280917407EE
:10ABE00090917507A0917607B09177070097A1051E
:10ABF000B10509F44AC05C01AA0CBB1CAA0CBB1C21
:10AC000010927407109275071092760710927707CA
:10AC1000B5010B2C000C880B990B0E942CE720919E
:10AC2000BB073091BC074091BD075091BE070E9401
:10AC30008BE720916113309162134091631350911F
:10AC400064130E9444EE6B017C0120E030E040EA96
:10AC500051EC0E94A7EF87FD18C020E030E040EAE9
:10AC600051E4C701B6010E9426E7181674F0C50129
:10AC70000E94E0C4C0926113D0926213E092631309
:10AC8000F092641382E080936A0180916A018823C4
:10AC900009F497CFC0906113D0906213E0906313D2
:10ACA000F090641320E030E44CE156E4C701B601B3
:10ACB0000E948BE74B015C0120E030E0A901C70155
:10ACC000B6010E9426E720E030E040EA50E487FF2A
:10ACD00004C020E030E040EA50ECC501B4010E941D
:10ACE00044EE2DEC3CEC4CEC5DE30E948BE70E94C3
:10ACF00023EF6B017C018BE2F7FE09C0F094E09436
:10AD0000D094C094C11CD11CE11CF11C8DE2809335
:10AD10009B02C701B60120E137E240E050E00E940B
:10AD200076ED6AE0862E912CA12CB12CCA01B901D6
:10AD3000A50194010E9476ED605D60939C02C701BD
:10AD4000B60128EE33E040E050E00E9476EDCA0103
:10AD5000B901A50194010E9476ED605D60939D02AA
:10AD60008EE280939E02C701B60124E630E040E007
:10AD700050E00E9476EDCA01B901A50194010E943C
:10AD800076ED605D60939F02C701B601A501940155
:10AD90000E9476ED6B01CA01B901A50194010E94E0
:10ADA00076ED605D6093A00260E36C0D6093A1029C
:10ADB0006BE972E084EF92E00E947972C0906113B7
:10ADC000D0906213E0906313F09064138090E503D9
:10ADD0009090E603A090E703B090E803A5019401EA
:10ADE000C701B6010E9426E78823E9F020E030E0A1
:10ADF000A901C701B6010E9426E7882309F479C09A
:10AE0000A5019401C701B6010E9426E787FD73C022
:10AE100081E08093E403C092E503D092E603E092E0
:10AE2000E703F092E803D090E4038091CA138131E4
:10AE300088F48091CC13833068F044E04D195CEDC8
:10AE4000E52E52E0F52E0CE022E062E486E993E183
:10AE50000E94B8D18091CA13853180F48091CC13BF
:10AE6000843160F049EDE42E42E0F42E01E023E06D
:10AE700044E16CE386E993E10E94B8D18091CA1362
:10AE80008F3308F09ECE8091CC138F3208F499CE88
:10AE900040E34D198FEBE82E82E0F82E0DE022E022
:10AEA0006AE586E993E10E94B8D141E34D1995EA3C
:10AEB000E92E92E0F92E22E065E086E993E10E9416
:10AEC000B8D125E7E22E22E0F22E00E123E04FE2A6
:10AED00062E186E993E10E94B8D135E4E32E32E0E5
:10AEE000F32E23E04FE267E686E993E10E94B8D1B2
:10AEF00068CE80E08ECF8FEF8CCF0F931F93CF93D0
:10AF0000DF93FC01EB018091740790917507A0918C
:10AF10007607B0917707B7FF08C0109274071092B8
:10AF200075071092760710927707809163079091CA
:10AF30006407A0916507B09166074091740750912E
:10AF40007507609176077091770784179507A607B4
:10AF5000B70744F48093740790937507A09376071E
:10AF6000B093770780916A018823E1F060917407BC
:10AF70007091750780917607909177070091670728
:10AF8000109168072091690730916A07600F711F5F
:10AF9000821F931F0995BC0180916D0790916E07E8
:10AFA0000E94797280915907811108C080916007D1
:10AFB0008823A9F180916A01882389F180916B0728
:10AFC00090916C070097B1F040917407509175070C
:10AFD0006091760770917707009167071091680775
:10AFE0002091690730916A07400F511F621F731F3C
:10AFF000FE010995E0916107F0916207309741F0F9
:10B0000080916007811103C08091590781110995D2
:10B01000809159071092590781110E941B4ADF91B4
:10B02000CF911F910F9108956FEA7CE188EC9CE12C
:10B0300064CF6CE27DE181E894E45FCF6AE37DE177
:10B040008DE59EE15ACF6EE47DE182E69DE155CF2C
:10B050006BE97DE18DE994E450CFE091DD03E630CA
:10B0600028F581E08E0F8093DD03409174075091A5
:10B070007507609176077091770720916F0790911F
:10B08000700780919A0239E0E39FF0011124E9559D
:10B09000FC4FA0919013B0919113B183A083428390
:10B0A0005383648375832683978380870895A7E0FD
:10B0B000B0E0EDE5F8E50C940CEE0E9476C9F09056
:10B0C0006F072F2C85E08F0D8D833324339483E01D
:10B0D000E82E98EE892E93E0992EA12CB12C84E0D5
:10B0E0008F198E839E2D9F199F8382E0D82EDF18A3
:10B0F000C32CCF18F1102CC0809172078823C1F0A7
:10B1000080916A01882361F0622D619581E09091C0
:10B110007207911180E024E045E553E00E94C2C827
:10B12000F3949D81F912E6CF85E0809370070CC0FF
:10B130008091590710925907882311F30E941B4AE6
:10B14000809171078823E1F22796E2E10C9428EEC2
:10B1500081E0F8122DC0909172079130B9F0809182
:10B160006A018823E9F281E0913009F080E0909152
:10B170009C032DE133E0911102C029E133E001E0AD
:10B1800040E253E06C2D0E94E072CACF80915907D3
:10B1900010925907882319F380919C038F2580937F
:10B1A0009C03E0926A01809171078823C1F2CCCFA1
:10B1B00092E0F912D1C080917207823021F1809122
:10B1C0006A01882309F4ACCF11E0809172078230C4
:10B1D00009F010E06091060170910701072E000C44
:10B1E000880B990B0E942CE769837A838B839C835D
:10B1F000CE0101960E94944400E09C0142E153E09C
:10B200006D2D812FC0CF8091590710925907882347
:10B21000B1F210E000E025EF30E050E040E066E001
:10B2200071E082E193E00E943BCA8091710788231C
:10B2300031F28ACF80917207833019F180916A01CF
:10B24000882309F46DCF11E080917207833009F0F3
:10B2500010E06091040170910501072E000C880B2D
:10B26000990B0E942CE769837A838B839C83CE01A0
:10B2700001960E94944400E09C014BE053E06F81F2
:10B28000C0CF80915907109259078823B9F210E076
:10B2900000E025EF30E050E040E064E071E08BE05A
:10B2A00093E00E943BCA80917107882339F24CCF0A
:10B2B0008091590710925907882309F459C020E05A
:10B2C00030E048EC52E460910001709101018091FE
:10B2D0000201909103010E948BE70E9428EF2B014D
:10B2E00030927107BADEE0926A0183E093E09093B6
:10B2F0006E0780936D0780E091E090936C078093D8
:10B300006B071092670710926807109269071092F6
:10B310006A078092630790926407A0926507B092D3
:10B320006607712C612C40927407509275076092E9
:10B3300076077092770783E298E590939113809354
:10B34000901310926207109261071092600780912B
:10B350007107882369F0F8CE83E0F81609F46ACF04
:10B3600094E0F912DDCE80917207843009F4A0CF09
:10B3700080916A01882309F4D3CE11E0809172078D
:10B38000843009F010E0409000015090010160907D
:10B3900002017090030120E030E0A901C301B20175
:10B3A0000E9426E72DEB37E346E055EB87FD04C00E
:10B3B0002DEB37E346E055E3C301B2010E9444EEB2
:10B3C00069837A838B839C83CE0101960E94391B0B
:10B3D00000E09C0143E053E06E8113CFB0E0A0E0B9
:10B3E000E4EFF9E50C941CEE8D8190919F10891784
:10B3F00078F080939F109E01285F3F4F4E815F81C0
:10B4000064E570E08AE490E10E94EEE61092491053
:10B41000E2E00C9438EE0F931F93CF93DF936F3FCE
:10B4200011F410929F1020919F1021111EC08C01C9
:10B430000E9475E6800F911FEC01C01BD10BC53532
:10B44000D1053CF00197FC012491207C2038D1F3F8
:10B45000F3CFDD27AE01B8018AE490E10E9496E6C1
:10B46000C65BDF4E188210924910DF91CF911F9179
:10B470000F910895A6E8B0E0E0E4FAE50C9417EE29
:10B48000C358DF4F188219821A821B82CD57D040D1
:10B4900080918E0290918F02A0919002B0919102C2
:10B4A000CF57DF4F88839983AA83BB83C158D0408D
:10B4B00084E690E09093A9128093A8121092CD1286
:10B4C0001092CC1210921A0464E070E0CE018F57F3
:10B4D0009F4F0E949ECD8091A8129091A912029632
:10B4E0009093A9128093A8121092CD121092CC12B0
:10B4F00081E0CA57DF4F8883C658D040CE018A57B3
:10B500009F4F0E94CD2168E470E084E79DE00E9497
:10B510009ECD80E1E1E9F1E08E010F5F1F4FD80180
:10B5200001900D928A95E1F760E170E0C8010E94F8
:10B530009ECD86E997E00E94D5218CE0F80111921A
:10B540008A95E9F7C8010E94D1217E01FDE6EF0E40
:10B55000F11C8FEFF7018083C7010E94CD21198272
:10B560001A821B821C82C8010E94D5218091B402DC
:10B570009091B502A091B602B091B70289839A83E7
:10B58000AB83BC83C8010E94D521C358DF4F18820A
:10B5900019821A821B82CD57D04083E0F701808345
:10B5A0008983CE0183589F4F0E94D521C7010E94F5
:10B5B000CD21C8010E94CD212AE0D22EDA94DD20CF
:10B5C00031F0CE0183589F4F0E94D521F7CF89E5F6
:10B5D00093E10E94D121C358DF4F188219821A8249
:10B5E0001B82CD57D0409AE0D92EDA94DD2031F07D
:10B5F000CE0183589F4F0E94D521F7CF87E08983E2
:10B60000F7018083C8010E94CD21C7010E94CD218E
:10B6100068E070E084E893E00E949ECD68E070E00E
:10B620008CE793E00E949ECD64EC70E088EB92E0A2
:10B630000E949ECD1982DD24DA94F701D082C801E0
:10B640000E94F4CDC7010E94CD2164E070E08AEE33
:10B6500096E00E949ECD1982C8010E94F4CD6CE054
:10B6600070E08DE497E00E949ECD198A1A8A1B8AA9
:10B670001C8A80E090E0A0E8BFE38D879E87AF87BB
:10B68000B88B8091C0129091C112A091C212B0915A
:10B69000C31289839A83AB83BC8320E030E543ECFB
:10B6A00050E46091C4127091C5128091C6129091BD
:10B6B000C7120E948BE76D837E838F8398872CEA65
:10B6C00035EC47E25EE36091C8127091C912809137
:10B6D000CA129091CB120E948BE769877A878B8779
:10B6E0009C8764E170E0C8010E949ECD84E190E0F7
:10B6F0009A83898362E070E0C8010E949ECD8091A8
:10B70000410790914207A0914307B0914407898374
:10B710009A83AB83BC8320E030E543EC50E4609136
:10B7200045077091460780914707909148070E940E
:10B730008BE76D837E838F8398872CEA35EC47E215
:10B740005EE36091490770914A0780914B079091A1
:10B750004C070E948BE769877A878B879C87C80193
:10B760000E94C9218CE0E1EAF1E0D80101900D923C
:10B770008A95E1F7C8010E94C9211982C8010E9477
:10B78000CD218FE78983C8010E94CD21D982C801CC
:10B790000E94CD2185E0EDEAF1E0D80101900D9203
:10B7A0008A95E1F765E070E0C8010E949ECD19829C
:10B7B000C8010E94F4CD80E2E2EBF1E0D8010190F3
:10B7C0000D928A95E1F760E270E0C8010E949ECD7B
:10B7D000F7011082C7010E94F4CD1982C8010E94AE
:10B7E000F4CD80E090E0A0EEBFE3C358DF4F888344
:10B7F0009983AA83BB83CD57D040CE0183589F4FF6
:10B800000E94D521C358DF4F188219821A821B82E9
:10B81000CD57D040CE0183589F4F0E94D52182E161
:10B82000F80111928A95E9F762E170E0C8010E947F
:10B830009ECD84E2E2EDF1E0D80101900D928A956F
:10B84000E1F764E270E0C8010E949ECD80E1F8015A
:10B8500011928A95E9F760E170E0C8010E949ECDDF
:10B8600089E0F80111928A95E9F769E070E0C80172
:10B870000E949ECDC358DF4F188219821A821B8204
:10B88000CD57D040CE0183589F4F0E94D5218CE0E8
:10B89000D82EF8018D2D11928A95E9F76CE070E0B1
:10B8A000C8010E949ECD8CE6F80111928A95E9F7B5
:10B8B0006CE670E0C8010E949ECD8EE094E00E948C
:10B8C000C921F7011082118212821382148215821B
:10B8D0001682178268E070E0C7010E949ECDF701D2
:10B8E0001192DA94E9F7CB57DF4F1882C558D04050
:10B8F00080E090E0A0E4B0E4ED968CAF9DAFAEAFF9
:10B90000BFAFED97C7010E94D121CE018B579F4F4A
:10B910000E94CD21CE0187589F4F0E94D521809152
:10B920001A04811127C00091A8121091A9128091C8
:10B93000CC129091CD12F7019183808384E690E040
:10B940009093A9128093A81264E070E082E292E0E2
:10B950000E949ECD62E070E0C7010E949ECD91E002
:10B960000037F3E01F0709F490E080911A04892B57
:10B9700080931A0480911A04811104C060E081E070
:10B980009AE049DD90911A0481E08927CA57DF4F78
:10B99000E7E00C9433EE6EDD0C943845A7E0B0E0A0
:10B9A000E4EDFCE50C940CEE8091820787708983AE
:10B9B0008090840390908503A0908603B0908703C5
:10B9C0000E9476C920916F072E833981373009F0A4
:10B9D00075C085E194E09B838A831E81312F3B5F94
:10B9E0003C8333243394812F81958D83232C211A1A
:10B9F00084E6482E512C612C712C2E81222309F4CF
:10BA000062C03981373009F433C22E81213009F008
:10BA100028C290917207913009F445C180916A0162
:10BA2000811154C182E0F82E81E08F0D8F839981BE
:10BA3000973009F063C020E030E0A901C501B401EE
:10BA40000E9426E7882309F459C03F818E8138136C
:10BA500031C09091B3029F83809172072E8182132F
:10BA600011C08091590710925907882359F09325E6
:10BA70009F8383E080936A010E94D921809171079E
:10BA800081110DC180916A018823A1F06E81611B33
:10BA900081E0909172073E81931380E09F8126EFB1
:10BAA00033E0911102C022EF33E001E049EF53E0AF
:10BAB0000E94E072F394F394FF8220C020E134E00E
:10BAC0003B832A838ACF80917207882309F4D9C0E7
:10BAD00080916A01882309F494CF81E090917207E4
:10BAE000911180E024E043E254E06D810E94C2C8DD
:10BAF0008981873009F41DC193E09F838091B4024E
:10BB00009091B502A091B602B091B702809332072E
:10BB100090933307A0933407B09335072F813E816C
:10BB200023131EC080917207821709F407C1809108
:10BB30006A018823A9F0EE80E11AFF24F394809132
:10BB400072073E818313F12C82E397E00E94444404
:10BB500000E09C0146EE53E06E2D8F2D0E94E072B6
:10BB60008F818F5F9E81891316C08091720789171C
:10BB700009F438C180916A01882369F06E81611BE4
:10BB800081E0909172072E81921380E023E047EDCF
:10BB900053E00E94C2C88F818E5F3E81831316C01E
:10BBA00080917207831709F42EC180916A0188235E
:10BBB00069F06E81611B81E0909172072E81921372
:10BBC00080E023E04AEC53E00E94C2C88F818D5F81
:10BBD0003E81831323C080917207831709F424C127
:10BBE00080916A018823D1F089E19AE49F938F9331
:10BBF0008CEB93E09F938F938E81811B8F9381E0D9
:10BC0000909172073E81931380E08F930E945E2291
:10BC10000F900F900F900F900F900F908F818C5F6F
:10BC20009E81891323C080917207891709F40BC183
:10BC300080916A018823D1F08BEC9CE59F938F93D0
:10BC40008DEA93E09F938F938E81811B8F9381E088
:10BC5000909172072E81921380E08F930E945E2252
:10BC60000F900F900F900F900F900F903E813F5FBD
:10BC70003E838C818313C1CE9F819B5F909370071D
:10BC80000EC08091590710925907882309F420CFDC
:10BC90000E941B4A80917107882309F419CF2796C7
:10BCA000E2E10C9428EE80915907109259078823FD
:10BCB00009F4B4CE26EB35E03093F0062093EF067E
:10BCC00080917107882309F4A9CEE9CF81E09130F2
:10BCD00009F080E020E249E154E0622D0E94C2C8F0
:10BCE000A1CE909172073E81931731F080916A0145
:10BCF000811113C08E8197CE8091590710925907F8
:10BD00008823A1F32A813B813093F0062093EF062C
:10BD100080917107882351F3C2CF6E81611B81E04E
:10BD20003E81931380E020E246E054E00E94C2C8C6
:10BD3000E1CF22E02F83FF24F3947DCE8091590739
:10BD400010925907882309F4F2CE0E946AC96091C3
:10BD500032077091330780913407909135070E9424
:10BD600028EF6B013092710778D983E080936A01E4
:10BD700086EE93E090936E0780936D0722E337E0A1
:10BD800030936C0720936B07109267071092680737
:10BD90001092690710926A074092630750926407F5
:10BDA0006092650770926607F12CE12CC0927407CF
:10BDB000D0927507E0927607F092770789E198E5CF
:10BDC00090939113809390132FED31E2309362079B
:10BDD000209361071092600780917107882309F40E
:10BDE000A6CE5DCF8091590710925907882309F498
:10BDF000C1CE8EEC95E50E94CCC980917107882355
:10BE000009F4B8CE4CCF8091590710925907882376
:10BE100009F4CBCE8AE496E40E94CCC980917107E4
:10BE2000882309F4C2CE3BCF80915907109259075D
:10BE3000882309F4D5CE0E94194A8091710788237E
:10BE400009F4CECE2CCF8091590710925907882340
:10BE500009F4EECEA0DD80917107882309F4E8CEC5
:10BE60001ECF2E81223009F43CCF33E03F8346CEF3
:10BE70008E81813009F435CF92E09F835CCFB0E0B2
:10BE8000A0E0E5E4FFE50C940FEE0E94A322D82F7A
:10BE90000E9476C9C0916F075C2E85E0682E6C0EFB
:10BEA00099E1E92E9AE4F92E2BE3C22E24E0D22E5A
:10BEB00014E01C1B39E4A32E35E4B32E05E00C1B63
:10BEC00083E0982E9C1A82E0882E8C1A81E0782ECE
:10BED0007C1AC11141C080917207882361F1809161
:10BEE0006A01882361F0652D619581E09091720768
:10BEF000911180E024E049E754E00E94C2C8D111CA
:10BF0000EDC0C43009F0A0C080917207843009F4FC
:10BF10007FC080916A01882309F4B6C0FF92EF9236
:10BF2000DF92CF921F9381E090917207943009F4D1
:10BF3000A2C080E0A0C080915907109259078823C1
:10BF400071F20E941B4A80917107882341F2CDB79C
:10BF5000DEB7EFE00C942BEEC13031F58091720723
:10BF6000813099F080916A01882361F081E090919D
:10BF70007207913009F080E023E047E654E0672D36
:10BF80000E94C2C8D111AAC07FC0809159071092E7
:10BF90005907882339F383E892E50E94CCC9809140
:10BFA00071078823F9F2D3CFC23009F06FC08091B6
:10BFB0007207823081F080916A01882309F48BC076
:10BFC00081E090917207923009F080E023E048E52B
:10BFD00054E0682DD5CF80915907109259078823D6
:10BFE00051F38EEC95E50E94CCC9809171078823AE
:10BFF00011F3ADCF8091590710925907882309F4A6
:10C000004DC0C9DC80917107882309F447C09FCFD8
:10C010008091590710925907882309F47ACF0E941A
:10C02000194A80917107882309F473CF90CF8091CA
:10C03000590710925907882369F00E944945809159
:10C040007107882339F083CFC530F1F480917207EE
:10C05000853069F380916A018823B1F0BF92AF9275
:10C060008AE294E09F938F930F9381E090917207FF
:10C07000953009F05ECF8F930E945E220F900F9053
:10C080000F900F900F900F9086E029C0C33009F0F9
:10C0900036CF80917207833009F4ACCF80916A016A
:10C0A0008823C9F08BEC9CE59F938F9389E494E0FF
:10C0B0009F938F939F9281E090917207933009F044
:10C0C00080E08F930E945E220F900F900F900F9050
:10C0D0000F900F9057CFDD2309F4B6CF84E0CF5FE8
:10C0E0006C12F7CE8093700732CF0E94CC3FC2D93A
:10C0F0000E9438450C948846CF9380919F0381110C
:10C1000009C08CED91E09093E3038093E20381E01A
:10C1100080939F030E942D5820E040E070E060E093
:10C120008EEA92E20E944C45C1E0C0939A020E94BE
:10C13000DB2B0E941B4AC0939A0260E08BED9CE2CD
:10C140006AD988ED91E09093F0068093EF06CF9145
:10C150000895A6E0B0E0EFEAF0E60C940CEE0E9441
:10C160001779382E8091E81484FB662460F8412CFE
:10C1700084FF03C00E942A79482E0E9476C920912C
:10C180006F072D83522E2B5F298380E00FED14E083
:10C1900091E0792E7518952D91959A839CE7E92E5B
:10C1A00090E6F92E2CEFC22E24E0D22E92E09519C3
:10C1B0009B8393E095199C833BE9832E34E0932E77
:10C1C00040EBA42E44E0B42E9D812981921709F4FE
:10C1D00009C2992349F131106AC00E946D7F8823FA
:10C1E00009F47AC19D81913009F444C122E02E8383
:10C1F0002D818E8128135FC180917207281709F461
:10C200006EC180916A01882309F455C16D81651959
:10C2100081E0909172072D81921380E023E048ED38
:10C2200054E00E94C2C847C180917207882379F107
:10C2300080916A01882379F281E0909172079111CF
:10C2400080E024E048E055E06A810E94C2C83320C3
:10C2500021F224E02E839D812E8192134AC0809189
:10C260007207981709F44CC180916A01882309F478
:10C2700040C06D81651981E0909172072D81921304
:10C2800080E023E04CEC54E00E94C2C832C08091B0
:10C29000590710925907882359F20E941B4A80912E
:10C2A0007107882329F22696E2E10C9428EE8D810D
:10C2B000813009F47FC0823009F4A6C09D8193309B
:10C2C00041F680917207833009F4C3C080916A01FE
:10C2D000882309F4BECF81E090917207933009F072
:10C2E00080E023E04CEE54E06C810E94C2C884E000
:10C2F0008E838E818F5F9D81981316C08091720707
:10C30000981709F40EC180916A01882369F06D8144
:10C31000651981E0909172072D81921380E023E0EE
:10C320004EEB54E00E94C2C88E818E5F662009F4F5
:10C3300030C141103BC09D8198131BC020907207F3
:10C34000921509F4FFC080916A01882391F01F9231
:10C35000BF92AF928D8185198F9381E02D8122113B
:10C3600080E08F930E945E220F900F900F900F90AD
:10C370000F908E818D5F9D81981316C080917207FA
:10C38000981709F4F5C080916A01882369F06D81DE
:10C39000651981E0909172072D81921380E023E06E
:10C3A0004FE954E00E94C2C88E818C5F9D819F5FDF
:10C3B0009D830ACF809172078130D1F080916A010C
:10C3C000882309F446CFFF92EF92DF92CF927F92BB
:10C3D00081E090917207913009F080E08F930E9484
:10C3E0005E220F900F900F900F900F900F9031CF13
:10C3F0008091590710925907882301F37DDE8091BF
:10C4000071078823D9F24FCF80917207823091F063
:10C4100080916A01882309F41CCF81E09091720712
:10C42000923009F080E023E041EF54E06B810E94FC
:10C43000C2C80FCF8091590710925907882341F342
:10C4400082E595E50E94CCC980917107882301F3AC
:10C450002ACF8091590710925907882309F436CFC3
:10C4600089E39AE40E94CCC980917107882309F47A
:10C470002DCF19CF80917207813009F180916A0127
:10C48000882309F4B3CE8EE393E49F938F931F9395
:10C490000F937F9281E090917207913009F080E0D4
:10C4A0008F930E945E220F900F900F900F900F902D
:10C4B0000F9082E08E838E818F5F8E83CCCE8091B1
:10C4C0005907109259078823C9F20E943E43809170
:10C4D0007107882399F2E7CE91E09E8389CE8091FF
:10C4E000590710925907882309F48BCE86EA9EE4F7
:10C4F0000E94CCC980917107882309F482CED3CEE3
:10C500008091590710925907882309F4ADCE82E033
:10C510009CE40E94CCC980917107882309F4A4CEC1
:10C52000C2CE8091590710925907882309F4EBCEA7
:10C530008FE39FE50E94CCC980917107882309F49D
:10C54000E2CEB1CE8091590710925907882309F4A1
:10C55000FACE4FE350E06AE874E081EF96E00E9483
:10C560007DF080917107882309F4EDCE8D811ECF77
:10C570008091590710925907882309F404CF83E664
:10C5800094E60E94CCC980917107882309F4FBCE00
:10C59000EDCF9D81981314C0909172072D812917BA
:10C5A00091F080916A01882359F06D81651981E0CD
:10C5B0002D81291380E020E24EE854E00E94C2C899
:10C5C0008E818D5FF3CE8091590710925907882391
:10C5D00041F39092F0068092EF06809171078823D4
:10C5E00001F3C4CF809370075ECE10929802109230
:10C5F00069010E942A799091E81480FB97F9909341
:10C60000E81460E08AEC91E00E940B5A0C94884692
:10C610000F931F930E94F7CD009194021091950201
:10C620002091960230919702601B710B820B930B45
:10C6300097FD0CC089B183FB882780F991E0892799
:10C640004A9B8260309B8460809393028091930226
:10C6500081709091930291FD826090919E03981752
:10C6600049F0813009F148F0823079F0833091F05F
:10C6700080939E031F910F910895913079F092302D
:10C68000B9F79091920291500CC0992339F09330F0
:10C69000C1F3EECF9130A9F3923051F7909192020D
:10C6A0009F5F90939202E4CF992359F3933001F75F
:10C6B000F5CF1F93CF93DF93809135018F3708F427
:10C6C00075C08F579091BF1290939E04992309F4DF
:10C6D0006BC05D9A9091400790939D04992309F453
:10C6E0006FC05C9A8F5F8093350180919C0491E0CC
:10C6F000892780939C0481118BDF8091340191E024
:10C70000980F85300CF090E0823009F4A8C00CF04E
:10C7100059C0882309F46EC0813009F495C0909304
:10C720003401C0918307D0918407209709F42DC06C
:10C73000F89413B1147082E00E945A2B00C000C01C
:10C740001C161D060CF0B9C02A9A00C000C02B9A16
:10C7500000C0000082E090E00197F0F72B9800C045
:10C7600000C0112309F4ABC02A9A00C000C078941D
:10C7700080918307909184071C161D060CF0A1C0C0
:10C78000019790938407809383078091BC0D9091CB
:10C79000BD0D009729F001979093BD0D8093BC0DBE
:10C7A000DF91CF911F9108955D9894CF90919E0451
:10C7B000891708F05D9890919D04891708F492CF2D
:10C7C0005C9890CF843009F461C00CF45BC0853074
:10C7D00009F0A5CF20919B04211102C080939B04F6
:10C7E00080919B04815080939B04882309F497CF08
:10C7F00095E095CF809133018F5F80311CF4809359
:10C8000033018DCF1092330180919D03811113C0AC
:10C810002091B5123091B6123093B8122093B7120E
:10C820002091360730913707309339072093380726
:10C8300081E080939D031092B6121092B51210926F
:10C840003707109236076BCF10927B0087E48093F6
:10C850007C0080917A00806480937A0060CF809120
:10C860007A0086FD26C04091780050917900209191
:10C87000B5123091B612240F351F3093B6122093A3
:10C88000B5124DCF10927B0086E4E1CF80917A0003
:10C8900086FD11C0409178005091790020913607B3
:10C8A00030913707240F351F309337072093360711
:10C8B00036CF92E034CF94E032CF2A9846CF2A98F0
:10C8C00054CF01965ECFACE3B0E0E9E6F4E60C9419
:10C8D0000CEE80917307882369F18091E81410E0D1
:10C8E00000E084FF23C089EE92E10E94EA238BE1FD
:10C8F000E9EEF2E1DE01919601900D928A95E1F761
:10C9000010E000E0BE016F5F7F4FCE0181960E9474
:10C91000A3D718163CF4CE0101960E9416D2080F38
:10C92000111DF0CFCE0181960E94BA251093ED0320
:10C930000093EC030E9476C910916F07312E85E0B9
:10C94000810F8CAF212E21948DEEA82E8CE1B82E74
:10C9500091E5892E95E0992E01E0011B26E5622ED6
:10C9600025E0722E111113C080917207882391F176
:10C9700080916A01882359F081E0909172079111AA
:10C9800080E024E04FE555E0622D0E94C2C880910E
:10C99000E81486FF3EC01130D9F4809172078130CF
:10C9A00049F180916A01882309F43EC11F927F9268
:10C9B0006F920F9381E090917207913009F080E0BF
:10C9C0008F930E945E220F900F900F900F900F9008
:10C9D00082E04FC08091590710925907882341F295
:10C9E0000E941B4A80917107882311F2EC96E2E1C4
:10C9F0000C9428EE8091590710925907882389F2E8
:10CA000010926F070E94FCDA80917107882349F227
:10CA1000EDCF84FF2DC01130D9F68091720781309F
:10CA2000D1F080916A01882309F4FEC0BF92AF92D1
:10CA30009F928F920F9381E090917207913009F04D
:10CA400080E08F930E945E220F900F900F900F90C6
:10CA50000F900F90BDCF80915907109259078823EE
:10CA600001F30E94ED1C809171078823D1F2BECFA3
:10CA700081E090916A01992309F4D7C0582ED12CF6
:10CA8000C12C412E4318852DE090EC03F090ED036E
:10CA9000CE14DF0408F0C9C05112A5C091E0E91A14
:10CAA000F108EC18FD0889EE92E10E94EA238BE17F
:10CAB000E9EEF2E1DE01919601900D928A95E1F79F
:10CAC000F12CBE016F5F7F4FCE0181960E94A3D7EC
:10CAD00018167CF4CE0101960E9416D2882389F3A1
:10CAE000EF106BC0BE016F5F7F4F85E897E00E943B
:10CAF00031D2CE0181960E94BA258091E81490919E
:10CB0000720785FF75C0911363C080915907109219
:10CB10005907882309F45CC019821C828091EC12A9
:10CB200064E073E1882311F069EE72E121E045E8E9
:10CB300057E0CE0101960E94BF25882309F43FC02B
:10CB40008BE1FE013196A9EEB2E101900D928A953A
:10CB5000E1F78091E8148F7B8093E814A091DE14B4
:10CB6000AA3080F481E08A0F8093DE148BE18A9FE3
:10CB7000D0011124A053BC4EE9EEF2E101900D92D8
:10CB80008A95E1F7CE0101960E94BA2510926F07AF
:10CB900082E090E0A0E0B0E0809374079093750786
:10CBA000A0937607B093770781E080937107109286
:10CBB000990283E080936A0119CFF39482CF0E9497
:10CBC000B88765E877E08BE395E00E94F1D1DACF92
:10CBD00080916A01882339F081E0911380E041E07F
:10CBE000642D0E9400C98FEFC81AD80A53944BCF06
:10CBF000911759F080916A018823A9F381E09091FF
:10CC00007207911380E040E0EBCF809159071092BA
:10CC10005907882379F38EE095E50E94CCC980916D
:10CC20007107882339F3E2CE82E01F5F9CAD911338
:10CC300099CE80937007DACEFC01A081B1811C925D
:10CC4000A281B3818C918F5F8C930280F381E02D60
:10CC500090818CE0989F800D1124E2E9F3E113AEFE
:10CC600084AF0895FC0184910895FC0180810895AA
:10CC7000009751F0FC0180E09191992331F0907C74
:10CC80009038D1F38F5FF8CF80E00895119800C0FD
:10CC900087FD43C0419800C0119A00C000C01198A0
:10CCA00000C086FD46C0419800C0119A00C000C077
:10CCB000119800C085FD3BC0419800C0119A00C08A
:10CCC00000C0119800C084FD30C0419800C0119A86
:10CCD00000C000C0119800C083FD25C0419800C06D
:10CCE000119A00C000C0119800C082FD1AC041987E
:10CCF00000C0119A00C000C0119800C081FD0FC093
:10CD0000419800C0119A00C000C0119800C041981D
:10CD100000C0119A00C000C00895419ABCCF419A4A
:10CD2000F0CF419AE5CF419ADACF419ACFCF419ADD
:10CD3000C4CF419AB9CF90E080E00895CF93DF93BC
:10CD4000DB01F9019C919130C1F0943080F0945056
:10CD50009C938830D1F480819181009771F0019784
:10CD600091838083480F591FEA01188206C08C35D1
:10CD700039F49C5F9C93943041F4DF91CF910895F6
:10CD80008B3339F781E08C93F8CF20813181B90161
:10CD90006F5F7F4F71836083420F531FEA01888367
:10CDA000808191818F3591056CF7E7CF0F931F93A9
:10CDB00081E00091E4141091E5142091E614309183
:10CDC000E7144091E0145091E1146091E2147091E5
:10CDD000E314041715072607370708F480E01F91AE
:10CDE0000F91089590E080E008952091020683302D
:10CDF00021F425FD0CC024FD0CC030E0A90102C0C7
:10CE0000559547958A95E2F7CA018170089581E0AA
:10CE1000089580E0089580911E0684FD0BC08091E6
:10CE2000200687FD07C090912106937081E019F4D8
:10CE300080E0089581E008952FEB280F2A3108F053
:10CE400047C0E22FF0E080911E0690911F06A0914E
:10CE50002006B091210604C0B695A79597958795B1
:10CE60002A95D2F780FD02C081700895EC5FF94FDA
:10CE7000E081EE2341F18091940790919507E80FAE
:10CE8000F92FF11D808190ED980F9A3030F08E329D
:10CE900051F4818180538A3098F4F093F305E09344
:10CEA000F20581E008958D3211F08B3249F48181D1
:10CEB00090ED980F9A3088F38E3211F48281EACF88
:10CEC000F0E0E0E0EACF1092F3051092F205E9CF2E
:10CED00080E00895CF93DF9385E4AEDF882309F1E6
:10CEE00088E040911E0650911F06609120067091C7
:10CEF0002106972F9170C92F90E0D92FCC0FDD1FFD
:10CF000071FB222720F930E0220F331F220F331F3D
:10CF1000C22B67FB442740F9C42B8C2BDF91CF91A8
:10CF2000089580E0DECF88DF882341F081E0209102
:10CF3000F2053091F305232B09F480E00895CF9397
:10CF4000DF93C0913E07D0913F07209729F1609170
:10CF50003A0770913B0780913C0790913D070E94F2
:10CF600023EF6E5F7F4F24976C177D07ACF47093AF
:10CF70009703609396030E94F7CD605A75418F4FD7
:10CF80009F4F609398037093990380939A039093B3
:10CF90009B03DF91CF91089510929803109299030B
:10CFA00010929A0310929B03F4CFB0E0A0E0EBED57
:10CFB000F7E60C9415EE6B01E9014A3009F4D5C08F
:10CFC000453109F081C0DB011296ED91FC91F280B0
:10CFD00096818781139A00C00000E6E2F0E0319765
:10CFE000F0F7092F182FEF2CE29420EFE22230E126
:10CFF000B32EBF0CE80188EF49DE00C0000086E2D6
:10D0000090E00197F0F7BFE1BF1508F49BC08F2DAA
:10D01000807780683BDE8E2D39DE00C0000086E21E
:10D0200090E00197F0F780E831DE80E02FDE00C06D
:10D03000000086E290E00197F0F78AEF27DE00C05B
:10D04000000086E290E00197F0F7005F1F4F8881B3
:10D05000807F1CDE89918295807F18DEC017D10702
:10D06000B1F700C0000086E290E00197F0F7F3947A
:10D07000E0E1EE0EFB10BECF1398D6011296ED91B3
:10D08000FC9180819281980F92832181921708F000
:10D090009FC194819F5F94839381890F821710F0C1
:10D0A0008FEF820F8383458150E0440F551F70E05E
:10D0B00060E0868197810E9443F081E0CDB7DEB7C2
:10D0C000E9E00C9431EEDEC1FB01028113814233B1
:10D0D00009F485C108F48DC1463409F475C147349B
:10D0E00009F482C14B3349F789812B81D80112960B
:10D0F0007C91129713963C91213009F4BFC12330E3
:10D1000009F0A0C148EF480F582F91E0341708F4F8
:10D1100090E031E0541708F030E0492F432B61E0F4
:10D12000571708F460E0462311F4932331F2FA8094
:10D1300030E0F901E25CFD4FD080265C3D4FF90103
:10D14000E08099C180EE8F0D8068807F9FDD8F2DFC
:10D150008295807F9BDD00C0000086E290E0019711
:10D16000F0F780E893DD80E861CF0B9A1398399A45
:10D170004198099A119A139A00C0000086E290E043
:10D180000197F0F788E790E0CEE9DFE0FE01319704
:10D19000F1F70197D9F788EF79DD00C0000086E24A
:10D1A00090E00197F0F780E271DD80E06FDD00C074
:10D1B000000086E290E00197F0F780E067DD80E80C
:10D1C00065DD00C0000086E290E00197F0F780E0A6
:10D1D0005DDD80E15BDD00C0000086E290E001974C
:10D1E000F0F7CE010197F1F7CE010197F1F7CE01EB
:10D1F0000197F1F7CE010197F1F7CE010197F1F711
:10D20000CE010197F1F7CE010197F1F7CE01019719
:10D21000F1F7CE010197F1F7CE010197F1F7CE01B9
:10D220000197F1F7CE010197F1F7CE010197F1F7E0
:10D23000CE010197F1F72197F1F780E227DD80E435
:10D2400025DD00C0000086E290E00197F0F780E263
:10D250001DDD80E61BDD00C0000086E290E0019746
:10D26000F0F7D0E0C0E08C2F807780680FDD8D2F45
:10D270000DDD00C0000086E290E00197F0F780E845
:10D2800005DD80E003DD00C0000086E290E001974C
:10D29000F0F78AEFFBDC00C0000086E290E0019727
:10D2A000F0F780E2119800C0419800C0119A00C0C8
:10D2B00000C0119800C0419800C0119A00C000C081
:10D2C000119800C0419800C0119A00C000C0119888
:10D2D00000C0419800C0119A00C000C0119800C061
:10D2E000419800C0119A00C000C0119800C0419838
:10D2F00000C0119A00C000C0119800C0419800C041
:10D30000119A00C000C0119800C0419800C0119A45
:10D3100000C000C0119800C0419800C0119A00C020
:10D3200000C0119800C0419800C0119A00C000C010
:10D33000119800C0419800C0119A00C000C0119817
:10D3400000C0419800C0119A00C000C0119800C0F0
:10D35000419800C0119A00C000C0119800C04198C7
:10D3600000C0119A00C000C0119800C0419800C0D0
:10D37000119A00C000C0119800C0419800C0119AD5
:10D3800000C000C000C00000E6E2F0E03197F0F716
:10D39000815009F087CF88EF79DC00C0000086E279
:10D3A00090E00197F0F7CF5FD05FC03209F05BCF1C
:10D3B00080E06CDC80EC6ADC00C0000086E290E07B
:10D3C0000197F0F7139879CEF8018581888375CE9F
:10D3D00080E0CDB7DEB7E9E00C9431EE53C0B9017F
:10D3E000C8010E94F5CE69CED80111968C91888330
:10D3F00064CE443191F0473109F05FCE1882D801F4
:10D4000012968C911297898315968C91159781505D
:10D410008A8313968C918B8350CED80115964C91AC
:10D42000159750E0440F551F70E060E016968D91FF
:10D430009C910E9443F0F801128280818150838385
:10D4400014823BCE381708F438CE871708F435CE4F
:10D45000FA80E12CD12C243070F46ACEBE01C801D0
:10D460000E94F5CE898198819D0D98838E0D8983C8
:10D47000FF0C09F422CEF7FEF6CFF0CF58E0580F9C
:10D48000482F43CEEF92FF920F931F93CF93DF93DA
:10D49000EC018B017A018A859B858617970731F00D
:10D4A000888199810E94E2D01B870A87B701888111
:10D4B00099810E9438C92E813F81820F932F911D3F
:10D4C0009F838E8390E080E0CDB7DEB7E6E00C94DA
:10D4D00034EEB0E0A0E0EFE6FAE60C9414EEEC01D6
:10D4E0007B018A018A859B858617970731F08881A1
:10D4F00099810E94E2D0FB86EA868885998501960B
:10D5000009F5CC80DA808E81D80EA880B980D5014B
:10D510005596ED91FC91C5010995C80E780110E072
:10D52000F70121917F0121111FC08E819F81810F01
:10D53000911D9F838E8390E080E0CDB7DEB7EAE057
:10D540000C9430EEEE80FF80B801888199810E94B2
:10D5500038C98E0D9F2D911D2885398528173907CB
:10D5600080F681E090E0E9CF4C2D6D2DC5010E9441
:10D570003AD1D80E180FD4CFB0E0A0E0E2ECFAE632
:10D580000C9417EEEC01D62E1CAD0BAD7C0184E0A3
:10D59000E80EF11CE98DFA8DC7010995412F480F5E
:10D5A0002D2D602FC7010E943AD19BAD890F8BAF03
:10D5B00081E090E0CDB7DEB7E7E00C9433EE682F62
:10D5C00070E090E080E00C9446B08091F20590917C
:10D5D000F305009731F04AE050E070E060E00C9411
:10D5E00047E560E070E0CB0108958091F2059091ED
:10D5F000F305009731F04AE050E070E060E00C94F1
:10D600001AE460E070E0CB010895EFDF97FD0AC0F7
:10D61000ECDF6F3F71058105910509F02CF4E5DF22
:10D62000862F089580E008958FEF0895CF93C62F39
:10D630007ADC882311F0E9DFC82F8C2FCF91089571
:10D640008091F2059091F305892B39F0DEDF91E0AE
:10D65000811101C090E0892F089591E0FCCFCF9314
:10D66000DF93C82FD62F5FDC882321F0E9DFDF911D
:10D67000CF9108958C2FE0DB8111F9CF8D2FF7CF5B
:10D68000B4DFCB010895CF93DF93EB014CDC88230B
:10D6900011F0F6DFEC01CE01DF91CF9108950F93E9
:10D6A0001F93CF938091F2059091F3050097D9F0E5
:10D6B000FC018F01C1912C2F2F7D81F0C53411F019
:10D6C000C536B9F7F801108270E060E00E94C4E24C
:10D6D000F801C083CF911F910F91089570E060E031
:10D6E0000E94C4E2F7CF60E070E0CB01F3CFCF92AD
:10D6F000DF92EF92FF926A017B0115DC882319F01B
:10D70000CEDF6B017C01C701B601FF90EF90DF9087
:10D71000CF900895CF92DF92EF92FF92CF93C82FD0
:10D720000E94F7CD6B017C0124EA30E74DE75FE30F
:10D73000609108017091090180910A0190910B019B
:10D740000E9426E787FD18C08AEF90E0A0E0B0E0D5
:10D750008C0D9D1DAE1DBF1D80935F0690936006CE
:10D76000A0936106B0936206C0935D01CF91FF90D4
:10D77000EF90DF90CF90089580E090E0DC01E8CF5B
:10D78000CF9380912E06811154C01092CD13109228
:10D79000CE131092CF1310929B1310929A131092E3
:10D7A0009D1310929C1310929F1381E080939E13FF
:10D7B00082E28093A0131092A5131092A413E9EBB8
:10D7C000F3E127EC33E18FEF81932E173F07E1F769
:10D7D000C1E0C093B6132AE73EEA3093AC1320931E
:10D7E000AB13C093AD131092AE131092AF1390E42D
:10D7F0009093B0131092B11329E73EEA3093C81307
:10D800002093C71325E531E03093991320939813A3
:10D810009EE19093BD1391E19093BE139CE1909390
:10D82000BB138093BA138093B9130E9434CFC09373
:10D830002E0681E080932D0686E691E29093AC124D
:10D840008093AB121092AE121092AD1253985B9A65
:10D8500052985A9A3898409A0E94086310929202FD
:10D86000CF910895FC0180E0309749F0949199237D
:10D8700031F0907C903809F08F5F3196F7CF0895A2
:10D88000B0E0A0E0E6E4FCE60C9414EEEC015B01F1
:10D890008A01FB01099587FD10C0C82ED12CF12CFF
:10D8A000E12C2196F801C082D182E282F382CE017E
:10D8B000CDB7DEB7EAE00C9430EE982F907E903C26
:10D8C000A9F48F7190E0B0E0A0E06C017D0156E01A
:10D8D000CC0CDD1CEE1CFF1C5A95D1F7CE01019635
:10D8E000F50109958F73C82A2296DCCF982F907F77
:10D8F000903E11F58F7090E0B0E0A0E06C017D01EA
:10D9000036E0CC0CDD1CEE1CFF1C3A95D1F7CE01A5
:10D910000196F50109958F73C82A46E0CC0CDD1CF1
:10D92000EE1CFF1C4A95D1F7CE010296F501099530
:10D930008F73C82A2396B6CF982F987F903F79F59A
:10D94000877090E0B0E0A0E06C017D0186E0CC0C37
:10D95000DD1CEE1CFF1C8A95D1F7CE010196F50166
:10D9600009958F73C82A96E0CC0CDD1CEE1CFF1CB9
:10D970009A95D1F7CE010296F50109958F73C82AC1
:10D9800026E0CC0CDD1CEE1CFF1C2A95D1F7CE0145
:10D990000396F50109958F73C82A249683CF982F93
:10D9A000907C903841F4807C803869F42196CE01D7
:10D9B000F5010995F8CF8E7F8D3F28F02196CE0195
:10D9C000F5010995F8CFC12CD12C76016BCF9CE0E5
:10D9D000899F802D112491E0980F90932C062CE0C4
:10D9E000280F20937D0730E02E5F3F4F4091CA13F0
:10D9F0004217130619F014F080E008952091CC131B
:10DA00009217D0F7662341F08E5F0E9419D0809163
:10DA10007D078E5F0E9419D080917D079091CA1377
:10DA2000891750F32091CC1390912C06291720F3DD
:10DA30001092CD138093CE1381E0089520912B0690
:10DA4000022E000C330B8217130641F080932B0635
:10DA500061ED72E286E993E10C94E2D00895ACE0C6
:10DA6000B0E0E5E3FDE60C9416EE6F3F710581052D
:10DA7000910509F070F482E993E17EDDE0919A135B
:10DA8000F0919B133196849190E02C96E8E00C94F1
:10DA900032EEF090CD13E090CE1320912D0621119F
:10DAA0000FC048E351E26E2D8F2D0E9493D190E07C
:10DAB00080E0F80EF092CD13E092CE139927E5CFD7
:10DAC000C0909A13D0909B1326E933E13A832983BF
:10DAD0002F2D30E03C832B832E2D30E03E832D8391
:10DAE00018861F822FEF3FEF3A8729871C861B86F7
:10DAF00009E61AE69E012F5F3F4FAB01BC01C6014C
:10DB00000E9488AFB60186E993E10E94E2D08F813E
:10DB10009885CFCF4F925F926F927F928F929F9214
:10DB2000BF92CF92DF92EF92FF920F931F93CF930A
:10DB3000DF93CDB7DEB728970FB6F894DEBF0FBEE0
:10DB4000CDBF7C016A014901FB0190818CE0989F67
:10DB5000800D1124982FF7012081822F880F820FCA
:10DB6000880F8093CD139093CE134115510559F131
:10DB7000FA82E9827C836B8301111EC0AE014B5F88
:10DB80005F4FB401C6017CDE6C016D817E818F81A7
:10DB900098856115710581059105A9F060DFF70190
:10DBA00080818F5F8083853148F3CE01019644D810
:10DBB000E5CFB12C860129C08A01B12C26C04528A9
:10DBC00046284728B1F728960FB6F894DEBF0FBE57
:10DBD000CDBFDF91CF911F910F91FF90EF90DF901C
:10DBE000CF90BF909F908F907F906F905F904F905D
:10DBF0000895B39407C0B1102DC001151105C9F2E5
:10DC00000F5F1F4F01151105A9F2AE014B5F5F4F6A
:10DC1000B401C60135DE6C014D805E806F80788472
:10DC20004114510461047104A9F0F0E24F1651044B
:10DC30006104710401F3D301C2018D97A109B109F7
:10DC40000297A105B10530F04BE24416510461047E
:10DC5000710479F6F7018081482F4B0D5527551F28
:10DC60004631510534F0853020F0CE0101960E94F6
:10DC70001C6681E0411451046104710409F480E0E0
:10DC8000B80EF70180818B0D8083BB2009F497CFFC
:10DC9000BA94AE014B5F5F4FB401C801F1DD8C0156
:10DCA0006D817E818F819885DADEEFCFCF93DF9310
:10DCB000FC0125AD211104C021E025AF0E9434CF25
:10DCC000C0919813D0919913E091C713F091C813A4
:10DCD00082E00995E091C713F091C81381E009959E
:10DCE00030E020E044E1BE0186E993E10E942FCFBD
:10DCF00029EC33E147E1BE0186E993E10E942FCF91
:10DD0000E091C713F091C81380E00995DF91CF919E
:10DD100008954F925F926F927F928F929F92AF92EF
:10DD2000BF92CF92DF92EF92FF921F93CF93DF9338
:10DD300000D000D0CDB7DEB70E94F7CD6B017C01DB
:10DD400080915D018F3FC1F10E94F7CD80905F0609
:10DD500090906006A0906106B090620668197909FB
:10DD60008A099B0997FD28C080916A1390916B13D3
:10DD70008F5F8F70891701F1E0915D01E53008F048
:10DD800054C024E0E29FF0011124EE5BFD4F80813E
:10DD90009181A281B38189839A83AB83BC8320E084
:10DDA00030E0A901BE016F5F7F4F85E791E00E94DF
:10DDB000BCC38FEF80935D010E9408638091930242
:10DDC00082FF3CC080916E0681113AC091E0909331
:10DDD0006E068091980289278093590710929802C5
:10DDE00083E080936A01109293020E94F7CD6C50F9
:10DDF0007E4F8F4F9F4F6093940270939502809354
:10DE000096029093970268E873E182E090E00E94A6
:10DE10000C4516E01150A1F00E94B04462E070E0A1
:10DE200080E090E00E946BCDF5CF80916B019091E6
:10DE30006C01A0916D01B0916E01ADCF10926E0694
:10DE400080916A0690916B06A0916C06B0916D0668
:10DE5000A7019601281B390B4A0B5B0BDA01C9019C
:10DE6000B7FF05C080919902882309F4B9C1D70191
:10DE7000C6018C599F4FAF4FBF4F80936A06909356
:10DE80006B06A0936C06B0936D0660919202062E0D
:10DE9000000C770B77FF03C0719561957109909124
:10DEA000920280916906981365C0633008F062C0E1
:10DEB000109292028091920280936906643008F079
:10DEC00069C0809159078111E7C0809190139091AA
:10DED00091138853994741F480915E01882309F496
:10DEE000EDC0815080935E010E94AF2E8090AE07FE
:10DEF0009090AF07A090B007B090B10781110E9439
:10DF0000BC2ED501C4013AE0B695A79597958795A3
:10DF10003A95D1F7009741E0A407B10520F08FEFC3
:10DF20009FEFA0E0B0E09695879520916A012111BE
:10DF3000D7C030919902311180C180919013909196
:10DF400091138853994709F45FC180919A02811116
:10DF50005BC18091650690916606A0916706B091BD
:10DF60006806C81AD90AEA0AFB0AF7FC5BC10E94D4
:10DF7000884658C1633009F09DCF8091920287FD99
:10DF800007C081E0880F880F8093920264E092CFEF
:10DF90008FEFF8CF80917C0721E030E040E050E047
:10DFA000882309F456C08090780790907907A09054
:10DFB0007A07B0907B0781149104A104B104E9F1C0
:10DFC00070E090E080E00E942AE720E030E040E846
:10DFD0005EE30E948BE72B013C01C701B601681983
:10DFE00079098A099B090E942AE79B01AC01C301B8
:10DFF000B2010E94BBEE20E030E04AE754E40E9408
:10E000008BE74B015C0120E030E040EA52E40E94E3
:10E01000A7EF24E630E040E050E087FF12C020E0A8
:10E0200030E040EF51E4C501B4010E94A7EF2AE0BF
:10E0300030E040E050E087FF04C021E030E040E005
:10E0400050E0C0927807D0927907E0927A07F09278
:10E050007B07A09192020A2E000CBB0B0E949CED44
:10E0600024E030E040E050E00E9476ED80917407BB
:10E0700090917507A0917607B0917707820F931F53
:10E08000A41FB51F8093740790937507A09376071C
:10E09000B093770710929202D701C6018856954C2B
:10E0A000AF4FBF4F8093650690936606A0936706B7
:10E0B000B093680681E080936A0107CF8CE080937B
:10E0C0005E018091630690916406009729F00197A4
:10E0D000909364068093630681E080936A0104CF85
:10E0E000009741F040916306509164064817590724
:10E0F00008F023CF80919902811111C0223038F0AD
:10E10000243008F43FC0243011F410926A0182E9EF
:10E1100093E1CCDD81E0809373078093990283E0E3
:10E120008DDC81E08093B613E0919013F091911310
:10E1300009951092730780919902811127C010925E
:10E14000590780919013909191138853994709F042
:10E15000FCCE0E94F7CDDC01CB018C199D09AE09E4
:10E16000BF098090630690906406B12CA12C88169C
:10E170009906AA06BB0608F0E0CE90936406809349
:10E180006306DBCE81E080936A01C1CF86E993E12B
:10E190000E94B2D091E0811101C090E09093990269
:10E1A000882369F280919013909191138853994735
:10E1B000B9F40E94F7CDDC01CB018C199D09AE09A1
:10E1C000BF09C0906306D0906406F12CE12CC816FC
:10E1D000D906EA06FB0620F4909364068093630652
:10E1E0000F900F900F900F90DF91CF911F91FF90A4
:10E1F000EF90DF90CF90BF90AF909F908F907F90E7
:10E200006F905F904F90089548E9C40E4AE3D41E82
:10E21000E11CF11CC0926506D0926606E09267068A
:10E22000F0926806809199028111DACF80916A019B
:10E230008130B1F610926A01D3CF009709F46FCF05
:10E2400051CFACE0B0E0E7E2F1E70C9416EEF090CD
:10E25000CD13E090CE1320912D06211112C048E17C
:10E2600051E26E2D8F2D0E9493D190E080E0F80E48
:10E27000F092CD13E092CE1399272C96E8E00C94FF
:10E2800032EEC0909A13D0909B1326E933E13A8383
:10E2900029832F2D30E03C832B832E2D30E03E83CD
:10E2A0002D8318861F827A8769871C861B8609E65C
:10E2B0001AE69E012F5F3F4F42E356E6BC01C601BE
:10E2C0000E941DB0B60186E993E10E94E2D08F81E1
:10E2D0009885CDCFA4E0B0E0E0E7F1E70C9412EE32
:10E2E0007C01062F5A01122F862F660F990B9C0175
:10E2F0002A5C3D4F690186E0882E912C11160CF0A6
:10E300003DC0AE014F5F5F4F62E376E6C701B8DA0A
:10E310007C0169817A818B819C8161157105810500
:10E32000910561F16D3371058105910509F450C0C6
:10E330006E3771058105910509F44AC06A3271058D
:10E340008105910501F507FF11C08CE591E20E3FB3
:10E3500011F088E591E236E01302B001112471DF7B
:10E3600066E070E00E94DEED161B60C065E470E0C0
:10E3700080E090E074DB115069F510E0812F249665
:10E38000ECE00C942EEE643271058105910571F478
:10E39000A114B104D1F0E6E01E02B0011124C501C0
:10E3A00050DFB4010E94DEED161BA8CF603471056A
:10E3B0008105910551F41150F6016081062E000C83
:10E3C000770B880B990B4BDB99CF49DB115096CF1C
:10E3D00007FDBBCF61E089819A81AB81BC81CD977C
:10E3E000A105B10509F460E0600F6A30A4F0115096
:10E3F000862F6AE00E94BDED092F682F880F770BEA
:10E40000605D7F4F072E000C880B990B28DB1123D2
:10E4100009F4B3CF602F062E000C770B605D7F4FA1
:10E42000072E000C880B990B1ADB1150112309F4ED
:10E43000A4CF86E01802B0011124C70102DF66E014
:10E4400070E00E94DEED161B99CFE2E9F3E183AFA5
:10E4500064AF6FEF7FEFCA01F4CEACE0B0E0E3E36E
:10E46000F2E70C9416EEF090CD13E090CE132091CD
:10E470002D06211112C048EF50E26E2D8F2D0E9403
:10E4800093D190E080E0F80EF092CD13E092CE139D
:10E4900099272C96E8E00C9432EEC0909A13D09015
:10E4A0009B1326E933E13A8329832F2D30E03C8307
:10E4B0002B832E2D30E03E832D8318861F827A8792
:10E4C00069871C861B8609E61AE69E012F5F3F4F6F
:10E4D00045E356E6BC01C6010E941DB0B60186E9BF
:10E4E00093E10E94E2D08F819885CDCF6FEF7FEFCF
:10E4F000B4CFB0E0A0E0EFE7F2E70C9414EE5C01DB
:10E500006B01B0D9E82EC6010E943866F12C03E1F8
:10E5100010E0081B1109C5E20E151F050CF4CFE130
:10E520008C2F90E09C012E5F3F4F4091CA13421701
:10E53000130609F08CF509972091CC1328171906BA
:10E540005CF140917F075091800760917E071092A7
:10E55000CD13C093CE1325E1C501BCDED1E0C114BB
:10E56000D104A9F06AE370E080E090E078DA0E155B
:10E570001F05A4F4C45F8091CA13C81740F020910E
:10E58000CC134C2F4950550B241715064CF4CDB71E
:10E59000DEB7EAE00C9430EED0E0E1CFDD23B9F352
:10E5A000802F880F080F000F0093CD13C093CE1358
:10E5B00060E270E080E090E052DAC60197DFE7CFDA
:10E5C000ACE0B0E0E6EEF2E70C9412EE982F862F66
:10E5D0006A017901B02E692FFAD9882309F487C01E
:10E5E00010912D06C701002371F13CD9A82E80900F
:10E5F0009A1390909B13111142C02FEF3FEF122FEF
:10E6000023E12A1940917F075091800760917E078E
:10E61000C60160DEAA2009F46AC0B6E08B9F6001E3
:10E6200011246AE370E080E090E019DA57E0C51643
:10E63000D10408F442C060E270E080E090E00FDABC
:10E64000C81AD90AF3CF0E943866A82E80909A1370
:10E6500090909B13112389F2FE0133968AE0DF012B
:10E660001D928A95E9F786E993E19A83898302E40A
:10E670001AE69E012F5F3F4F45E356E612C0FE01AA
:10E6800033968AE0DF011D928A95E9F786E993E1E6
:10E690009A83898302E41AE69E012F5F3F4F42E38B
:10E6A00056E6B701C4010E941DB0B40186E993E1AA
:10E6B0000E94E2D02F813885A2CF40917D07212F83
:10E6C00030E0A6E0AA9EC00111242E5F3F4F28171C
:10E6D00039070CF49C0180E8821B8093CD13409392
:10E6E000CE13BB2041F06FEF7FEFC701AADD2C9660
:10E6F000ECE00C942EEEC701F9DEF9CFE2E9F3E18C
:10E7000083AF64AFCA01F2CE0C94A3B04F925F9274
:10E710006F927F928F929F92BF92CF92DF92EF92F1
:10E72000FF920F931F93CF93DF93109223061092C3
:10E7300022062FE320932606109225061092240627
:10E7400010921E0610921F061092200610922106AB
:10E750009C01F90190812F5F3F4F9032D1F39E349D
:10E76000C9F4818190ED980F9A3020F08D3211F02C
:10E770008B3281F432969F012F5F3F4F808180530F
:10E780008A3008F46DC09F012F5F3F4F8081803237
:10E7900009F468C0F0939507E09394078F010F5F29
:10E7A0001F4FC0816AE270E0C8010E945DF00097CF
:10E7B00031F0FC01319780818032E1F31182CD3458
:10E7C00021F0C43511F0C734D9F5F80180810F5F0D
:10E7D0001F4F8032D1F380538A3090F5C0932606C4
:10E7E00090E080E06AE0AF014F5F5F4F689F90016B
:10E7F000699F300D1124C901C0972081820F911D9E
:10E8000027FD9A95FA01208120532A3060F39093D6
:10E81000250680932406DF0131962C912032D9F30E
:10E82000CD3461F58E31910539F0F0F487319105E1
:10E8300019F08C31910511F5B0932306A0932206AF
:10E84000DF91CF911F910F91FF90EF90DF90CF90CC
:10E85000BF909F908F907F906F905F904F900895A2
:10E86000F90189CFF9018FCF8537910538F08737C6
:10E87000910510F3803A13E09107F1F2809094072C
:10E880009090950740E050E0BA0130E020E0C12CC4
:10E89000D12C7601C394FD013196DC91DD2309F47E
:10E8A00084C0D132F1F4CD34E1F480329105C9F461
:10E8B00040931E0650931F06609320067093210616
:10E8C000F0932306E093220663E270E0CF010E94FA
:10E8D0005DF0009709F4B4CFFC011082B1CFDF01E5
:10E8E000DACFD154DA3108F05BC0DF011D9110326C
:10E8F00091F0A0EDA10FAA30E8F01E3271F4A181D1
:10E90000A053AA30B8F02115310519F49F01215008
:10E910003109B12C13C0FD01E8CF1D3211F01B32BB
:10E9200091F7A181B0EDBA0FBA3020F0AE3259F7AD
:10E93000A281E6CFBE2EB818309759F3AD2FB0E0C4
:10E940002601370104C0440C551C661C771CDA955F
:10E95000D2F74429552966297729AC5FB94FBC9273
:10E96000A081A154AA3108F4BACFDF01D191DD23EF
:10E9700009F491CF00EDB02EBD0E19E01B15A8F7DC
:10E9800013EDB12EBD0E11E01B1578F7DB3269F3E4
:10E99000FD013196DC91D03209F07DCFDF01F8CF57
:10E9A00021153105E9F69D01DBCF30932306209335
:10E9B000220640931E0650931F0660932006709314
:10E9C00021063ECFFC016591759185919491089542
:10E9D0008F929F92AF92BF92CF92DF92EF92FF926F
:10E9E000CF93DF93EC018090B4029090B502A09099
:10E9F000B602B090B70220E030E0A901C501B40131
:10EA00000E9426E7882309F452C0C880D980EA8092
:10EA1000FB80A7019601C501B4010E9426E71816E4
:10EA20000CF04AC02091EE053091EF054091F005C1
:10EA30005091F105C701B6010E9426E7882321F114
:10EA4000C092EE05D092EF05E092F005F092F1054C
:10EA50002091EA053091EB054091EC055091ED05D0
:10EA6000C701B6010E948BE79B01AC0160E070E03A
:10EA700080E89FE30E9443EE60934A0170934B014C
:10EA800080934C0190934D0160914A0170914B012C
:10EA900080914C0190914D01DF91CF91FF90EF90CB
:10EAA000DF90CF90BF90AF909F908F90089560E0DF
:10EAB00070E080E89FE3F0CF60E070E0CB01ECCF46
:10EAC000B0E0A0E0E6E6F5E70C940EEEEC01209154
:10EAD0007C0330917D0340917E0350917F036881D8
:10EAE00079818A819B810E9443EE4B015C012091D8
:10EAF00080033091810340918203509183036C81A4
:10EB00007D818E819F810E9443EE6B017C01A50176
:10EB10009401609142017091430180914401909170
:10EB200045010E9426E7882309F454C080924201DF
:10EB300090924301A0924401B09245012091E205D8
:10EB40003091E3054091E4055091E505C501B4011C
:10EB50000E948BE72B013C010E9454EF4B015C01AA
:10EB600020E030E040EA50E40E9426E7181634F432
:10EB7000812C912CC0EAAC2EC0E4BC2E20E030E009
:10EB8000A901C501B4010E94A7EF87FF03C0812C32
:10EB9000912C5401A5019401C301B2010E9443EEDE
:10EBA0006093DA057093DB058093DC059093DD05B7
:10EBB000C501B4010E9423EF6093D805062E000C16
:10EBC000770B6F5F7F4F6630710514F066E070E081
:10EBD0006093D605D09140011091D805A701960108
:10EBE00060914601709147018091480190914901DF
:10EBF0000E9426E7811123C0D11375C02091BE0564
:10EC00003091BF054091C0055091C1056091DA0572
:10EC10007091DB058091DC059091DD050E948BE70A
:10EC20002091C2053091C3054091C4055091C5059E
:10EC30000E9444EECDB7DEB7E0E10C942AEEC0921C
:10EC40004601D0924701E0924801F092490120919B
:10EC5000E6053091E7054091E8055091E905C701C7
:10EC6000B6010E948BE74B015C010E9454EF6B01DF
:10EC70007C0120E030E040EA50E40E9426E71816CC
:10EC800034F4C12CD12CB0EAEB2EB0E4FB2E20E002
:10EC900030E0A901C701B6010E94A7EF87FF03C0BA
:10ECA000C12CD12C7601A7019601C501B4010E94A7
:10ECB00043EE6093DE057093DF058093E00590934B
:10ECC000E105C701B6010E9423EF6093D905062E26
:10ECD000000C770B6F5F7F4F6630710514F066E0B4
:10ECE00070E06093D705C091D905D11305C080911C
:10ECF00041018C1709F470C08091D8059091D90515
:10ED000090934101809340010C2E000CDD0B27E015
:10ED10001203C0011124FC01EC0FFD1FEE0FFF1FB9
:10ED2000EE0FFF1FE854FD4F208131814281538156
:10ED30002093D2053093D3054093D4055093D50545
:10ED40000091D705002E000C110BFC01E00FF11F04
:10ED5000EE0FFF1FEE0FFF1FE854FD4F6081718122
:10ED6000828193810E9443EE6093CE057093CF051C
:10ED70008093D0059093D1052091D60537E02303E9
:10ED8000F0011124CE0FDF1FCC0FDD1FCC0FDD1FD4
:10ED9000C854DD4F288139814A815B812093CA059F
:10EDA0003093CB054093CC055093CD05E00FF11F78
:10EDB000EE0FFF1FEE0FFF1FE854FD4F60817181C2
:10EDC000828193810E9443EE6093C6057093C705CC
:10EDD0008093C8059093C9058090DE059090DF056B
:10EDE000A090E005B090E1052091CE053091CF05CF
:10EDF0004091D0055091D105C501B4010E948BE727
:10EE00002091D2053091D3054091D4055091D5057C
:10EE10000E9444EE6B017C01C092C205D092C305F2
:10EE2000E092C405F092C5052091C6053091C70552
:10EE30004091C8055091C905C501B4010E948BE7F6
:10EE40002091CA053091CB054091CC055091CD055C
:10EE50000E9444EEA70196010E9443EE6093BE0516
:10EE60007093BF058093C0059093C105C7CEACE0F9
:10EE7000B0E0EDE3F7E70C941BEE182F882379F050
:10EE800020E030E0A90160918403709185038091B6
:10EE90008603909187030E9426E78823F1F08091F2
:10EEA000B3028117D1F00E94DB2B8CE0EAE2F2E0A2
:10EEB000DE01119601900D928A95E1F7CE0101963F
:10EEC000FFDD8091B302882361F085E791E00E9425
:10EED000312C1092B3020E94D63E2C96E3E00C94A3
:10EEE00037EE81E08093B30285E791E00E94FD2B2D
:10EEF000F2CFCF92DF92EF92FF9280E0B8DF1092D4
:10EF00008003109281031092820310928303109267
:10EF10007C0310927D0310927E0310927F03109267
:10EF200088031092890310928A0310928B03109227
:10EF3000840310928503109286031092870348EB96
:10EF400052E027E0C12CD12C60ECE62E6FE7F62EC4
:10EF500090E080E0FC01EE0FFF1FEE0FFF1FE40FBB
:10EF6000F51FC082D182E282F3820196873091053B
:10EF700089F72150445E5F4F2111EACFFF90EF9057
:10EF8000DF90CF9008954F925F926F927F928F9211
:10EF90009F92AF92BF92CF92DF92EF92FF921F9318
:10EFA000CF93DF93EC01162F2091B4023091B5027C
:10EFB0004091B6025091B702688179818A819B8124
:10EFC0000E9426E7882309F497C0B090B30280E03E
:10EFD0004EDFC880D980EA80FB8020E030E0A901C4
:10EFE000C701B6010E94A7EF87FF03C0C12CD12C37
:10EFF0007601C092B402D092B502E092B602F092CD
:10F00000B7022DEB37E346E855EBC701B6010E9486
:10F0100026E787FD0BC02DEB37E346E855E3C70134
:10F02000B6010E94A7EF18160CF076C0A701960152
:10F0300060E070E080E89FE30E94BBEE6093EA0529
:10F040007093EB058093EC059093ED0580EF9FEFB7
:10F05000A9E7B4EC8093EE059093EF05A093F0053B
:10F06000B093F105BB2009F447C040907501509062
:10F07000760160907701709078018090790190908E
:10F080007A01A0907B01B0907C01C0907D01D0906E
:10F090007E01E0907F01F090800181E0E8DE1123A5
:10F0A00059F1A301920160917501709176018091EF
:10F0B0007701909178010E9426E781111BC0A5017C
:10F0C00094016091790170917A0180917B01909116
:10F0D0007C010E9426E781110DC020917D013091B5
:10F0E0007E0140917F0150918001C701B6010E94CD
:10F0F00026E781110E94FC3EDF91CF911F91FF9086
:10F10000EF90DF90CF90BF90AF909F908F907F90C7
:10F110006F905F904F90089560E070E0CB018ECFCC
:10F120008F929F92AF92BF92CF92DF92EF92FF9217
:10F13000C0908403D0908503E0908603F09087030D
:10F1400020E030E0A901C701B6010E9426E788232C
:10F15000E1F1A701960160E070E080E89FE30E9482
:10F16000BBEE6B017C018090880390908903A09096
:10F170008A03B0908B0320E030E0A901C501B401FF
:10F180000E9426E7882329F1A501940160E070E040
:10F1900080E89FE30E94BBEEC092E205D092E305B7
:10F1A000E092E405F092E5056093E6057093E705CB
:10F1B0008093E8059093E905FF90EF90DF90CF9062
:10F1C000BF90AF909F908F900895C12CD12C760165
:10F1D000CACF60E070E0CB01DFCFCF92DF92EF9239
:10F1E000FF926B017C0183E3C816D104E104F104B2
:10F1F00070F082E3C81AD108E108F10862E370E018
:10F2000080E090E00E946BCD0E941D29ECCFC701E9
:10F21000B6010E946BCD0E941D29FF90EF90DF90F8
:10F22000CF900895BC0190E080E00C9446B08091AE
:10F230009207813069F09091E81492FB882780F959
:10F2400092FF07C097FB882780F991E089270895EE
:10F2500081E008959091E81494FB882780F994FF49
:10F2600006C081E09091D112911101C080E0089513
:10F27000A4E0B0E0EEE3F9E70C940EEE10927C0708
:10F280008091590710925907882361F020E040E0EF
:10F2900070E060E089EA90E60E944C452496E0E147
:10F2A0000C942AEE209110013091110140917407C5
:10F2B00050917507CA01820F931F2436310509F05A
:10F2C0001DC44730510544F006978A3091050CF073
:10F2D00024C48AE090E02BC406964A3F5F4FACF30B
:10F2E00080917307882309F4C8C16091BD127091A1
:10F2F000BE12072E000C880B990B0E942CE7B1E080
:10F30000B9832091B9123091BA124091BB12509139
:10F31000BC120E94A7EF18160CF0198260913E07EC
:10F3200070913F07072E000C880B990B0E942CE769
:10F3300020913A0730913B0740913C0750913D079F
:10F340000E94A7EF18161CF4E981E260E983C980E6
:10F35000C0925E06C0907501D0907601E090770172
:10F36000F09078018091790190917A01A0917B01D0
:10F37000B0917C0189839A83AB83BC8380907D01AB
:10F3800090907E01A0907F01B090800120E030E05D
:10F390004AE754E4C501B4010E948BE72B013C010C
:10F3A00020E030E0A901C501B4010E9426E720E079
:10F3B00030E040EA50EC87FD04C020E030E040EA55
:10F3C00050E4C301B2010E9444EE2DEC3CEC4CEC45
:10F3D0005DE30E948BE70E9423EF4B015C0180E21A
:10F3E000B7FE09C0B094A09490948094811C911CA5
:10F3F000A11CB11C8DE280939B0260E290E1891612
:10F4000097E29906A104B1048CF0C501B40120E192
:10F4100037E240E050E00E9476EDCA01B9012AE0EF
:10F4200030E040E050E00E9476ED605D60939C0229
:10F4300060E2A8EE8A16A3E09A06A104B1048CF05B
:10F44000C501B40128EE33E040E050E00E9476EDC3
:10F45000CA01B9012AE030E040E050E00E9476EDB8
:10F46000605D60939D02C501B40124E630E040E098
:10F4700050E00E9476ED6AE0462E512C612C712CF2
:10F48000CA01B901A30192010E9476ED605D60930B
:10F490009E02C501B401A30192010E9476ED4B01C9
:10F4A000CA01B901A30192010E9476ED882009F4F6
:10F4B0004EC32EE220939F02605D6093A002B0E3F2
:10F4C0008B0E8092A1026BE972E086E596E00E94C5
:10F4D00068F020E030E0A901C701B6010E9426E7EC
:10F4E00020E030E040E05FEB87FD04C020E030E04A
:10F4F00040E05FE3C701B6010E9444EE0E9423EFA3
:10F50000CB010E949043BC0181E596E00E9468F027
:10F5100020E030E0A90169817A818B819C810E9481
:10F5200026E720E030E040E05FEB87FD04C020E00C
:10F5300030E040E05FE369817A818B819C810E94A9
:10F5400044EE0E9423EFCB010E949043BC018CE467
:10F5500096E00E9468F08091E81483FD0AC37ADE89
:10F56000882309F409C38091E0149091E114A091DB
:10F57000E214B091E3140097A105B10509F4FCC2AF
:10F58000BC01CD016D597F4F8F4F9F4F24E630E076
:10F5900040E050E00E9454ED6091E4147091E51455
:10F5A0008091E6149091E7140E9454ED29830E9403
:10F5B000CF424B015C01162F80915C01C9808C15F4
:10F5C000C1F0C0925C0128E4C29EB001112490E019
:10F5D00080E00E942AE72AE037ED43E25CE30E94E4
:10F5E0008BE70E9428EF60934B06C110C7C21092B0
:10F5F000460680915B01181709F43FC080925B01B9
:10F60000C501B40120E13EE040E050E00E9454ED2D
:10F61000690189019CE3492E512C612C712CC50193
:10F62000B401A30192010E9454ED4B015C01CA0197
:10F63000B901A30192010E9454EDC114D10409F053
:10F64000C4C29F928F927F936F938CE791E29F93B6
:10F650008F9386E396E09F938F930E94BFE60FB649
:10F66000F894DEBF0FBECDBF85E0982F990F990F9C
:10F67000891B880F8058809335060E94F7CD009132
:10F6800030061091310620913206309133066B011D
:10F690007C01C01AD10AE20AF30A9701860137FDFC
:10F6A00011C020912F06209520932F066A547C4F7D
:10F6B0008F4F9F4F609330067093310680933206D0
:10F6C00090933306D0902F06D98281E00E941E6D60
:10F6D0008091CA13873180F48091CC13843060F01C
:10F6E0008FE5E82E82E2F82E03E126E044E064E0B4
:10F6F00086E993E10E94B8D180915E06982F9270BE
:10F7000048E00CE081FD02C042E102E08091CA13B2
:10F71000843180F48091CC13841760F0992309F42C
:10F7200073C28BE392E27C0123E060E586E993E11A
:10F730000E94B8D18091CA138431C0F48091CC1357
:10F740008230A0F0C980CC2009F461C28091B20758
:10F75000882309F45CC28FEF91E27C0102E123E08F
:10F7600042E068E686E993E10E94B8D18091CA132D
:10F770008C3108F09DC08090B9129090BA12A09080
:10F78000BB12B090BC12C090BD12D090BE1284319A
:10F7900098F48091CC13883078F080915E0680FFD9
:10F7A00039C281EB91E27C010CE022E048E069E3A0
:10F7B00086E993E10E94B8D18091CA13883040F461
:10F7C000D7FE2BC245E951E267E087E30E9425722C
:10F7D0008091CA138C31B0F48091CC13843190F0B5
:10F7E00020E030E040E05FE3C501B4010E9444EE58
:10F7F0000E9423EF77FF34C245E951E26CE187E3D1
:10F800000E942572C0903A07D0903B07E0903C07D9
:10F81000F0903D078091CA13883060F480913E07D4
:10F8200090913F0797FF3FC245E951E267E081E5CC
:10F830000E9425728091CA138C31B0F48091CC1350
:10F84000843190F020E030E040E05FE3C701B60192
:10F850000E9444EE0E9423EF77FF47C245E951E240
:10F860006CE181E50E9425728091CA138C3100F50C
:10F870008091CC138431E0F08091B2078823C1F0ED
:10F8800024E6829FC001112481589F4F6FEF70E0E2
:10F890000E94DEEDCB010E940F44AC016CE187E6D3
:10F8A0000E947E7365E270E080E090E00E942F6D20
:10F8B000D1DC882379F18091CA13843358F5809183
:10F8C000CC138A3238F107E028E04AE26AE286E99E
:10F8D00093E10E945FD005E022E04CE262E386E91A
:10F8E00093E10E945FD024E04AE061E38AE20E9453
:10F8F0002FD0609198137091991382E38093B21383
:10F900008BE28093B31322EB33E142E386E993E188
:10F910000E942FCF8091CA13853350F48091CC136D
:10F92000813330F024E04AE461E386E30E942FD083
:10F930008091CA13843368F48091CC13823348F0E9
:10F9400002E020914B0642E367E386E993E10E94DF
:10F950005FD08091CA138033D8F48091CC13883261
:10F96000B8F080914606882361F046E456E060E3F3
:10F9700087E30E947E7365E270E080E090E00E9481
:10F980002F6D46E356E060E3809135060E947E735A
:10F990008091CA13883208F060C08091CC138D31F9
:10F9A00008F45BC02BE040E86DE180E00E942FD0BE
:10F9B0008091CA13873208F050C08091CC138F31E8
:10F9C00008F44BC083E08093CD1316E21093CE135E
:10F9D00068E570E080E090E00E942F6D8BE08093FE
:10F9E000CD131093CE13C980CC2009F4A1C181E5B9
:10F9F00096E00E94767288E28093CD1316E210930F
:10FA0000CE1369E570E080E090E00E942F6D80E306
:10FA10008093CD131093CE13C980CC2009F4ABC1D1
:10FA20008CE496E00E9476728DE48093CD1316E20A
:10FA30001093CE136AE570E080E090E00E942F6D95
:10FA400085E58093CD131093CE13C980CC2009F4A3
:10FA5000B5C186E596E00E9476728091CA13833321
:10FA600038F58091CC138B3218F183E00E941E6D23
:10FA700083E08093CD1383E38093CE1366E070E040
:10FA800080E090E00E942F6D81E00E941E6D8091C9
:10FA90001001909111010E940F44AC0163E38CE0CE
:10FAA0000E947E7365E270E080E090E00E942F6D1E
:10FAB0008091CA13813408F0F1CB8091CC13863346
:10FAC00008F4ECCB1092CD138EE38093CE138AE42E
:10FAD00090E10E943866182F863108F092C18AE4BE
:10FAE00090E10E947672153109F4D8CB60E270E0A3
:10FAF00080E090E00E942F6D1F5FF5CF2436310526
:10FB00004CF48536910504F58A30910534F48AE089
:10FB100090E009C084369105BCF0883EA3E09A07C6
:10FB200014F087EE93E02817390709F4D9CB9093A6
:10FB300011018093100110927407109275071092B2
:10FB4000760710927707CCCB84E690E0F0CF66235F
:10FB500051F02EE220939F02605D6093A00280E24C
:10FB60008093A102B0CC80E28093A00280939F0298
:10FB7000F6CFE4E6E9831BCD198219CD498180E2F5
:10FB8000443628F0842F64E60E94B1ED805D8093B6
:10FB90009F02698190E26A3040F02AE0862F622F4E
:10FBA0000E94B1ED0E94B1ED905D9093A002898119
:10FBB0006AE00E94B1ED905D9093A1026FE972E05E
:10FBC00086E496E00E9468F014CD0436110538F4FE
:10FBD0007F936F93DF92CF9280E791E238CD7F934E
:10FBE0006F93DF92CF9286E691E29F938F9386E3A5
:10FBF00096E09F938F930E94BFE60FB6F894DEBF06
:10FC00000FBECDBF86E031CD85E392E28CCD89EC8D
:10FC100091E2A3CD89E991E2C6CDC6010E940F44CD
:10FC2000FC01808193E0803229F4818192E080326E
:10FC300009F491E043E050E0491B51094E0F5F1F6A
:10FC4000892F880F880F981B892F67E0805C0E949E
:10FC50007E7369E070E080E090E00E942F6DB8CD87
:10FC6000CB010E940F44FC01808193E0803229F493
:10FC7000818192E0803209F491E043E050E0491B39
:10FC800051094E0F5F1F892F880F880F981B892FEE
:10FC90006CE1805C0E947E7369E070E080E090E03F
:10FCA0000E942F6DAFCD0E940F44FC01808193E034
:10FCB000803229F4818192E0803209F491E043E0BE
:10FCC00050E0491B51094E0F5F1F892F880F880F85
:10FCD000981B892F67E0865A0E947E7369E070E066
:10FCE00080E090E00E942F6DA5CDCB010E940F44D3
:10FCF000FC01808193E0803229F4818192E080329E
:10FD000009F491E043E050E0491B51094E0F5F1F99
:10FD1000892F880F880F981B892F6CE1865A0E94C3
:10FD20007E7369E070E080E090E00E942F6D9CCDD2
:10FD300087E00E94FF3980FF13C001E516E0D8017B
:10FD40006D918D01662309F456CE6F320CF06FE38E
:10FD5000062E000C770B880B990B0E942F6DEFCFAE
:10FD60008091820780FD43CE6FEF7FEF80E991E2C3
:10FD70000E94217140CE87E00E94FF3981FF13C0AD
:10FD80000CE416E0D8016D918D01662309F44CCE88
:10FD90006F320CF06FE3062E000C770B880B990B7B
:10FDA0000E942F6DEFCF8091820781FD39CE6FEFDA
:10FDB0007FEF80E991E20E94217136CE87E00E94B8
:10FDC000FF3982FF13C006E516E0D8016D918D0161
:10FDD000662309F442CE6F320CF06FE3062E000C5E
:10FDE000770B880B990B0E942F6DEFCF80918207C4
:10FDF00082FD2FCE6FEF7FEF88E891E20E942171A4
:10FE00002CCE81E0C980C11001C080E09091340601
:10FE10008917C9F0D0904910D982809334068AE4BA
:10FE200090E10E943866D81608F054C029812F5FEF
:10FE30002983E22FF0E0E65BFF4E8081807C8038F2
:10FE4000A9F3209349100091491010E0065B1F4E62
:10FE5000C8010E943866898360E870E0C8010E948A
:10FE60002D724981453108F019CA60E270E080E0E6
:10FE700090E00E942F6D6981643109F40FCA60E23D
:10FE800070E080E090E00E942F6D8981833109F459
:10FE900005CA60E270E080E090E00E942F6D9981D9
:10FEA000923109F4FBC9292F30E02E5F3F4F4AEF12
:10FEB0004203B001439F700D112460587F4F8AE4C4
:10FEC00090E10E942D7260E270E080E090E00E947C
:10FED0002F6DE4C910924910B6CF809192078230FD
:10FEE00059F0B8D9882349F08091E81482FB88271B
:10FEF00080F991E08927089581E0089581E00895CF
:10FF0000DC01EC918E2F90E0FC01EE0FFF1FE80F5B
:10FF1000F91FEF5CFC4E80818F7780830895892BD9
:10FF200079F41092900082E08093910010929500F5
:10FF300010929400C19A8091710082608093710048
:10FF40000895B0E0A0E0E7EAFFE70C9411EEEC01C1
:10FF50006B0188818C3008F0A6C090E0FC01EE0FA8
:10FF6000FF1FE80FF91FEF5CFC4E80818F770E9426
:10FF7000CEB219821A8288812CE0622F0E94B1EDE4
:10FF8000829FB001112430E020E0AB01420F531FEB
:10FF9000FA01EE0FFF1FE40FF51FEF5CFC4E90819E
:10FFA00097FD07C02F5F3F4F2C30310571F790E070
:10FFB000B6DF7880E72CF12C8701000F111FF801C4
:10FFC000EE0DFF1DEF5CFC4E80818068808377FC26
:10FFD0006AC080E2C81682E0D8060CF03FC08A8171
:10FFE00028E532E0281B310987FD3395220F331FA6
:10FFF000220F331F032E000C440B550B898178E828
:020000021000EC
:10000000872E912C881A910887FD9394880C991C4F
:10001000880C991C092C000CAA08BB0860E070E051
:10002000CB01D7FC0AC0B601653B710514F064EB47
:1000300070E0072E000C880B990B281939094A0922
:100040005B090E9445ED24EB30E040E050E00E9467
:1000500076ED820E931EA41EB51E64018BE08715FB
:10006000D8F0298188E890E0821B910927FD9395BB
:10007000880F991F880F991FC816D906CCF40297CC
:100080002FB7F8940E0D1F1DF801EF5CFC4E880F82
:10009000991F928381832FBF6EE571E080E090E02D
:1000A0009CD8CE012DDFCDB7DEB7EDE00C942DEE60
:1000B0002A8188E592E0821B910927FD9395880F9C
:1000C000991F880F991FC816D906CCF6C601D7CF3D
:1000D0001F920F920FB60F9211240BB60F922F930F
:1000E0003F934F935F936F937F938F939F93AF93C0
:1000F000BF93EF93FF938091AF0587FF27C01092C6
:100100009500109294008091AF058F5F8093AF05AA
:100110008091AF05082E000C990B209155132817DC
:10012000190629F024F08091AF058C30DCF1809124
:10013000940090919500049680349C4908F47DC009
:100140008091940090919500049679C08091AF05BC
:10015000082E000C990B209155132817190699F2B7
:1001600094F2E091AF058E2FEE0F990BFC01EE0F8C
:10017000FF1FE80FF91FEF5CFC4E808187FFC3CFA4
:10018000E091AF058E2FEE0F990BFC01EE0FFF1FD4
:10019000E80FF91FEF5CFC4E808160E08F770E94D2
:1001A0000FCDB1CF2091940030919500E091AF0533
:1001B0008E2FEE0F990BFC01EE0FFF1FE80FF91FBA
:1001C000EF5CFC4E81819281820F931F9093990086
:1001D00080939800E091AF058E2FEE0F990BFC01F4
:1001E000EE0FFF1FE80FF91FEF5CFC4E808187FFC9
:1001F00011C0E091AF058E2FEE0F990BFC01EE0FB1
:10020000FF1FE80FF91FEF5CFC4E808161E08F77E4
:100210000E940FCDFF91EF91BF91AF919F918F9170
:100220007F916F915F914F913F912F910F900BBEF6
:100230000F900FBE0F901F90189580E49CE990934B
:100240009900809398008FEF8093AF05E3CF909152
:10025000C00095FFFCCF8093C6000895CF93DF9335
:10026000EC018991882311F0F2DFFBCFDF91CF9170
:100270000895CF93DF93EC018991882311F0E7DF94
:10028000FBCF8DE0E4DF8AE0E2DFDF91CF910895DC
:10029000CF93DF93EC01FE0184912196882311F026
:1002A000D6DFF9CFDF91CF9108950F931F93CF93AE
:1002B0008C01C62F8AED9EE1EBDFC801E9DF8AE3FE
:1002C000C6DF80E38C0FC3DF8AE0C1DFCF911F91CF
:1002D0000F910895CF92DF92EF92FF926A017B0116
:1002E000D7DF42E0C701B6010E94EDB2FF90EF9068
:1002F000DF90CF900895CF93DF9361EF7EE10E946E
:100300003AC4C0916513D0916613488159816A81BE
:100310007B8188EE9EE1DEDF4C815D816E817F8195
:100320008EEE9CE2D7DF4091611350916213609191
:100330006313709164138BEE9CE2CCDF85EE9EE13B
:10034000A7DF8FED9EE1A4DF8AE081DFDF91CF910F
:100350000895C0DF8AE07BCFADE5B0E0E2EBF1E8E5
:100360000C940CEE70E060E085E40E94436B7C012D
:10037000182F8F3FB1F1882341F084ED90E288DFA0
:10038000C35ADF4FE2E10C9428EE6EEB70E083E598
:100390000E94436B5C0165E070E083E40E94436B64
:1003A0006C0160E085E50E942F6B2C968FAF2C9737
:1003B00060E087EC90E20E940B5A0E94F7CD6987BB
:1003C0007A878B879C871F3F09F067C434E7A316A1
:1003D000B1040CF489C18CE990E25ADF0E94BDC4DB
:1003E000CFCF6CE370E0D3CF20E030E040E05EE3BD
:1003F0002BAF3CAF4DAF5EAFABC12AE939E949E164
:100400005FE323962CAF3DAF4EAF5FAF2397ADC1F7
:100410004090B9125090BA126090BB127090BC120A
:1004200051C22B96EEADFFAD2B974083A4C24BEE8D
:10043000C42ED12CE12CF12C22C384E190E0A0E069
:10044000B0E08D879E87AF87B88B34E1C32ED12C67
:10045000E12CF12C24C3CD86DE86EF86F88A1FC3FB
:100460002B96EEADFFAD2B978083E9C3D501C40178
:100470002EA53FA548A959A9821B930BA40BB50B28
:10048000B7FD47C02D968FAD2D970E9479268AE043
:10049000DEDED501C4018053984FAF4FBF4F8EA70A
:1004A0009FA7A8ABB9AB9AA991116FC02BA93CA982
:1004B0004DA95EA9C301B2010E94A7EF18160CF066
:1004C00050C020E030E040E050E4C301B2010E949F
:1004D00044EE6BAB7CAB8DAB9EAB2AA53BA54CA58C
:1004E0005DA5280D391D4A1D5B1D2FAB38AF49AFE7
:1004F0005AAF6D966CAD7DAD8EAD9FAD6D970E9480
:100500002CE7A30192010E9426E7881F8827881FF5
:100510008AAB89859A85AB85BC85898F9A8FAB8F8D
:10052000BC8F29893A894B895C89281739074A0782
:100530005B0720F4298F3A8F4B8F5C8F898D9A8DC2
:10054000AB8DBC8D881A990AAA0ABB0A91E8891654
:100550009FE4990692E1A906B10460F180EC9FE165
:100560002DC2D501C4012FA938AD49AD5AAD821BAA
:10057000930BA40BB50B45EB52E164EC72E1B7FDB4
:10058000C8CF812F0E94C027C4CF69966CAD7DADC6
:100590008EAD9FAD69970E942CE79B01AC01C30112
:1005A000B2010E9426E787FFB4CF42EF52E162E03A
:1005B00073E1E7CF2996AEADBFAD2997A215B3057C
:1005C0000CF08FC0B3E02B1631040CF48AC083E624
:1005D0009FE15EDE1F3F09F066C0E3E5FFE1FE83B9
:1005E000ED8382E49FE154DE8D819E8151DE49815D
:1005F0005A816B817C818FE59FE1ABDE82E49FE1D4
:1006000047DE8D819E8144DE4D8D5E8D6F8D78A19C
:100610008BE59FE19EDE82E49FE13ADE8D819E8143
:1006200037DE49A15AA16BA17CA187E59FE191DE4C
:100630002C963FAD2C97332309F4D0CE2CEA35EC21
:1006400047E25EE36D8D7E8D8F8D98A10E948BE7D2
:100650006B017C0120E030E543EC50E469A17AA114
:100660008BA19CA10E948BE729813A814B815C81FF
:100670001F3FF1F420934107309342074093430713
:1006800050934407C0924507D0924607E09247072F
:10069000F09248076093490770934A0780934B078D
:1006A00090934C079BCE2EE33CE23E832D8399CF63
:1006B0002093C0123093C1124093C2125093C312C0
:1006C000C092C412D092C512E092C612F092C71224
:1006D0006093C8127093C9128093CA129093CB1280
:1006E0007DCE0E94896ECEC088E890E2D1DD0E9466
:1006F00022278FE7809340072CE330E0C9A6A8EEBD
:10070000B3E00E94A2ED6AA77BA78CA79DA72985CD
:100710003A854B855C85260F371F481F591F2FAB25
:1007200038AF49AF5AAF81E08093690160E084E758
:1007300090E20E940B5A02E00E0D023008F054CEF7
:100740008BEA9AEAAAEABEE38BAF9CAFADAFBEAF2D
:10075000023008F052CE8DEC9CECACE4BEE3239664
:100760008CAF9DAFAEAFBFAF2397023008F4E12C42
:100770002D96EFAE2D9789859A85AB85BC85898BA3
:100780009A8BAB8BBC8B8EA79FA7A8ABB9AB19A2DA
:100790001AA21BA21CA21D8E1E8E1F8E18A21982C9
:1007A0001A821B821C822FE730E040E050E02D8748
:1007B0003E874F87588B80E090E4ACE1B6E48D83B0
:1007C0009E83AF83B8871D8A1E8A1F8A188EFFE713
:1007D000CF2ED12CE12CF12C1AAA1BAA1CAA1DAADF
:1007E0001EAA1DA21EA21FA218A691E024969FAFCA
:1007F0002497312C212C412C512C320195010B2CAA
:10080000000C440B550B61962CAF3DAF4EAF5FAF64
:10081000619749A5042E000C550B29965FAF4EAF8A
:10082000299757E11502C0011124DC01A154BD4EE6
:100830002B96BFAFAEAF2B97C5014E969C01092EEC
:10084000000C440B550B65962CAF3DAF4EAF5FAF20
:100850006597CC979C01990F440B550B69962CAF6B
:100860003DAF4EAF5FAF699736E0A31AB108C5013F
:100870000B2C000CAA0BBB0B6D968CAF9DAFAEAFD3
:10088000BFAF6D9780916901882309F498C00E94D9
:10089000F7CD4B015C0190919D036E969FAF6E97D3
:1008A000992309F47BC00E94B62810929D031F3F34
:1008B00009F0AECD40903A0750903B0760903C075E
:1008C00070903D07A30192016D897E898F89988D73
:1008D0000E94A7EF87FF04C04D8A5E8A6F8A788ED8
:1008E000A30192016D817E818F8198850E9426E708
:1008F000181624F44D825E826F82788661966CAD04
:100900007DAD8EAD9FAD61970E942CE7698F7A8F88
:100910008B8F9C8F2496AFAD2497AA2309F454C0E3
:100920009B01AC01C301B2010E94A7EF1816B4F5F8
:10093000D501C40129893A894B895C89821B930BB3
:10094000A40BB50BAC01BD014858534161097109B5
:1009500077FD24C04D855E856F8578894C195D09CA
:100960006E097F0975956795579547951F3F09F063
:1009700058CD409340078DA39EA3AFA3B8A7298D60
:100980003A8D4B8D5C8D2D8B3E8B4F8B588F89868E
:100990009A86AB86BC8624961FAE249765966CAD6E
:1009A0007DAD8EAD9FAD65970E942CE7A3019201AE
:1009B0000E9426E787FF5ACD8EED9FE169DC1092F9
:1009C00069010E9422270ACD298D3A8D4B8D5C8DBD
:1009D000C301B2010E9426E787FFE0CFD501C40121
:1009E00029853A854B855C85821B930BA40BB50B3F
:1009F000AC01BD01485853416109710977FDCECF63
:100A00002114310409F40AC12DA13EA14FA158A51A
:100A1000280F391F4A1F5B1F298B3A8B4B8B5C8B2E
:100A20002DA13EA14FA158A5281B390B4A0B5B0BEA
:100A3000C701B6010E9445ED29893A894B895C8935
:100A40000E9476EDCD84DE84EF84F888C20ED31E3A
:100A5000E41EF51E34E1C316D104E104F1040CF4E4
:100A6000ECCC4CEEC416D104E104F1040CF0DFCC64
:100A700050E8C516D104E104F1040CF4ECCCCD86A9
:100A8000DE86EF86F88A8EEF90E0A0E0B0E09C0171
:100A9000AD012C193D094E095F0969017A018CE607
:100AA00090E2F6DB6D857E858F8598890E94847340
:100AB00087E690E2EDDBC701B6010E9484734D81A9
:100AC0005E816F81788580E690E204DC4D895E89E5
:100AD0006F89788D89E590E2FDDB93E0291631047A
:100AE0000CF49CC0C701B6010E942CE720E030E066
:100AF00040E850E40E948BE769837A838B839C8370
:100B00002D813E814F8158856D897E898F89988D91
:100B10000E9443EE2BED3FE049EC5FE30E948BE740
:100B20009B01AC0169817A818B819C810E94BBEE23
:100B300027966CAF7DAF8EAF9FAF279769897A8973
:100B40008B899C890E942CE72FE632E143E85AE327
:100B50000E948BE76D837E838F83988723962CADCD
:100B60003DAD4EAD5FAD239727966CAD7DAD8EAD9F
:100B70009FAD27970E948BE769837A838B839C8341
:100B80009B01AC010E9444EE2D813E814F8158852E
:100B90000E94BBEE6D8F7E8F8F8F98A32BAD3CADE7
:100BA0004DAD5EAD6D817E818F8198850E948BE712
:100BB00029813A814B815C810E948BE769A37AA3EA
:100BC0008BA39CA327964CAD5DAD6EAD7FAD2797F3
:100BD00083E590E27FDB4D815E816F8178858DE4D6
:100BE00090E2B7DB8EE390E2023010F08FE290E209
:100BF0004FDB49815A816B817C8189E290E26ADB1B
:100C00004D8D5E8D6F8D78A183E290E263DB49A10B
:100C10005AA16BA17CA18DE190E29BDB8D859E8525
:100C2000AF85B8898C0D9D1DAE1DBF1DB595A795CF
:100C3000979587951F3F09F013CC8093400729961D
:100C4000FFAD2997FF9329A52F933F922F9289E01B
:100C500090E29F938F9384E190E29F938F931F92F2
:100C60000E94EE593FEF231A330A0FB6F894DEBF05
:100C70000FBECDBF898D9A8DAB8DBC8D8D839E832C
:100C8000AF83B887898A9A8AAB8ABC8A6E969FADF1
:100C90006E9724969FAF249781CE8E2C0E2C000C3D
:100CA0009908F40183E0EE0FFF1F8A95E1F7EF59F1
:100CB000FE4F868197810F978A159B050CF48BCB8D
:100CC00088E890E2E5DA0E94222787E1889DF0011A
:100CD000899DF00D1124EB54FD4E8FE7828724E1AE
:100CE00030E00CCDCF93DF9369EF77E10E943AC4F7
:100CF000C6E3D7E04B855C856D857E8580EF97E107
:100D0000E9DA20E030E543EC50E46F8578898989A1
:100D10009A890E948BE7AB01BC018DEE97E1DADA8C
:100D20002CEA35EC47E25EE36B897C898D899E89EC
:100D30000E948BE7AB01BC018AEE97E10ADBDF91F1
:100D4000CF9108956FE577E10E943AC46091840DD8
:100D50007091850D8091860D9091870D0E942AE7F4
:100D6000AB01BC0186E597E1B5DA4091B40D509135
:100D7000B50D6091B60D7091B70D83E597E1AADAD4
:100D80004091B80D5091B90D6091BA0D7091BB0DA5
:100D900080E597E19FDA409196075091970760911F
:100DA0009807709199078DE497E1D3CACF93DF93A9
:100DB00063E077E10E943AC4C4E7DDE04CA95DA995
:100DC0006EA97FA98AEF96E185DA48AD59AD6AAD83
:100DD0007BAD87EF96E17EDA4CAD5DAD6EAD7FAD5C
:100DE00080E597E1B6DADF91CF910895CF93DF9355
:100DF0006FED76E10E943AC4C4E7DDE04CA15DA14D
:100E00006EA17FA186ED96E165DA48A559A56AA590
:100E10007BA58EEE9CE25EDA4CA55DA56EA57FA556
:100E20008BEE9CE257DA48A959A96AA97BA988EEFA
:100E30009CE28FDADF91CF910895CF93DF936AEB35
:100E400076E10E943AC4C4E7DDE0688179818A8155
:100E50009B810E942AE7AB01BC0181EB96E13ADA63
:100E60006C817D818E819F810E942AE7AB01BC014C
:100E70008EEE9CE22FDA688579858A859B850E94B3
:100E80002AE7AB01BC018BEE9CE224DA6C857D8500
:100E90008E859F850E942AE7AB01BC0188EE9CE20B
:100EA00058DADF91CF9108958F929F92AF92BF92BF
:100EB000EF92FF920F931F93CF93DF9384E995E115
:100EC000E7D9C0E0D7E0D15019F080E2C0D9FBCF1C
:100ED0008C2F0E94DF6ACF5FC730A1F78AE0B7D9B5
:100EE00008EB12E0C0E080E2B2D98C2F0E94DF6AEA
:100EF0007801D7E080E2ABD9F70180809180A280B1
:100F0000B38020E030E0A901C501B4010E94A7EF41
:100F100087FD02C08BE29BD943E0C501B4010E946A
:100F2000EDB2D150FCE1EF0EF11CD111E3CF8AE01C
:100F30008ED9CF5F0C5F1F4FC730A9F68AE087D9E3
:100F4000DF91CF911F910F91FF90EF90BF90AF90E5
:100F50009F908F900895811105C08DE895E198D9F3
:100F60008AE075C981E995E1FACF86E895E190C9F3
:100F700080E895E18DC9811101C0FACF0895CF9322
:100F8000DF93C82F6FED77E10E9423C48C2FF3DF2E
:100F9000C5EBD2E14B855C856D857E8586ED97E15D
:100FA00099D920E030E543EC50E46F857889898950
:100FB0009A890E948BE7AB01BC0183ED97E18AD946
:100FC0002CEA35EC47E25EE36B897C898D899E894A
:100FD0000E948BE7AB01BC0180ED97E17BD98AE0F1
:100FE00036D9DF91CF9108950F931F93CF93DF935D
:100FF000C82F63EC77E10E943AC48C2FBCDF8AEBE8
:1010000097E146D980E00E94DF6ACAEED6E0088107
:10101000198187EB97E13CD9C8010E9412790A80B7
:10102000DB81C02D84EB97E133D9CE010E94127988
:101030008AE00DD9DF91CF911F910F910895B0E013
:10104000A0E0E5E2F8E80C9416EE61E083E50E948A
:101050002F6BC1E0C82768EB78E18C2F0E9423C476
:101060008C2F89DF80EB98E113D98FED9EE110D9A9
:101070008AE0EDD86EE978E18C2F0E9423C48C2F92
:101080007ADF81E898E104D98C2F0E9442C48C2F2A
:10109000ADDE8C2FD2DE8C2F89DE8C2F53DE65E304
:1010A00078E18C2F0E943AC4D091B3028CE298E18F
:1010B000EFD86D2F70E090E080E00E94A3B04091E7
:1010C000B4025091B5026091B6027091B7028BEEF6
:1010D0009CE200D98FE198E1DBD88091B3023BDF3D
:1010E00020E030E0A9016091840370918503809134
:1010F0008603909187030E9426E7882371F188EB8D
:10110000E82E82E0F82E10E0670100E08C2F33DF3C
:1011100087E798E1BDD8802F0E94DF6A84E798E1D5
:10112000B7D8812F0E94DF6A8BEE9CE2B1D8F6011E
:10113000608171818281938145E00E94EDB28AE0F5
:1011400086D80F5FFCE1CF0ED11C0730F9F61F5F88
:1011500084E0E80EF11C1730B9F68C2F45DF69E505
:1011600078E18C2F0E9423C40DE417E0D0E08C2F8F
:1011700002DF80E598E18CD88D2F0E94DF6AF801AC
:1011800060817181072E000C880B990B0E942CE75F
:10119000AB01BC018DE498E19DD8F80162817381B7
:1011A000072E000C880B990B0E942CE7AB01BC01A9
:1011B0008AE498E18FD8F801E480F58087E498E12B
:1011C00067D8C7010E9412798AE041D80A5F1F4F91
:1011D000D13059F48C2FD3DE8C2F84DD8C2F8BD81B
:1011E000CDB7DEB7E8E00C9432EED1E0C0CFCF93BC
:1011F00084E50E949367C0E08823D9F00E94056BC4
:10120000C82F1816B4F4B4DE8DE421D880912406DA
:10121000909125060E94127985EC98E139D86C2FBF
:10122000CC0F770B880B990B0E94A3B08AE00FD8E4
:10123000CFEF8C2FCF910895ACE1B0E0E2E2F9E876
:101240000C940CEE83E50E941C67182F882309F488
:101250001CC10E94206B8D83809175019091760155
:10126000A0917701B0917801898F9A8FAB8FBC8F55
:101270002091790130917A0140917B0150917C015C
:101280002D8B3E8B4F8B588F80917D0190917E01ED
:10129000A0917F01B09180018D879E87AF87B88B29
:1012A000112331F09D81911103C080E00E943777B6
:1012B00080911E0690911F06A0912006B0912106F4
:1012C00035E1B695A795979587953A95D1F79C0105
:1012D000AD01217033274427552729873A874B874B
:1012E0005C8720E030E0A901609184037091850360
:1012F00080918603909187030E9426E7882309F452
:10130000C8C083E40E941C67882309F493C00E942C
:101310004F6B698B7A8B8B8B9C8B48EB52E05F8396
:101320004E838A0157E05887412C512C98EC692E46
:1013300092EC792E812C912C28ECA22E22E4B22E54
:10134000312C212CF101EE0FFF1FEE0FFF1FE00FDC
:10135000F11FC080D180E280F380A7019601C50112
:10136000B4010E9426E7181614F446015701A7019C
:101370009601C301B2010E94A7EF87FF02C02601B8
:1013800037018FEF281A380A97E029163104D1F671
:10139000A885A150A887045E1F4FA111D1CFA3013A
:1013A0009201C501B4010E9444EE20E030E040E02B
:1013B0005FE30E948BE729893A894B895C890E9407
:1013C00044EE4B015C012DEB37E346E855EB0E9400
:1013D00026E787FD0AC02DEB37E346E855E3C50154
:1013E000B4010E94A7EF18162CF580E00E94377711
:1013F00017E0EE80FF8007E0F70161917191819124
:1014000091917F016F01F4E0CF1AD108A5019401F9
:101410000E9443EED6016D937D938D939C93139719
:10142000015051F71150EE81FF817C96FF83EE83CE
:101430001111DFCF89859A85AB85BC85892B8A2BD5
:101440008B2B79F020E030E0A9016091840370914A
:10145000850380918603909187030E9426E781117E
:1014600023DD8AE50E941C67882359F00E944F6B98
:1014700069837A838B839C8360E0CE0101960E940E
:10148000C3778D810E94377714C02091B3022D83DA
:10149000E3CEFD81F11108C029853A854B855C8535
:1014A000232B242B252BE9F263DD8CEE95E10E94A2
:1014B00048819D81992349F08091B302811105C033
:1014C00054DD8DEC95E10E94488152DD8FEB95E172
:1014D0000E9448818091B3023EDD4ADD82EB95E1B6
:1014E0000E944881C090B402D090B502E090B6024C
:1014F000F090B70220E030E0A901C701B6010E94D8
:10150000A7EF18160CF040C042E0C701B6010E94D8
:10151000EDB28DE00E9427818AE00E942781298D0B
:101520003A8D4B8D5C8D6091750170917601809143
:101530007701909178010E9426E781111FC02D89C3
:101540003E894F89588D6091790170917A0180911F
:101550007B0190917C010E9426E781110FC02091B0
:101560007D0130917E0140917F01509180016D8518
:101570007E858F8598890E9426E781110E94FC3E16
:101580006C96E2E10C9428EE8DEA95E10E94488188
:10159000C6CFCF93DF93EB010E944881BE01DD0FE0
:1015A000880B990B0E94A3B0DF91CF910895EC01B5
:1015B0008B01F42E0E942227209709F47AC0D8DCF0
:1015C000CE010E9448818AE00E9427810115110501
:1015D00011F40EE31CE20E94C06B1F930F93DF9384
:1015E000CF9380E595E19F938F9381E08F930E9445
:1015F000EE590E948846C0919713C695C69582E918
:1016000093E10E94566EDC2FDD0F1D2F1C0F8DB74E
:101610009EB707960FB6F8949EBF0FBE8DBF83E0AE
:101620000E941E6D4AE450E16C2F80E00E947E73A0
:101630001092CD13D093CE136FEF7FEF81E495E13D
:101640000E9421711092CD131093CE136FEF7FEF94
:1016500084E395E10E94217186E993E10E94B2D072
:101660008111DDCF82DC80E695E10E94488189EE20
:1016700093E0019739F000C00000EEE5F9E0319702
:10168000F0F7F7CFF89489EE93E0019739F000C0B6
:101690000000E6EEF3E03197F0F7F7CF0E94222743
:1016A000FF2021F00E94532BA895FECF0E940E2B05
:1016B000FBCF0115110511F40EE31CE2C7E5D5E1DE
:1016C0008ACF8091BE0D9091BF0D2FEF3FEF9817FD
:1016D00051F0E92FF0E0E254F24F228130E09F5FB9
:1016E0009F779093BF0DC90108951F920F920FB677
:1016F0000F9211240F900FBE0F901F9018951F92FC
:101700000F920FB60F9211240BB60F922F938F9357
:101710009F93EF93FF939091C6002091BF0DE091AE
:10172000BE0D81E08E0F8F77281729F0F0E0E2548C
:10173000F24F9283E82FE093BE0DFF91EF919F91BE
:101740008F912F910F900BBE0F900FBE0F901F9097
:1017500018958EBD0DB407FEFDCF08958FEF8EBD99
:101760000DB407FEFDCF8EB50895909164009B7F68
:1017700090936400982F906A96959CBD80FD03C05D
:1017800091E0863009F490E09DBD0895A8E0B0E0B6
:10179000ECECFBE80C940CEEB82E8091A70E843094
:1017A00008F0F6C131E6D32E8091A70E843008F000
:1017B00021C18091BE0D9091BF0D891B8F7709F4D7
:1017C00019C17FDF97FF0AC0D0DB80E894E10E9457
:1017D00048818091BE0D8093BF0DE6CF8A3019F00D
:1017E0008D3009F0FEC01092A60E8091440E9091AB
:1017F000450EFC01E05CF14F1682892B19F40E9422
:101800001D29D2CF1092450E1092440E06E41EE020
:10181000F8018191803209F446C08E3409F09DC0F0
:101820006BE774E1C8010E94A5E67C01892B41F0B9
:101830006EE470E0C80104960E945DF0009709F420
:10184000C8014AE050E070E060E001960E941AE4AE
:101850002B013C018091400E9091410EA091420ECF
:10186000B091430E0196A11DB11D481659066A0696
:101870007B0629F060E088E494E1EF2851F16AE208
:1018800070E0C8010E948CF09C01009729F1982F0C
:10189000901BF12C992349F09150F801E90FF11DAB
:1018A0008081F826F7CF8F01B3CF4AE050E070E097
:1018B00060E0C90101960E941AE42F2D30E050E04B
:1018C00040E0621773078407950751F060E089E2F2
:1018D00094E10E948DC368CF60E08FEF93E1F9CF70
:1018E0004092400E5092410E6092420E7092430E12
:1018F000809131078130E1F467E470E0C8010E9413
:101900005DF00097A9F04AE050E070E060E00196D9
:101910000E941AE4623071058105910548F48EE554
:1019200093E10E94488160E084E593E10E940B5AB4
:10193000F80180818D3481F58381823309F445C0BB
:10194000883301F1803341F58181843329F5828127
:10195000813311F50E94D83E1FC08091E81480FFAA
:10196000C7CF67EE7BE2C8010E94A5E6009731F081
:10197000FC01838180538A3008F0BACF60E085EDA6
:1019800093E1A7CF8281803339F48181813321F4BF
:1019900010926901109298028091460E8B3309F4DF
:1019A00003CF8091A70E843008F0FECE8091A90E5F
:1019B0008D9DC001112466E47EE08655914F0E9402
:1019C00068F080E00E944DC3EFCE8281813321F721
:1019D0008181813309F741E070E060E08AE49AE1B7
:1019E000E6DD24E43EE046E45EE066EA7EE00E9456
:1019F0009E66DACE8091E81483FDCAC082FFC8C01B
:101A000087FDC6C01A82198281E6F82E94E0E92E7D
:101A100029E6D22E8091A70E843008F0B9C00E942A
:101A2000D6668111B5C041E050E0BE016D5F7F4FC9
:101A30008EEC92E10E94C5D60B8110E0019711F067
:101A40000FEF1FEF8091D6129091D712A091D8126C
:101A5000B091D9128093E4149093E514A093E61406
:101A6000B093E7140E94D6660F3F100741F481112E
:101A700006C07BDA88E994E10E944881CBCF40918F
:101A8000A90E242F30E00A3061F00D3051F0882388
:101A900009F470C089819A81009719F001969A83A0
:101AA00089831092B00589819A81F29EF001F39E9C
:101AB000F00D1124E955F14FDF01A80FB91F13965E
:101AC0001C92892BA9F50E941D290E94D6668823A5
:101AD00009F4A0CF8EEC92E10E94BB228091DF142A
:101AE0008823F1F181508093DF148D9DC001112472
:101AF00062E08D58994F0E94CCD8E091DF1424E029
:101B0000E29FF0011124E159F94F40815181628136
:101B100073814093E4145093E5146093E61470933A
:101B2000E7148EEC92E10E94CAD50E940DD272CFCA
:101B30001A82198283818D3479F48481823361F42D
:101B40008581853349F4868180538A3028F08091DD
:101B5000E8148B7F8093E81481E00E944DC3B5CFD9
:101B60000E94FFD18091E81488608093E814E0928D
:101B7000310750CF4F9DA00111244655514F9E0172
:101B80002F5F3F4F60EB75E0802F0E949E6642CF33
:101B90000E94F7CD6B017C01BB2041F0C09227066B
:101BA000D0922806E0922906F0922A068091FE053E
:101BB0009091FF05A0910006B09101060097A10544
:101BC000B10529F140912706509128066091290618
:101BD00070912A06840F951FA61FB71FA7019601B3
:101BE000281B390B4A0B5B0BDA01C901B7FD0FC08B
:101BF000BCD9609194077091950787EA94E10E949F
:101C0000F1D140E070E060E090E080E0E9CE8091CA
